:100000000C94AA1A0C94DB1A0C94DB1A0C94DB1ACD
:100010000C94DB1A0C94DB1A0C94DB1A0C94DB1A8C
:100020000C94DB1A0C94DB1A0C94DB1A0C94DB1A7C
:100030000C94DB1A0C94DB1A0C94DB1A0C94DB1A6C
:100040000C94DB1A0C9480D10C94DB1A0C94DB1A00
:100050000C94DB1A0C94DB1A0C947DBE0C941DAA34
:100060000C94DB1A0C944B560C9441560C94DB1AEE
:100070000C94DB1A0C94DB1A0C94DB1A0C94DB1A2C
:100080000C9431340C94DB1A0C94DB1A0C94DB1AAC
:100090000C94DB1A0C94DB1A0C94DB1A0C94DB1A0C
:1000A0000C94DB1A0C94DB1A0C9403340C94DB1ABA
:1000B0000C94DB1A0C94DB1A0C94DB1A0C94DB1AEC
:1000C0000C94DB1A0C94DB1A0C94DB1A0C943F375B
:1000D0000C9409370C94DB1A0C94DB1A0C94DB1A81
:1000E0000C94DB1A084AD73B3BCE016E84BCBFFDA3
:1000F000C12F3D6C74319ABD56833DDA3D00C77FF8
:1001000011BED9E4BB4C3E916BAAAABE0000008090
:100110003F05A84CCDB2D44EB93836A9020C50B91F
:10012000918688083CA6AAAA2ABE000000803F004B
:100130000C943AFD0C94D1370C948FA40C94E55692
:100140000C9439FC0C9455FC0C94DBFC0C94F1A839
:100150000C94B8560C943DFC0C9451FC0D94550134
:100160000C9424FC0D94B90B0C94E1370C940338D7
:100170000C94DD370C9407570C9463FC0C947F446B
:100180000D9480010D949C1F0C94ADFC0C94A0FC6C
:100190000C94CA370C948B420C9459FC0C9430A9E3
:1001A0000C9430FD0C945FFC0D948E0C0C94BB37BA
:1001B0000D94E20B0D94CE0F0C94F8440D94190C91
:1001C0000D94870F0C9433FC0C94D3FC0C94E537FE
:1001D0000C94F3A70C9443FC0D94A10C0C94534481
:1001E0000D942D0C0D94B5090C9412FD0C94F9FC92
:1001F0000C94E9370C9428FC0C94C1FC0D94FC037E
:100200000D947D050D9461140D948A110C9473A8BE
:100210000C94D9370C94AC370C9412A50C940F574E
:100220000D9420080C9430FC0C947D370C9441FF05
:100230000C9412FC0D94DB0F0D94850A0D94500D57
:100240000D94A20F0D9499090C9403A90D945A0FC3
:100250000D946B000C940DFC0C94E1560C94D65646
:100260000D94B7100D948A0F0C94C0440D94BA1FCE
:100270000C9458A80C94C7560D94F60B0D94EB02F1
:100280000D94E9090D94C7100C94FC560C94FAA92E
:100290000C9411A50C9414A80D94B00F0D944B0B55
:1002A0000C94CBFC0D94BA0F0D9466090C9408FDC8
:1002B0000C9447FC0C94F5560C94E5FC0C94A8FCAB
:1002C0000D944C0C0C9489560C941CFD0D94150B3C
:1002D0000C94DD560D94810F0C945EA70C9487420C
:1002E0000C94ED560C94D5370C9426FD0C94F156D5
:1002F0000C94EFFC0C94F0370C94FB370C947BA718
:100300000C94E9560C944BFC0C94B7FC0C943842BA
:100310000C942CFC4E414E494E495459494E46CD01
:10032000CCCC3D0AD7233C17B7D13877CC2B3295AC
:1003300095E6241FB14F0A000020410000C842008A
:10034000401C4620BCBE4CCA1B0E5AAEC59D740054
:10035000407A10F35A00A0724E18090010A5D4E894
:100360000000E87648170000E40B54020000CA9A27
:100370003B000000E1F50500008096980000004079
:10038000420F000000A086010000001027000000BE
:1003900000E803000000006400000000000A000004
:1003A0000000000100000000002C76D888DC674FB8
:1003B0000823DFC1DFAE59E1B1B796E5E3E453C6E8
:1003C0003AE651997696E8E6C28426EB898C9B62E0
:1003D000ED407C6FFCEFBC9C9F40F2BAA56FA5F48A
:1003E00090055A2AF75C936B6CF9676DC11BFCE0B2
:1003F000E40D47FEF520E6B500D0ED902E03009405
:100400003577050080841E080000204E0A00000099
:10041000C80C333333330F986E12831141EF8D21A3
:1004200014893BE65516CFFEE6DB18D1844B381B0A
:10043000F77C1D901DA4BBE424203284725E2281CF
:1004400000C9F124ECA1E53D27434F4D4D554E49E0
:10045000434154494F4E0044525952554E00455263
:10046000524F525300494E464F004543484F0045B6
:1004700072726F722077726974696E6720746F2070
:10048000454550524F4D210A0053544F505045445A
:100490002E20005072696E7465722073746F7070D4
:1004A00065642064756520746F206572726F727365
:1004B0002E2046697820746865206572726F7220FC
:1004C000616E6420757365204D39393920746F2051
:1004D000726573746172742E202854656D70657234
:1004E00061747572652069732072657365742E205E
:1004F0005365742069742061667465722072657337
:1005000074617274696E67290A004E6F20436865D2
:10051000636B73756D2077697468206C696E6520F4
:100520006E756D6265722C204C617374204C696E1F
:10053000653A20004E6F20436865636B73756D20CC
:1005400077697468206C696E65206E756D6265727E
:100550002C204C617374204C696E653A20006368EE
:1005600065636B73756D206D69736D617463682C61
:10057000204C617374204C696E653A20004C696EA2
:1005800065204E756D626572206973206E6F7420F0
:100590004C617374204C696E65204E756D62657296
:1005A0002B312C204C617374204C696E653A20000D
:1005B0004D3131300053657269616C207374617420
:1005C0007573206D69736D617463680A0077616982
:1005D000740A0053442072656164206572726F7200
:1005E0000A002121204B494C4C20636175736564DE
:1005F00020627920746F6F206D75636820696E6169
:1006000063746976652074696D65202D2063757249
:1006100072656E7420636F6D6D616E643A20004880
:100620006F74656E642049646C652054696D656FF4
:10063000757400486F74656E642049646C6520545D
:10064000696D656F75740A003D3D6F6E46696C613A
:100650006D656E7452756E6F75743D3D0070617599
:100660007365004D363030002066696C616D656ED3
:10067000745F72756E6F7574200066696C616D656C
:100680006E745F72756E6F757420540046696C618C
:100690006D656E7452756E6F75742054002A2A2A27
:1006A000496E6974696E67206361726420697320A2
:1006B0004F4B2A2A2A004D6564696120496E736593
:1006C00072746564004D656469612052656D6F7672
:1006D0006564004D313030305300627573793A20D3
:1006E00070617573656420666F7220696E707574D1
:1006F0000A00627573793A207061757365642066CB
:100700006F7220757365720A00627573793A207092
:10071000726F63657373696E670A002A2A2A6B69B0
:100720006C6C2A2A2A00706F7765726F6666004BC0
:10073000494C4C45442E20005072696E74657220FD
:1007400068616C7465642E206B696C6C2829206369
:10075000616C6C6564210A0053544F505045442E1F
:1007600020005072696E7465722073746F707065CA
:10077000642064756520746F206572726F72732EC9
:100780002046697820746865206572726F722061F6
:100790006E6420757365204D39393920746F20726D
:1007A0006573746172742E202854656D7065726172
:1007B000747572652069732072657365742E205399
:1007C0006574206974206166746572207265737443
:1007D000617274696E67290A006563686F3A004543
:1007E00072726F723A0042696C696E656172204C78
:1007F0006576656C696E6720477269643A0A002104
:10080000212053544F502063616C6C6564206265F5
:100810006361757365206F6620424C546F75636821
:10082000206572726F72202D20726573746172740C
:100830002077697468204D3939390A002121205305
:10084000544F502063616C6C656420626563617510
:100850007365206F6620424C546F75636820657223
:10086000726F72202D2072657374617274207769C3
:100870007468204D3939390A002F2F616374696F0C
:100880006E3A0070726F6D70745F00656E64005335
:10089000656E64204D31303820746F207265737539
:1008A0006D650A00496E736572742066696C616DCE
:1008B000656E7420616E642073656E64204D313006
:1008C000380A005265686561742066696E697368EC
:1008D00065642E0052656865617420446F6E650022
:1008E000526568656174696E672E2E2E00526568C8
:1008F000656174004865617465722054696D656F47
:1009000075740053656E64204D31303820746F204B
:1009100068656174206E6F7A7A6C650A004E6F7A32
:100920007A6C65205061726B656400486F74656E07
:100930006420746F6F20636F6C640A00706175735C
:1009400065640050617573650044697361626C652C
:1009500052756E6F75740050757267654D6F726574
:10096000005061757365640073686F770062757419
:10097000746F6E00626567696E004C6F616420463B
:10098000696C616D656E74004C6F61642046696CC2
:10099000616D656E74205400496E736572742066D3
:1009A000696C616D656E7420616E642073656E6440
:1009B000204D3130380A00726573756D65640052E0
:1009C0006573756D696E670057616974696E67203C
:1009D000666F72206865617475702E0A004C6561DF
:1009E00076696E6720473236003F537065636966EB
:1009F00069656420582C5920636F6F7264696E6159
:100A00007465206F7574206F6620626F756E6473F5
:100A10002E0A003F28522965706561742076616C4A
:100A20007565206E6F7420706C61757369626C659A
:100A30003B206D757374206265206174206C656164
:100A4000737420312E0A003F285229657065617445
:100A5000206D7573742062652073706563696669C3
:100A60006564207768656E206E6F74207573696E9B
:100A70006720616E204C43442E0A003F537065632B
:100A80006966696564206E6F7A7A6C652074656D3D
:100A90007065726174757265206E6F7420706C6120
:100AA000757369626C652E0A003F537065636966F1
:100AB0006965642066696C616D656E742073697A1E
:100AC00065206E6F7420706C61757369626C652E41
:100AD0000A003F53706563696669656420707269D6
:100AE0006D65206C656E677468206E6F7420706C25
:100AF00061757369626C652E0A003F5072696D659D
:100B0000206C656E677468206D7573742062652053
:100B1000737065636966696564207768656E206EC9
:100B20006F74207573696E6720616E204C43442E8C
:100B30000A003F537065636966696564206E6F7A69
:100B40007A6C652073697A65206E6F7420706C61B1
:100B5000757369626C652E0A003F52657472616339
:100B600074696F6E204D756C7469706C6965722064
:100B70006D7573742062652073706563696669655D
:100B8000642E0A003F53706563696669656420528C
:100B9000657472616374696F6E204D756C746970F1
:100BA0006C696572206E6F7420706C617573696218
:100BB0006C652E0A003F5370656369666965642041
:100BC0006C6179657220686569676874206E6F74FE
:100BD00020706C61757369626C652E0A0043292E62
:100BE0000A003F53706563696669656420626564E5
:100BF0002074656D7065726174757265206E6F74B6
:100C000020706C61757369626C65202834302D002A
:100C1000473236207374617274696E672E2E2E0A05
:100C2000004F46460A00466164652048656967686A
:100C3000742000426564204C6576656C696E67209F
:100C4000004661696C656420746F20656E61626C3A
:100C50006520426564204C6576656C696E670A00A4
:100C6000496E76616C6964206D6573682E0A005068
:100C7000726F62696E6720506F696E740025532031
:100C800025692F2569002E0A002F0050726F6269B6
:100C90006E67206D65736820706F696E7420002028
:100CA0002844525952554E29004732392041757413
:100CB0006F20426564204C6576656C696E67003F05
:100CC00020284C2C522C462C4229206F7574206F02
:100CD0006620626F756E64732E0A003F2856296580
:100CE00072626F7365206C6576656C20696D706CDF
:100CF00061757369626C652028302D34292E0A00D5
:100D0000426164205A2076616C75650A004E6F203E
:100D100062696C696E65617220677269640A004479
:100D20006576696174696F6E0025533A20257300FA
:100D300046696E6973686564210A003A207A3A2030
:100D400000206F662000476F696E6720746F3A203D
:100D5000580043570A00206469723A0020616E67A8
:100D60006C653A00537461727420726164697573C2
:100D70003A004D343820506F696E740025533A2084
:100D800025642F256400506F736974696F6E696EF6
:100D900067207468652070726F62652E2E2E0A00BF
:100DA0003F4C656773206F66206D6F76656D656E6D
:100DB0007420696D706C61757369626C6520283090
:100DC0002D3135292E0A003F2028582C5929206F13
:100DD0007574206F6620626F756E64732E0A005002
:100DE000726F6265206F7574206F6620626F756E1A
:100DF0006473003F53616D706C652073697A652080
:100E00006E6F7420706C61757369626C6520283434
:100E10002D3530292E0A004D3438205A2D50726F4E
:100E20006265205265706561746162696C6974798C
:100E300020546573740A003F2856296572626F73E7
:100E400065206C6576656C20696D706C6175736981
:100E5000626C652028302D34292E0A005374616E8F
:100E60006461726420446576696174696F6E3A20CA
:100E7000002052616E67653A2000204D61783A206B
:100E800000204D696E3A2000205369676D613A2059
:100E9000004D65616E3A20005741524E494E472140
:100EA000204C6F77205A204A65726B206D61792043
:100EB0006C65616420746F20756E77616E74656413
:100EC000207061757365732E0A004F4646004F4EC1
:100ED0000020204D61783A2000200020204D696ECE
:100EE0003A2000536F667420656E6473746F70737C
:100EF0003A20003D3D4F6E506F7765724C6F7373B3
:100F0000526573756D653D3D004D32342053256C3F
:100F1000642054256C64004739322E3920452573EE
:100F200000473120462564004739322E39205A25A2
:100F300073004731205A302046323030004731208C
:100F400058257320592573204633303030004D34F6
:100F5000323020532569205A2573004D3130362018
:100F600050256920532569004D32303020442573C7
:100F70000047323852305859004739322E3920450F
:100F800030205A300A47315A2573004D313039200C
:100F9000532569004D31393020532569004D3432D5
:100FA00030205330205A300020496E76616C6964DD
:100FB000206578747275646572200047322F47335C
:100FC0002062616420706172616D65746572730A7C
:100FD00000536C6565702E2E2E005A2050726F6281
:100FE000652050617374204265640A005A20507273
:100FF0006F62652050617374204265640047323827
:101000004C30004D3131372050726F62652066617F
:10101000696C65642E0A4732380A0070726F626527
:101020005F72657769706500473239205265747266
:1010300079696E670050726F62696E6720466169F8
:101040006C6564004D31313720426564206C6576F3
:10105000656C696E67206661696C65642E0A47304D
:10106000205A31300A4D3330302050323520533839
:1010700038300A4D333030205035302053300A4D4F
:101080003330302050323520533838300A4D333029
:1010900030205035302053300A4D3330302050321C
:1010A0003520533838300A4D333030205035302019
:1010B00053300A47342053310070726F62655F66A7
:1010C00061696C6564004D31313720426564206C84
:1010D0006576656C696E6720646F6E652E00205AB8
:1010E0003A200020593A200042656420583A2000F6
:1010F0004D65736820706F696E74206F7574206F12
:10110000662072616E67650A004D302053746F70FF
:10111000004D312053746F7000436F6E74696E75AB
:101120006500436C69636B20746F20526573756D45
:10113000652E2E2E004E6F204D6F76652E00456E6B
:10114000642066696C65206C6973740A0042656787
:10115000696E2066696C65206C6973740A004E6F55
:10116000206D656469610A00526573756D696E670B
:1011700020534400286E6F2066696C652900437512
:101180007272656E742066696C653A2000507269EF
:101190006E742074696D653A20000A53746174732B
:1011A0003A2046696C616D656E7420757365643AAA
:1011B00020002C204C6F6E67657374206A6F623A52
:1011C0002000546F74616C2074696D653A2000537F
:1011D000746174733A20002C204661696C65643A2E
:1011E00020002C2046696E69736865643A200050BF
:1011F00072696E74733A200053746174733A2000FC
:10120000436F6F6C696E672E2E2E0048656174699E
:101210006E672E2E2E0045202553006F6B006F66E3
:1012200066006A0465045E04570449044445425557
:10123000473A004D31313320530042656420436FFB
:101240006F6C696E672E2E2E0042656420486561C2
:1012500074696E672E2E2E00544D3344204D6178F4
:10126000204F46462E002F2F002052004163636519
:101270006C65726174696F6E3A2050004D32303681
:1012800020580046523A0020466C6F773A20003AC8
:10129000200020536572766F2000206F7574206FD8
:1012A000662072616E67650A00536572766F200072
:1012B00020643A0020693A0020703A00496E766155
:1012C0006C69642065787472756465720A002064C4
:1012D0003A0020693A0020703A0064697300656E34
:1012E0000043290A0061626C656420286D696E20E4
:1012F00074656D702000436F6C642065787472753E
:101300006465732061726520005049442041757402
:101310006F74756E6500504944204175746F747523
:101320006E65206661696C65642120426164206895
:1013300065617465722069640A0046696C616D6557
:101340006E742072756E6F75742064697374616E4B
:10135000636520286D6D293A200046696C616D65D2
:101360006E742072756E6F757420004D34323120AA
:10137000696E636F727265637420706172616D650E
:101380007465722075736167650A004D6573682026
:10139000706F696E74206F7574206F662072616E55
:1013A00067650A004F666673657473204170706CE0
:1013B000696564004572723A20546F6F20666172ED
:1013C0002100546F6F206661722066726F6D20720B
:1013D00065666572656E636520706F696E740A007C
:1013E000454550524F4D204F4B0A00506F77657264
:1013F0002D6C6F7373207265636F76657279200050
:101400004D383400446F6E65207072696E74696E79
:10141000672066696C650A004D3737004D3331002F
:101420004361703A004D4541545041434B00434F96
:101430004F4C45525F54454D5045524154555245CD
:10144000004348414D4245525F54454D504552413D
:101450005455524500424142595354455050494E0B
:10146000470041524353004D4F54494F4E5F4D4F3B
:1014700044455300544845524D414C5F50524F54DF
:10148000454354494F4E004C4F4E475F46494C45EB
:101490004E414D45004155544F5245504F52545FB7
:1014A00053445F5354415455530053445F5752497A
:1014B0005445005245504541540053444341524421
:1014C0000050524F4D50545F535550504F5254009E
:1014D000454D455247454E43595F50415253455241
:1014E00000434153455F4C494748545F4252494786
:1014F00048544E45535300544F47474C455F4C4961
:101500004748545300534F4654574152455F504F3C
:10151000574552004255494C445F50455243454E51
:1015200054004C4556454C494E475F444154410098
:101530005A5F50524F42450052554E4F555400414C
:1015400055544F4C4556454C005052494E545F4AF5
:101550004F420050524F4752455353004155544F4C
:101560005245504F52545F54454D5000564F4C55C4
:101570004D455452494300454550524F4D00424954
:101580004E4152595F46494C455F5452414E534675
:1015900045520053455249414C5F584F4E5F584F9A
:1015A0004646004649524D574152455F4E414D45D2
:1015B0003A4D61726C696E20322E302E375F44577F
:1015C000372E332E3120544D33442035534D444271
:1015D000422028417072203239203230323120319D
:1015E000333A34363A31322920534F555243455F0E
:1015F000434F44455F55524C3A68747470733A2FA8
:101600002F6769746875622E636F6D2F496E736101
:101610006E6974794175746F6D6174696F6E2F4D69
:1016200061726C696E2F747265652F437265616CAF
:101630006974794477696E5F322E302050524F546E
:101640004F434F4C5F56455253494F4E3A312E301F
:10165000204D414348494E455F545950453A544DF9
:101660003344204D61782045585452554445525FCB
:10167000434F554E543A3120555549443A636564B9
:1016800065326132662D343161322D343734382D74
:10169000396231322D63353563363266333637661B
:1016A000660A0050726F6265204F6666736574202B
:1016B0005A0050726F6265204F6666736574205AD7
:1016C00000290A0020746F20003F5A206F75742093
:1016D0006F662072616E6765202800290A002074F9
:1016E0006F20003F59206F7574206F662072616E05
:1016F000676520282D00290A0020746F20003F58BC
:10170000206F7574206F662072616E676520282DCA
:101710000050726F6265204F6666736574205800D2
:1017200043616E6E6F74206F70656E2073756264B6
:10173000697220002569730025696D202569730091
:101740002569682025696D20256973002569642055
:101750002569682025696D20256973002569792030
:10176000256964202569682025696D202569730035
:101770003D3D4477696E20496E697420436F6D70FA
:101780006C6574653D3D002A2A2A4E6F7A7A6C6535
:1017900054656D705374617475735B325D203D00E8
:1017A0003D3D48656174696E6720446F6E652043F6
:1017B00068616E67652046696C616D656E743D3D5C
:1017C000002020737461727470726F677265737336
:1017D00020003D3D7761697477617920353D3D009A
:1017E0003D3D7761697477617920343D3D003D3D31
:1017F0007761697477617920333D3D003D3D7761C4
:10180000697477617920313D3D003D3D6F6E5072C6
:10181000696E7454696D657253746F707065643D60
:101820003D003D3D6F6E466163746F727952657322
:1018300065743D3D00270A0A000027202700202765
:10184000002D006E6F74696669636174696F6E2044
:101850000063616E63656C005072696E7420416252
:101860006F72746564004469736D697373005549E0
:101870002041626F7274656400726573756D6500F6
:101880004D3234002A2A2A43506C617920546F6EFD
:10189000652A2A2A003D3D6F6E5072696E74546944
:1018A0006D65725061757365643D3D00486F6D698B
:1018B0006E67204661696C6564006F70656E0054E8
:1018C0005249474745524544003A200066696C61D9
:1018D0006D656E74007A5F6D696E00795F6D696E1B
:1018E00000785F6D696E005265706F7274696E6723
:1018F00020656E6473746F70207374617475730AFD
:101900000020746F6F206C6F6E672065787472753D
:1019100073696F6E2070726576656E7465640A0017
:1019200020636F6C6420657874727573696F6E20C4
:1019300070726576656E7465640A00486F6D652027
:10194000257325732573204669727374005761727D
:101950006E696E673A20486F6D696E672042756DDB
:10196000702044697669736F72203C20310A00024E
:101970000204000000000000000000000000000061
:10198000E1430000E1430000EB43000000410000A0
:10199000004100000040FFFFFF00000001000000C8
:1019A00001000080005555550000004000333333DE
:1019B00000AAAA2A004992240000002000C7711C36
:1019C0000099991900D1451700555515003BB113E1
:1019D000002449120011111100000010000F0F0F18
:1019E00000E3380E0043790D00CCCC0C00C3300C62
:1019F00000E8A20B0064210B00AAAA0A00703D0AAD
:101A0000009DD80900427B090092240900DCD3081C
:101A100000888808001042080000000800F0C10794
:101A2000008787070075500700711C07003EEB0612
:101A300000A1BC06006990060066660600703E06BE
:101A4000006118060017F4050074D105005BB005AD
:101A500000B2900500627205005555050078390501
:101A600000B81E0500050505004EEC040087D404EF
:101A700000A1BD040090A7040049920400C17D04A8
:101A800000EE690400C7560400444404005C3204BC
:101A9000000821040041100400000004003FF0038E
:101AA00000F8E0030026D20300C3C30300CCB50353
:101AB000003AA803000A9B0300388E0300C081038C
:101AC000009F750300D0690300505E03001D53039F
:101AD0000034480300913D0300333303001629030B
:101AE00000381F030097150300300C0300030303A5
:101AF000000BFA020049F10200BAE802005CE002C1
:101B0000002DD802002DD0020059C80200B0C0023A
:101B10000031B90200DAB10200AAAA0200A0A302B1
:101B200000BC9C0200FA9502005C8F0200DF880274
:101B30000082820200457C020027760200277002A4
:101B400000436A02007C640200D05E02003F59023A
:101B500000C8530200FFFDFCFAF8F6F4F2F0EEECD8
:101B6000EAE9E7E5E3E1E0DEDCDAD9D7D5D4D2D0A3
:101B7000CFCDCBCAC8C7C5C3C2C0BFBDBCBAB9B739
:101B8000B6B4B3B2B0AFADACAAA9A8A6A5A4A2A1A1
:101B9000A09E9D9C9A99989795949392908F8E8DE4
:101BA0008B8A8988878684838281807F7E7D7B7A09
:101BB000797877767574737271706F6E6D6C6B6A0D
:101BC000696867666564636261605F5E5D5C5B5AFD
:101BD0005958585756555453525150504F4E4D4CDA
:101BE0004B4A4A4948474646454443424241403FA2
:101BF0003E3E3D3C3B3B3A39383837363535343359
:101C000032323130302F2E2E2D2C2B2B2A29292801
:101C1000272726252524232322212120201F1E1E9D
:101C20001D1C1C1B1B1A191918181716161515142C
:101C3000131312121111100F0F0E0E0D0D0C0C0BB1
:101C40000A0A09090808070706060505040403032C
:101C500002020100003D3D6F6E5072696E7454695E
:101C60006D6572537461727465643D3D000000E1FE
:101C7000430000E1430000EB4300000000000000CF
:101C800000000000003D3D6F6E53746F7265536538
:101C90007474696E67733D3D003D3D6F6E436F6EBA
:101CA00066696775726174696F6E53746F72655798
:101CB00072697474656E3D3D0053657474696E6736
:101CC000732053746F726564000A20696E69742012
:101CD0007A70726F62655F7A6F6666736574203DB5
:101CE00020003D3D6F6E436F6E666967757261746B
:101CF000696F6E53746F7265526561643D3D004556
:101D00004550524F4D20496E697469616C697A651E
:101D1000640A003B20003A0A0020204D3630332070
:101D20000020440020204D34313220530046696C9D
:101D3000616D656E742072756E6F75742073656E5B
:101D4000736F723A002055004C0046696C616D65F6
:101D50006E74206C6F61642F756E6C6F6164206CA3
:101D6000656E677468733A0020204D38353120580D
:101D7000005A2D50726F6265204F6666736574005D
:101D800020204D343133205300506F7765722D4C35
:101D90006F7373205265636F766572793A002044E1
:101DA0000020490020204D333034205000204400D2
:101DB00020490020204D333031205000504944202C
:101DC00073657474696E67733A00204A0020204777
:101DD0003239205720490020204D34323020530022
:101DE0004175746F20426564204C6576656C696E40
:101DF000673A0020204D323036205800486F6D651C
:101E0000206F66667365743A0020580020530020E6
:101E1000204D323035204200416476616E63656446
:101E20003A20423C6D696E5F7365676D656E745FE5
:101E300074696D655F75733E20533C6D696E5F66B6
:101E4000656564726174653E20543C6D696E5F74B3
:101E5000726176656C5F66656564726174653E206B
:101E6000583C6D61785F785F6A65726B3E20593CC3
:101E70006D61785F795F6A65726B3E205A3C6D6177
:101E8000785F7A5F6A65726B3E20453C6D61785F72
:101E9000655F6A65726B3E0020540020520020206E
:101EA0004D323034205000416363656C657261745B
:101EB000696F6E2028756E6974732F7332293A200A
:101EC000503C7072696E745F616363656C3E205252
:101ED0003C726574726163745F616363656C3E201C
:101EE000543C74726176656C5F616363656C3E003F
:101EF00020204D3230312058004D6178696D756D6C
:101F000020416363656C65726174696F6E2028752A
:101F10006E6974732F7332293A0020204D323033AA
:101F20002058004D6178696D756D20666565647235
:101F3000617465732028756E6974732F73293A0074
:101F400053746570732070657220756E69743A0001
:101F500020440020204D323030205300204469734B
:101F600061626C65640A0046696C616D656E74201F
:101F700073657474696E67733A0020286D6D29006B
:101F80002020473231202020203B20556E69747379
:101F900020696E206D6D003D3D6F6E4C6F61645326
:101FA000657474696E67733D3D000000FA4300007C
:101FB000C84300007041000096420000A0420000AB
:101FC000A0420000C84300000C43E8030000BC022C
:101FD0000000640000004B00000024F4D43050C323
:101FE0008E20C2A24017828B7011127A910D816CE3
:101FF000D90AA861E108C7586607615143061E4B1C
:102000005D05C145A7041A411104093D98037139C2
:1020100031034036DB0265339102D4305402802E06
:102020001D02632CEE01752AC501B028A0011027FE
:1020300081018F2564012B244B01E0223401AC2166
:102040001F018D200D01801FFC00841EED00971DD7
:10205000DF00B81CD200E61BC600201BBC00641ABF
:10206000B200B219A8000A19A0006A189900D11785
:10207000910040178B00B516840031167E00B31511
:1020800079003A157300C7146F0058146A00EE13F4
:1020900066008813630025135E00C7125B006C1294
:1020A000570015125400C111510070114F00211139
:1020B0004B00D61049008D10470046104400021016
:1020C0004200C00F4000800F3E00420F3C00060F50
:1020D0003B00CB0E3800930E37005C0E3500270E08
:1020E0003400F30D3200C10D3100900D3000600D51
:1020F0002E00320D2D00050D2C00D90C2B00AE0C3E
:102100002900850C29005C0C2700350C27000E0CDB
:102110002600E80B2400C40B2400A00B23007D0B39
:1021200023005A0B2100390B2100180B2000F80A5C
:102130001F00D90A1E00BB0A1E009D0A1D00800A4E
:102140001D00630A1C00470A1B002C0A1B00110A11
:102150001A00F7091A00DD091900C4091900AB09B2
:102160001900920917007B091800630917004C0930
:10217000160036091600200916000A091500F50890
:102180001500E0081400CC081400B8081400A408D6
:102190001400900813007D0812006B081300580803
:1021A000120046081200340811002308110012081A
:1021B000110001081100F0071000E0071000D0071F
:1021C0001000C0071000B0070F00A1071000910712
:1021D0000E0083070F0074070F0065070E005707F6
:1021E0000E0049070E003B070D002E070E002007CA
:1021F0000D0013070D0006070D00F9060C00ED0693
:102200000D00E0060C00D4060C00C8060C00BC064D
:102210000C00B0060C00A4060B0099060C008D06FD
:102220000B0082060B0077060B006C060B006106A4
:102230000A0057060B004C060A0042060A00380640
:102240000A002E060A0024060A001A060A001006D2
:10225000090007060A00FD050900F4050900EB0561
:102260000900E2050900D9050900D0050900C705E4
:102270000900BE050900B5050800AD050800A50563
:1022800009009C050800940508008C0508008405D9
:1022900008007C050800740508006C05070065054A
:1022A00008005D050700560508004E0507004705B4
:1022B00007004005080038050700310507002A051A
:1022C0000700230507001C050600160507000F057B
:1022D00007000805060002050700FB040600F504D8
:1022E0000700EE040600E8040600E2040700DB0431
:1022F0000600D5040600CF040600C9040600C30486
:102300000600BD040600B7040600B1040500AC04D5
:102310000600A6040600A00405009B040600950420
:102320000500900406008A04050085040500800469
:1023300006007A04050075040500700405006B04AE
:10234000050066040500610405005C0405005704EF
:102350000500520405004D0405004804050043042F
:1023600005003E0404003A0405003504050030046D
:1023700004002C04050027040400230405001E04A7
:1023800004001A04040016040500110404000D04DE
:102390000400090405000404040000040400FC0314
:1023A0000400F8030400F4030400F0030400EC0349
:1023B0000400E8030400E4030400E0030400DC0379
:1023C0000400D8030400D4030400D0030400CC03A9
:1023D0000400C8030300C503030024F404D9201B30
:1023E000C40C5C0E9804C4095F0265077101F40512
:1023F000F900FB04B30048048700C10369005803D7
:10240000550003034500BE023A0084023100530226
:102410002A002902250004022000E4011C00C80152
:102420001900AF0117009801140084011300710115
:1024300010006101100051010E0043010D00360132
:102440000B002B010B0020010B00150109000C01F2
:10245000090003010800FB000800F3000800EB007E
:102460000700E4000600DE000600D8000600D200E7
:102470000600CC000500C7000500C2000500BD0035
:102480000400B9000400B5000400B1000400AD0070
:102490000400A9000400A5000300A20003009F009F
:1024A00004009B00030098000300950002009300C5
:1024B0000300900003008D0002008B0003008800E1
:1024C00002008600020084000300810002007F00F9
:1024D00002007D0002007B0002007900020077000C
:1024E0000100760002007400020072000100710019
:1024F00002006F0002006D0001006C0002006A0023
:10250000010069000200670001006600010065002B
:10251000010064000200620001006100010060002F
:1025200001005F0002005D0001005C0001005B0033
:1025300001005A0001005900010058000100570035
:102540000100560001005500010054000100530035
:102550000000530001005200010051000100500032
:1025600001004F0001004E0000004E0001004D0030
:1025700001004C0001004B0000004B0001004A002C
:102580000100490001004800000048000100470028
:102590000100460000004600010045000000450023
:1025A000010044000100430000004300010042001C
:1025B0000000420001004100000041000100400015
:1025C00001003F0000003F0001003E0000003E000F
:1025D00001003D0000003D0001003C0000003C0007
:1025E00000003C0001003B0000003B0001003A00FD
:1025F00000003A00010039000000390001003800F5
:1026000000003800000038000100370000003700EB
:1026100001003600000036000000360001003500E1
:1026200000003500000035000100340000003400D7
:1026300000003400010033000000330000003300CC
:1026400001003200000032000000320001003100C1
:1026500000003100000031000100300000003000B7
:102660000000300001002F0000002F0000002F00AC
:1026700000002F0001002E0000002E0000002E00A0
:1026800001002D0000002D0000002D0000002D0095
:1026900001002C0000002C0000002C0000002C0089
:1026A00001002B0000002B0000002B0000002B007D
:1026B00001002A0000002A0000002A0000002A0071
:1026C0000100290000002900000029000000290065
:1026D0000000290001002800000028000000280058
:1026E000000028000000280001002700000027004B
:1026F000000027000000270000002700010026003E
:102700000000260000002600000026000000260031
:102710000100250000002500000025000000250024
:102720000000250000002500010024000000240016
:102730000000240000002400000024000100230009
:1027400000002300000023000000230000002300FD
:1027500000002300000023000100220000002200EE
:1027600000002200000022000000220000002200E1
:1027700001002100000021000000210000002100D4
:1027800000002100000021000000210001002000C5
:1027900000002000000020000000200000002000B9
:1027A00000002000000020000000200001001F00A9
:1027B00000001F0000001F0000001F0000001F009D
:1027C00000001F0000001F0001001E0000001E008E
:1027D00000001E0000001E000000393000003325FC
:1027E000000087190000B00F0000DB080000BD04E6
:1027F0000000740200003F01000020436F756E74FA
:1028000020583A0023646566696E65204445464158
:10281000554C545F0000626564004B6420004B69B6
:1028200020004B702000504944204175746F74752E
:102830006E652066696E69736865642120507574E1
:1028400020746865206C617374204B702C204B6978
:1028500020616E64204B6420636F6E7374616E74CC
:10286000732066726F6D2062656C6F7720696E747D
:102870006F20436F6E66696775726174696F6E2E43
:10288000680A00504944204175746F74756E652064
:102890006661696C6564212074696D656F75740A81
:1028A00000504944204175746F74756E65206661EF
:1028B000696C6564212054656D7065726174757210
:1028C0006520746F6F20686967680A00204B643A5E
:1028D0002000204B693A2000204B703A2000204312
:1028E0006C617373696320504944200A00204E6F65
:1028F000206F76657273686F6F740A002054753AA2
:102900002000204B753A2000206D61783A2000208D
:102910006D696E3A200020643A200020626961737C
:102920003A2000504944204175746F74756E6520DB
:1029300073746172740A00504944204175746F7455
:10294000756E65206661696C6564212054656D70E3
:102950006572617475726520746F6F20686967684D
:102960000A0042656400453100626564002C2073F2
:10297000797374656D2073746F707065642120487D
:1029800065617465725F49443A2000486561746905
:102990006E67204661696C65640048656174696EA4
:1029A00067206661696C6564004D3131322053687F
:1029B0007574646F776E001000C90210012C01401D
:1029C00001220170011801B0010E01F00104015053
:1029D00002FA00B002F0003003E600D003DC009001
:1029E00004D2007005C800A006BE000008B400B004
:1029F00009AA00D00BA000600E960060118C0000A8
:102A000015820020197800C01D6E00A0226400B05D
:102A1000275A00902C500000314600E0343C001052
:102A2000383200903A2800603C1E00A03D1400801F
:102A30003E0A00203F0000544845524D414C205270
:102A4000554E4157415900546865726D616C205272
:102A5000756E61776179004572723A204D41585424
:102A6000454D50004D415854454D50207472696792
:102A70006765726564004572723A204D494E54454F
:102A80004D50004D494E54454D5020747269676752
:102A90006572656400202F002042403A0020403AD1
:102AA0000020573A0020573A00496E76616C6964FD
:102AB0002065787472756465720A007C3C3E5E2BFA
:102AC0003D3F2F5B5D3B2C2A225C0043616E6E6FA5
:102AD00074206F70656E2073756264697220005394
:102AE0004420496E6974204661696C005344206338
:102AF000617264206F6B0A006F70656E526F6F7445
:102B0000206661696C65640A00766F6C756D652E70
:102B1000696E6974206661696C65640A004E6F2095
:102B2000534420636172640A000A4D3234004D320E
:102B300033202573002E0A006F70656E2066616970
:102B40006C65642C2046696C653A200046696C65AA
:102B50002073656C65637465640A002053697A6547
:102B60003A200046696C65206F70656E65643A2096
:102B700000454E4420535542524F5554494E450A44
:102B8000002220706F73002220706172656E743AAB
:102B90002200535542524F5554494E452043414C13
:102BA0004C207461726765743A22005375626361E8
:102BB0006C6C204F766572666C6F77004578636544
:102BC00065646564206D617820535542524F5554B9
:102BD000494E452064657074683A002E0A004465C9
:102BE0006C6574696F6E206661696C65642C204643
:102BF000696C653A200046696C652064656C657493
:102C000065643A005344207072696E74696E67207F
:102C10006279746520004E6F74205344207072698D
:102C20006E74696E670A0057726974696E67207402
:102C30006F2066696C653A2000667265736800648F
:102C40006F696E67002066696C653A20004E6F7789
:102C500020002F6175746F25632E67002020506C53
:102C6000616E6E65724275666665724279746573EF
:102C70003A20002046726565204D656D6F72793A85
:102C80002000436F6D70696C65643A20417072205A
:102C9000323920323032310A00204C6173742055B1
:102CA0007064617465643A20323032312D30342DD5
:102CB0003138207C20417574686F723A2054696EF7
:102CC000794D616368696E657333440A00322E3052
:102CD0002E375F4457372E332E310A004D61726C08
:102CE000696E0020536F6674776172652052657358
:102CF00065740A00205761746368646F67205265C9
:102D00007365740A002042726F776E206F757420AD
:102D100052657365740A002045787465726E616C43
:102D20002052657365740A00506F77657255700A9A
:102D30000073746172740A004739310A47315A3599
:102D40000A4739300A4D38340A4D31303453300A8D
:102D50004D3134305330004D3130303100657272B6
:102D60006F722077726974696E6720746F2066696C
:102D70006C650A00446F6E6520736176696E67202A
:102D800066696C652E0A004D323900456E647374B5
:102D90006F70730025532025632025632025632051
:102DA000256300205A3A0020593A0020583A00651D
:102DB0006E6473746F7073206869743A20007001D8
:102DC0002C0190012701B0012201C0011D01F00179
:102DD00018011002130130020E0160020901900275
:102DE0000401C002FF000003FA004003F500800365
:102DF000F000D003EB002004E6007004E100E004E2
:102E0000DC004005D700C005D2004006CD00D0064A
:102E1000C8008007C3003008BE00F008B900C00930
:102E2000B400B00AAF00B00BAA00D00CA500000E91
:102E3000A000500F9B00C01096005012910000148B
:102E40008C00C0158700B0178200B0197D00D01B20
:102E50007800001E730040206E0090226900F0246C
:102E6000640040275F0090295A00E02B5500102E87
:102E7000500020304B0010324600E03341009035C6
:102E80003C001037370070383200A0392D00B03ABE
:102E90002800A03B2300603C1E00103D1900903D1F
:102EA0001400103E0F00703E0A00C03E0500003FB7
:102EB0000000403FFBFF803FF6FFC03FF1FF0000F6
:102EC0000A0B02090C0D0E080703040100000000A4
:102ED00000000000000000000000000000000000F2
:102EE00000000000000000000000121110000000AF
:102EF00000000000000000000000000000000000D2
:102F00000000000050726F62696E67204661696C54
:102F1000656400205A3A200020593A200042656436
:102F200020583A20003D3D6F6E55736572436F6EB9
:102F30006669726D52657175697265643D3D002206
:102F40000A00556E6B6E6F776E20636F6D6D616EEC
:102F5000643A2022002042002050006F6B00204580
:102F600000205A00205900204D39322058002045B9
:102F70003A00205A3A0020593A00583A0020746F1B
:102F80006F206C6F6E6720657874727573696F6EF1
:102F90002070726576656E7465640A0020636F6CDC
:102FA0006420657874727573696F6E2070726576CF
:102FB000656E7465640A0043616E6E6F7420656EA1
:102FC000746572207375626469723A20004D3235FF
:102FD00020500A4D323400526573756D65005549B5
:102FE000205061757365004E6F204D6174636820D9
:102FF0003A004D32320A4D323100526566726573C5
:10300000680050675570005067446F776E004973D1
:103010002046696C6520004973204469722000478E
:103020006F557044697200486173204D6564696131
:103030000046696C656E616D652053656C656374EF
:103040006564004D3130303043004D313030300058
:1030500046696C616D656E74205374617420302014
:103060002D20330046696C616D656E742053746168
:10307000742030202D20320046696C616D656E74BD
:1030800020537461742030202D2031002046696C5B
:10309000616D656E7420526573706F6E7365204E3E
:1030A0006F00526573756D65205965732064757284
:1030B000696E67207072696E74000A204E6F204638
:1030C000696C616D656E7400496E76616C6964202F
:1030D0004F7074696F6E004D3530300053746F72ED
:1030E000652053657474696E67730042656420508F
:1030F00049442053746172746564004D3939390A4A
:103100004D32383050305331363000424C546F75A8
:103110006368205265736574004D3530320A4D3551
:10312000303000496E697420454550524F4D00487B
:103130006F74656E642050494420537461727465E5
:103140006400456E676C69736820416C72656164E8
:103150007920536574004368696E657365204E6F0E
:103160007420537570706F7274656400496E4C61A1
:103170006E6743686F696365000A202A2A2A7265B0
:10318000636461742E646174615B305D203D00474F
:1031900032380A4731204631303030205A31300041
:1031A000556E737570706F72746564204F707469BA
:1031B0006F6E2053656C65637465640047323652E8
:1031C000323535004D3139305335350A4732380AFA
:1031D0004732390A4D3430300A4D313034533231B0
:1031E000350A4732380A4D313039533231350A4DBC
:1031F00034323053310A4731583130305931303060
:1032000046353030300A47315A300A4D3530300AB1
:103210004D31313720536574205A204F66667365EF
:1032200074004731204631303030205A302E300083
:103230004732380A4731204631303030205A302E5C
:1032400030004D353030005A204F6666736574206B
:103250003A202573004D353030005A204F66667392
:103260006574203A202573004732380A47314631C9
:103270003530305A302E30004732385A0A473146FE
:10328000313530305A302E30004D38340047314619
:10329000313030305A302E30004732380A4731460C
:1032A000313030305A302E30004D616E75616C53C4
:1032B000657454656D7000526571756573746564ED
:1032C000204F6666736574204265796F6E64204C8A
:1032D000696D697473005A204F6666736574203A8D
:1032E00020257300526F756E64696E6720746F20BD
:1032F0007374657000526571756573746564204FF1
:103300006666736574200053746F70205472696729
:1033100067657265640053746F70204E6F0053745C
:103320006F705072696E740048616E646C65204401
:103330006174612041646A7573742032205365742E
:1033400074696E672053637265656E200048616E14
:10335000646C652044617461205072696E744669C2
:103360006C6520332053657474696E6720536372F3
:1033700065656E200048616E646C6520446174610F
:10338000205072696E7446696C65203220536574F2
:1033900074696E672053637265656E20004D383422
:1033A0000048616E646C65204461746120507269EC
:1033B0006E7446696C6520506F73740048616E646A
:1033C0006C652044617461205072696E7446696C4A
:1033D000652050726500426567696E537769746352
:1033E00068003D3D20436865636B6B65793D3D003A
:1033F0007265636461742E61646472203D3D007285
:1034000065636461742E646174615B305D203D3D71
:103410000077616974776179203D3D0020202A2A78
:103420002A2A2A2A2A5254535F48616E646C6544E2
:103430006174612A2A2A2A2A2A2A2A2000526573BC
:10344000656E643A200000002200250028002B0051
:103450002E003100340002010000050108010B01BB
:1034600000002100240027002A002D003000330036
:1034700001010000040107010A0105050505070512
:1034800008080808020202020A0A080804040404E0
:10349000010101010101010103030303030303030C
:1034A000040707070C0C0C0C0C0C0C0C020202029B
:1034B00006060606060606060B0B0B0B0B0B0B0B84
:1034C0000102102020080810204010204080020136
:1034D000020108040201010204081020408080401B
:1034E000201008040201800402018040201008041A
:1034F00002010804020101020408102040800102B8
:10350000040810204080544D3344204D61782052EF
:10351000656164792E005072696E74696E672E2E33
:103520002E005072696E7420506175736564006E70
:103530006F74696669636174696F6E2000504944F5
:103540002054756E652046696E6973686564000075
:103550003601C20011241FBECFEFD1E2DEBFCDBFC6
:1035600000E00CBF13E0A0E0B2E0EAE5F1E602E023
:103570000BBF02C007900D92A83FB107D9F726E113
:10358000A8EFB3E001C01D92A432B207E1F71AE13F
:10359000C9EADAE100E006C021970109802FFE01A7
:1035A0000F94DA2CC83AD10780E00807A9F70F94E6
:1035B000511A0D949B300C9400009F92AF92BF92D1
:1035C000CF92DF92EF92FF920F931F93CF93DF93EF
:1035D00000D01F921F92CDB7DEB7E5E5FBE10027D3
:1035E000BB27462F572FA82FAA2341F4A52F542FCE
:1035F000B85FAA2319F4A52F5527B85FA03138F476
:103600005295A295452F4F70507FA42BBC5FA034DC
:1036100028F4550FAA1F550FAA1FBE5FA03818F433
:10362000550FAA1FB395550FAA1FEA0FF01F44911B
:1036300051E0AA27B85081F1C8F0B0FF02C0440F92
:10364000551FB1FF04C0440F551F440F551FB2FF53
:1036500006C052954295142F1F70407F512BB3FF27
:103660001BC0A52F542F44270C944C1BB195B0FFC1
:1036700002C055954795B1FF04C05595479555959E
:103680004795B2FF05C05295407F4295452B5F702C
:10369000B3FF02C0452F5527DD24CC24BB24B2E064
:1036A000649FD018C108B00AB00B749FC018B1084D
:1036B000B00B849FB018B109659FC018B108B00B5A
:1036C000759FB018B109859FB0196A9FB018B109EC
:1036D0007A9FB0194D9DA12C992433279927222731
:1036E0005D9DA00C911C301F901F201FAD9D900C64
:1036F000311D901F201F4C9DA00C911C301F901F4E
:10370000201F5C9D900C311D901F201FAC9D300D23
:10371000911D201F4B9D900C311D901F201F5B9D04
:10372000300D911D201FAB9D900D211D4B9F300D25
:10373000911D201F5B9F900D211DAB9F200DB1E0BF
:10374000BB24CC24DD24639FD018C108B00AB00B81
:10375000739FC018B108B00B839FB018B109699F5F
:10376000C018B108B00B799FB018B109899FB01982
:10377000629FB018B109729FB019D61AC70AB80A69
:1037800020F0B1E03B0F901F201F1124792F632FF1
:1037900090E0822F0F900F900F900F900F90DF917D
:1037A000CF911F910F91FF90EF90DF90CF90BF903E
:1037B000AF909F900895AF92BF92CF92DF92EF9219
:1037C000FF920F931F93CF93DF93CEE2DCE001EEE5
:1037D00018E08EE3A82E8CE0B82EC12CD12C7601F7
:1037E000C39469917991899199910F9418262889A8
:1037F00039894A895B890F9479260F94562EF801EE
:1038000061937193819391938F01C616D706E80651
:10381000F90610F46B017C01AC16BD0611F76FEFD1
:103820007FEFCB01A70196010F94572C2093F1084D
:103830003093F2084093F3085093F408DF91CF914E
:103840001F910F91FF90EF90DF90CF90BF90AF90BE
:103850000895CF92DF92EF92FF928091ED07882337
:1038600009F457C0C090E907D090EA07E090EB0751
:10387000F090EC0720E030E0A901C701B6010F94F9
:103880001326882309F445C020E030E040E05FE3E0
:10389000C701B6010F9479269B01AC010F947926DC
:1038A0002BED3FE049E450E40F9479269B01AC01F5
:1038B00060E070E080E89FE30F94DD2D6B017C01F8
:1038C000C092760CD092770CE092780CF092790C42
:1038D0006091650270916602072E000C880B990BAF
:1038E0000F941A262AE037ED43E25CE30F94792621
:1038F000A70196010F94792660936102709362028A
:103900008093630290936402FF90EF90DF90CF90DA
:103910000895C12CD12C80E8E82E8FE3F82ED0CF6B
:103920000F931F93CF93DF9350E0FC01E40FF51F3B
:103930008081440F551F440F551F4D565A4FEA01C1
:10394000882329F188819981AA81BB81EB010881B3
:1039500019812A813B810097A105B10569F40C59B1
:103960001F4F2F4F3F4FDA010D931D932D933C9323
:1039700013978FEF808306C0081B190B2A0B3B0B94
:1039800037FDF7CFDF91CF911F910F9108951882E6
:1039900019821A821B82F6CFCF93DF9324E0829F95
:1039A000C0011124EC01CC53D74FFC01E650F84F75
:1039B0008251984FDC012D913D914D915C91608138
:1039C0007181828193810F94E32C688379838A8348
:1039D0009B83DF91CF91089580918E0590918F0503
:1039E000A0919005B091910580934102909342027D
:1039F000A0934302B093440280918C0590918D0571
:103A0000909368028093670208958091410290919B
:103A10004202A0914302B091440280938E0590939C
:103A20008F05A0939005B0939105809167029091C6
:103A3000680290938D0580938C0584E690E09093C6
:103A4000680280936702089580917E1290917F12A0
:103A5000891B877089F48091860D81110DC080913A
:103A60007A0C90917B0C892B39F481E090919C0623
:103A7000911103C080E0089581E00895CF93DF9312
:103A8000DB01F9019C919130C1F0943080F09450A9
:103A90009C938830D1F480819181009771F00197D7
:103AA00091838083480F591FEA01188206C08C3524
:103AB00039F49C5F9C93943041F4DF91CF91089549
:103AC0008B3339F781E08C93F8CF20813181B901B4
:103AD0006F5F7F4F71836083420F531FEA018883BA
:103AE000808191818F3591056CF7E7CF0F931F93FC
:103AF00081E000912214109123142091241430911C
:103B0000251440911E1450911F146091201470913F
:103B10002114041715072607370708F480E01F91C2
:103B20000F91089590E080E00895282F9091E80784
:103B3000833021F495FD0FC094FD0FC0892F90E0D4
:103B4000B0E0A0E004C0B695A795979587952A9513
:103B5000D2F78170089581E0089580E00895FC0116
:103B6000659175918591949108958F929F92AF92EE
:103B7000BF92CF92DF92EF92FF92CF93DF93EC014F
:103B80008090C0089090C108A090C208B090C3086F
:103B900020E030E0A901C501B4010F941326882369
:103BA00009F454C0C880D980EA80FB80A70196013F
:103BB000C501B4010F94132618160CF04CC02091C7
:103BC000B8083091B9084091BA085091BB08C701B4
:103BD000B6010F941326882331F1C092B808D09211
:103BE000B908E092BA08F092BB082091BC08309165
:103BF000BD084091BE085091BF08688179818A81D3
:103C00009B810F9479269B01AC0160E070E080E815
:103C10009FE30F94E22C60930F0270931002809345
:103C200011029093120260910F0270911002809124
:103C3000110290911202DF91CF91FF90EF90DF90EF
:103C4000CF90BF90AF909F908F90089560E070E00C
:103C500080E89FE3F0CF60E070E0CB01ECCFCF9243
:103C6000DF92EF92FF92CF93DF93EC01CC80DD8067
:103C7000EE80FF8027E137EB41ED58EBC701B6013D
:103C80000F94432F87FD23C023E030E041EE53E43F
:103C9000C701B6010F9413261816CCF0C880D9803E
:103CA000EA80FB8027E137EB41ED58EBC701B60115
:103CB0000F94432F87FD0BC0C1E023E030E041EEBD
:103CC00053E4C701B6010F94132618160CF4C0E094
:103CD0008C2FDF91CF91FF90EF90DF90CF900895E0
:103CE0002FEB280F2A3108F047C0E22FF0E0809137
:103CF0002B0590912C05A0912D05B0912E0504C0A7
:103D0000B695A795979587952A95D2F780FD02C01D
:103D100081700895E35FFA4FE081EE2341F18091D5
:103D20007A0790917B07E80FF92FF11D808190EDC4
:103D3000980F9A3030F08E3251F4818180538A305E
:103D400098F4F093FC04E093FB0481E008958D3235
:103D500011F08B3249F4818190ED980F9A3088F3FD
:103D60008E3211F48281EACFF0E0E0E0EACF1092E7
:103D7000FC041092FB04E9CF80E008950E94701EBD
:103D8000882341F081E02091FB043091FC04232B37
:103D900009F480E008958F929F92AF92BF92CF92E4
:103DA000DF92EF92FF92C090CA05D090CB05E090D1
:103DB000CC05F090CD0520E030E0A901C701B601A7
:103DC0000F9413268823E1F1A701960160E070E0CB
:103DD00080E89FE30F94DD2D6B017C018090CE0580
:103DE0009090CF05A090D005B090D10520E030E0B4
:103DF000A901C501B4010F941326882329F1A50157
:103E0000940160E070E080E89FE30F94DD2DC092A4
:103E1000D404D092D504E092D604F092D7046093F3
:103E2000D8047093D9048093DA049093DB04FF9054
:103E3000EF90DF90CF90BF90AF909F908F900895BC
:103E4000C12CD12C7601CACF60E070E0CB01DFCF6E
:103E5000129A08955F9A80912C0C8E7F80932C0C7F
:103E60008A9A80912C0C8D7F80932C0C8091080174
:103E7000809581708093060180912C0C8B7F8093BC
:103E80002C0C0C94281F269A2E9A08958C3221E02F
:103E9000920714F08CE291E09093E3118093E21189
:103EA0000C947EFDE6E0F6E010821182128213820D
:103EB00014820C947EFD4F925F926F927F928F924C
:103EC0009F92AF92BF92CF92DF92EF92FF920F93A9
:103ED0001F93CF93DF93EC012091C2053091C3056E
:103EE0004091C4055091C505688179818A819B8183
:103EF0000F94E22C6B017C012091C6053091C7051F
:103F00004091C8055091C9056C817D818E819F814A
:103F10000F94E22C4B015C01A70196016091030212
:103F20007091040280910502909106020F9413266D
:103F3000882309F450C0C0920302D0920402E09298
:103F40000502F09206022091D4043091D5044091EC
:103F5000D6045091D704C701B6010F9479262B01DE
:103F60003C010F94852E6B017C0120E030E0A9011B
:103F70000F94132687FD70C020E030E040E450E449
:103F8000C701B6010F94432F18162CF4C12CD12C65
:103F9000C0E4EC2EFE2CA7019601C301B2010F94E0
:103FA000E22C6093CC047093CD048093CE04909364
:103FB000CF04C701B6010F944F2E6093CA04062E9A
:103FC000000C770B6F5F7F4F6430710514F064E075
:103FD00070E06093C804D09101021091CA04A50159
:103FE00094016091070270910802809109029091FA
:103FF0000A020F941326811133C0D11381C020917E
:10400000B0043091B1044091B2045091B304609176
:10401000CC047091CD048091CE049091CF040F9484
:1040200079262091B4043091B5044091B6045091A2
:10403000B7040F94E32CDF91CF911F910F91FF9064
:10404000EF90DF90CF90BF90AF909F908F907F9038
:104050006F905F904F900895C12CD12C76019BCF2B
:104060008092070290920802A0920902B0920A027E
:104070002091D8043091D9044091DA045091DB04A6
:10408000C501B4010F9479264B015C010F94852E74
:104090006B017C0120E030E0A9010F94132687FD1D
:1040A000F3C020E030E040E450E4C701B6010F94D3
:1040B000432F18162CF4C12CD12CB0E4EB2EFE2C7F
:1040C000A7019601C501B4010F94E22C6093D004BE
:1040D0007093D1048093D2049093D304C701B601A6
:1040E0000F944F2E6093CB04062E000C770B6F5F5E
:1040F0007F4F6430710514F064E070E06093C90490
:10410000C091CB04D11305C0809102028C1709F431
:1041100070C08091CA049091CB0490930202809366
:1041200001020C2E000CDD0B25E01203C00111244E
:10413000FC01EC0FFD1FEE0FFF1FEE0FFF1FEC57F2
:10414000F84F20813181428153812093C404309300
:10415000C5044093C6045093C7040091C904002EBF
:10416000000C110BFC01E00FF11FEE0FFF1FEE0F13
:10417000FF1FEC57F84F60817181828193810F940A
:10418000E22C6093C0047093C1048093C2049093A6
:10419000C3042091C80435E02303F0011124CE0F9D
:1041A000DF1FCC0FDD1FCC0FDD1FCC57D84F288170
:1041B00039814A815B812093BC043093BD044093D4
:1041C000BE045093BF04E00FF11FEE0FFF1FEE0F70
:1041D000FF1FEC57F84F60817181828193810F94AA
:1041E000E22C6093B8047093B9048093BA0490935E
:1041F000BB048090D0049090D104A090D204B090E1
:10420000D3042091C0043091C1044091C204509164
:10421000C304C501B4010F9479262091C4043091E0
:10422000C5044091C6045091C7040F94E32C6B0160
:104230007C01C092B404D092B504E092B604F0922E
:10424000B7042091B8043091B9044091BA04509158
:10425000BB04C501B4010F9479262091BC043091B0
:10426000BD044091BE045091BF040F94E32CA701FC
:1042700096010F94E22C6093B0047093B104809384
:10428000B2049093B304BBCEC12CD12C760118CFCD
:10429000CF92DF92EF92FF92CF93DF93EC010896DB
:1042A0000E94B51D6B017C0120E030E0A9010F9454
:1042B000132620E030E0A901882359F0CE010E94A6
:1042C0005B1F9B01AC01C701B6010F9479269B01CE
:1042D000AC01688579858A859B850F94E22C688777
:1042E00079878A879B87DF91CF91FF90EF90DF904E
:1042F000CF9008952F923F924F925F926F927F924C
:104300008F929F92AF92BF92CF92DF92EF92FF92E5
:104310000F931F93CF93DF93D62FC72FFC0180807D
:104320009180A280B380C501B40120E831E541E06D
:1043300050E00F94572CC9016DE671E00F94C62C24
:104340006B017C01C501B40120E13EE040E050E09A
:104350000F94572CCA01B90128E130E040E050E049
:104360000F94572C362E272E062F172F8CE3482E0E
:10437000512C612C712CC501B401A30192010F9441
:10438000572CB62EA72ECA01B901A30192010F9492
:10439000572CCB01C114D10479F1AF92BF927F9316
:1043A0006F932F923F92FF92EF92DF92CF928CE524
:1043B00097E19F938F93CF93DF930F94AA258DB7A7
:1043C0009EB70E960FB6F8949EBF0FBE8DBF8D2F71
:1043D0009C2FDF91CF911F910F91FF90EF90DF9075
:1043E000CF90BF90AF909F908F907F906F905F9095
:1043F0004F903F902F900895E114F104C9F0AF92CF
:10440000BF927F936F932F923F92FF92EF928CE433
:1044100097E19F938F93CF93DF930F94AA25EDB7E6
:10442000FEB73C960FB6F894FEBF0FBEEDBFCFCFE0
:10443000012BB9F0AF92BF927F936F932F923F926F
:1044400080E497E19F938F93CF93DF930F94AA25F6
:104450008DB79EB70A960FB6F8949EBF0FBE8DBF5C
:10446000B6CF892BA9F0AF92BF927F936F9388E369
:1044700097E19F938F93CF93DF930F94AA25EDB786
:10448000FEB738960FB6F894FEBF0FBEEDBF9FCFB4
:10449000AF92BF9284E397E19F938F93CF93DF9383
:1044A0000F94AA250F900F900F900F900F900F90E0
:1044B0008ECFEF92FF920F931F93CF93DF93CDB7E1
:1044C000DEB78C01EDB6FEB60F94602501962DB7D0
:1044D0003EB7281B390B0FB6F8943EBF0FBE2DBF59
:1044E0008DB79EB70196B8010F9459250E94A1F986
:1044F0000FB6F894FEBE0FBEEDBEDF91CF911F91B7
:104500000F91FF90EF9008958C38910514F08CE88E
:1045100090E090937811809377110C94B5BEAB0125
:10452000BC0140932214509323146093241470937D
:1045300025148AE895E10C946DAF2F923F924F922B
:104540005F926F927F928F929F92AF92BF92CF9223
:10455000DF92EF92FF920F931F93CF93DF93CDB72C
:10456000DEB760970FB6F894DEBF0FBECDBF8B8766
:104570006C87042F122F282F30E03E872D87462F7F
:1045800050E05A87498785E0982E929EC001939EFD
:10459000900D1124988B8F87FA01E80FF91FEE0F09
:1045A000FF1FEE0FFF1FEC57F84F60817181828172
:1045B00093819B01AC010F94D52F882309F445C149
:1045C0004B85400F6C85610F949EC0011124E985D5
:1045D000FA85E80FF91FEE0FFF1FEE0FFF1FEC57D4
:1045E000F84FC080D180E280F380040F909EA0013C
:1045F0001124E985FA85E40FF51FEE0FFF1FEE0F7A
:10460000FF1FEC57F84F0081918082807380262F26
:1046100030E0EF85F889E20FF31FEE0FFF1FEE0F7A
:10462000FF1FEC57F84F20807181798372817A8364
:1046300073817B83610F70E0EF85F889E60FF71FC8
:10464000EE0FFF1FEE0FFF1FEC57F84FF88BEF87B1
:10465000F081FC83EF85F889F181FD83EF85F8898E
:10466000F281FE83EF85F889F381FF83FC01E20F7D
:10467000F31FEE0FFF1FEE0FFF1FEC57F84F2081C7
:104680002887A180B2806380FA01E60FF71FEE0F42
:10469000FF1FEE0FFF1FEC57F84F40805180328014
:1046A0001381202F392D482D572D602F792D882DDE
:1046B000972D0F94D52F882321F000E0912C812C89
:1046C000712C9601A701B601C7010F94D52F88233D
:1046D00021F0C02ED92CE82CF72C2C813D814E8165
:1046E0005F816C817D818E819F810F94D52F88237E
:1046F00021F01C821D821E821F82222D39814A8157
:104700005B81622D79818A819B810F94D52F8823CB
:1047100039F02C803D8139834E814A835F815B83F0
:104720009201432D512FB201832D912F0F94D52F3C
:10473000882321F0412C512C312C10E028853A2D72
:104740004B2D562D68857A2D8B2D962D0F94D52FB8
:10475000882321F04886A52CB32C612E85E02D8579
:104760003E85829FF001839FF00D112449855A8573
:10477000E40FF51FEE0FFF1FEE0FFF1FEC57F84F72
:10478000FA87E9879601A701B601C7010F94E32CC8
:10479000202F392D482D572D0F94E22C6B017C01D1
:1047A000222D39814A815B81622D79818A819B81A9
:1047B0000F94E32C2C813D814E815F810F94E22C7C
:1047C0009B01AC01C701B6010F94E32C6B017C0186
:1047D00028853A2D4B2D562D68857A2D8B2D962DBB
:1047E0000F94E32C9201432D512F0F94E22C9B0147
:1047F000AC01C701B6010F94E32C20E030E040E4A7
:1048000050E40F94DD2DE985FA85608371838283FE
:1048100093836C858B8560960FB6F894DEBF0FBED0
:10482000CDBFDF91CF911F910F91FF90EF90DF905F
:10483000CF90BF90AF909F908F907F906F905F9040
:104840004F903F902F900C9434F860960FB6F894E8
:10485000DEBF0FBECDBFDF91CF911F910F91FF90B3
:10486000EF90DF90CF90BF90AF909F908F907F9010
:104870006F905F904F903F902F9008958091FB0430
:104880009091FC04009731F04AE050E070E060E065
:104890000D942E2460E070E0CB0108958091FB041C
:1048A0009091FC04009731F04AE050E070E060E045
:1048B0000D94002360E070E0CB010895CF93DF9367
:1048C000EB010E94BE1E882319F00E944E24EB01CA
:1048D000CE01DF91CF9108950E944E2497FD0CC028
:1048E0000E944E246F3F71058105910509F034F453
:1048F0000E944E24862F089580E008958FEF08953A
:10490000CF93C62F0E94BE1E882319F0CF910C941E
:104910006C248C2FCF9108958091FB049091FC041E
:10492000892B41F00E946C2491E0811101C090E03C
:10493000892F089591E0FCCFCF93DF93C82FD62F16
:104940000E94BE1E882321F0DF91CF910C948C240D
:104950008C2F0E94701E811101C08D2FDF91CF918D
:1049600008950E944E24CB010895CF93DF93EB016D
:104970000E94BE1E882321F0DF91CF910C94B124B8
:10498000CE01DF91CF9108950F931F93CF93809124
:10499000FB049091FC040097E9F0FC018F01C191A8
:1049A0002C2F2F7D81F0C53411F0C536B9F7F801F1
:1049B000108270E060E00F94A221F801C083CF91D3
:1049C0001F910F91089570E060E0CF911F910F91BA
:1049D0000D94A22160E070E0CB01F1CFCF92DF9285
:1049E000EF92FF926A017B010E94BE1E882331F084
:1049F000FF90EF90DF90CF900C94C424C701B601D4
:104A0000FF90EF90DF90CF9008954F925F926F925A
:104A10007F928F929F92AF92BF92CF92DF92EF924E
:104A2000FF921F93CF93DF9300D01F92CDB7DEB7D5
:104A300019821A821B821C82CE0101964C0188E6E3
:104A4000C82E87E0D82E9CE1E92E9CE0F92E24ECBC
:104A5000A22E28E0B22E10E088E5810F0E94BE1E33
:104A6000F40181934F01882309F4E0C00E94C4241B
:104A70002B013C01812F0E94951D882309F4CCC095
:104A8000F7012081318142815381C301B2010F942A
:104A9000E32CF60160837183828393831F5FF4E0CC
:104AA000CF0ED11C84E0E80EF11C94E0A90EB11CDD
:104AB000133091F685E40E94BE1E8C83882309F48E
:104AC000C0C00E94C4246B017C0183E00E94951D3C
:104AD000882371F02091280C3091290C40912A0CE8
:104AE00050912B0CC701B6010F94E32C6B017C0194
:104AF000C0927407D0927507E0927607F09277071C
:104B00008091C105882359F18091261482FF27C026
:104B10008C81882321F18981811103C08A818823B6
:104B2000F1F02DEC3CEC4CE45DE360910F087091EA
:104B3000100880911108909112080F94E32C9B01AA
:104B4000AC016091240C7091250C8091260C909101
:104B5000270C0F94432F181614F40E947AF740E0A4
:104B600050E0BA0186E40E94EE2420E030E0A90182
:104B70000F94432F181684F40E94C42420E030E0E0
:104B800040E752E40F94DD2D60934102709342029E
:104B900080934302909344028091DA0B83FD28C0F6
:104BA00080918706882321F12091280C3091290CCF
:104BB00040912A0C50912B0C6091740770917507ED
:104BC00080917607909177070F94E22C20919406BC
:104BD0003091950640919606509197060F94E32CDC
:104BE000609394067093950680939606909397062B
:104BF0000F900F900F900F90DF91CF911F91FF902A
:104C0000EF90DF90CF90BF90AF909F908F907F906C
:104C10006F905F904F900895F5012081318142811E
:104C20005381C301B2010F94E22C33CFF70180818D
:104C30009181A281B381F60180839183A283B383A2
:104C40002DCF8091280C9091290CA0912A0CB09125
:104C50002B0C8093740790937507A0937607B093FD
:104C600077074ECFCF92DF92EF92FF926B017C01DC
:104C700083E3C816D104E104F10470F082E3C81A9A
:104C8000D108E108F10862E370E080E090E00E9462
:104C90003FFD0E942FC2ECCFC701B6010E943FFD2D
:104CA000FF90EF90DF90CF900C942FC2CF92DF92C5
:104CB000EF92FF920F931F93CF93DF936B017A01D3
:104CC000EC01C057DB4F28813CE0389F8001399FC1
:104CD000100D112427FF24C0FB011182108288814E
:104CE0008F5F888388819801280F311D87FD3A9551
:104CF000C90120916912F6012817190629F024F03C
:104D000088818C300CF43CC0808191810496803481
:104D10009C4908F475C0F60180819181049672C0A7
:104D200088819801280F311D87FD3A95C90120918E
:104D300069122817190699F294F28881A801480F80
:104D4000511D87FD5A95FA01EE0FFF1FE40FF51F65
:104D5000EF5DFD4E808187FFC2CF8881F801E80FAB
:104D6000F11D87FDFA95CF01EE0FFF1FE80FF91F28
:104D7000EF5DFD4E808160E08F770E94DDFBAFCF5D
:104D8000808191812881A801420F511D27FD5A95EC
:104D90009A01FA01EE0FFF1FE20FF31FEF5DFD4EC8
:104DA00021813281820F931FF70191838083888153
:104DB0009801280F311D87FD3A95F901EE0FFF1F6D
:104DC000E20FF31FEF5DFD4E808187FF20C08881D9
:104DD000080F111D87FD1A95F801EE0FFF1FE00F58
:104DE000F11FEF5DFD4E808161E08F77DF91CF9104
:104DF0001F910F91FF90EF90DF90CF900C94DDFB0F
:104E000080E49CE9F701918380838FEF8883DF91B1
:104E1000CF911F910F91FF90EF90DF90CF90089569
:104E20000F931F93CF93DF9302E41CE0CBE5D1E116
:104E3000F80121913191419151918F0160E070E031
:104E400080E89FE30F94DD2D69937993899399937B
:104E5000F1E1CB36DF0761F70E94B9F5DF91CF9121
:104E60001F910F910C94DB1BCF92DF92EF92FF9278
:104E7000CF93DF9320912D0C222329F1EC0108968A
:104E80000E94B51D6B017C0120E030E0A9010F9468
:104E9000132620E030E0A901882359F0CE010E94BA
:104EA0005B1F9B01AC01C701B6010F9479269B01E2
:104EB000AC01688579858A859B850F94E32C68878A
:104EC00079878A879B87DF91CF91FF90EF90DF9062
:104ED000CF9008952F923F924F925F926F927F9260
:104EE0008F929F92AF92BF92CF92DF92EF92FF92FA
:104EF0000F931F93CF93DF93CDB7DEB76C970FB6A9
:104F0000F894DEBF0FBECDBF8C015B015A8349838D
:104F1000FC01EA5BFF4F2081318142815381298767
:104F20003A874B875C87CA01B9010F9418266B0139
:104F30007C01D5012D913D914D915C910F94792685
:104F40000F94C12D2B013C01E981FA81208131812F
:104F500042815381C701B6010F9479260F94C12D68
:104F60004B015C01C301B2010F94562E698B7A8B01
:104F70008B8B9C8B683771058105910540F428E780
:104F800030E040E050E0298B3A8B4B8B5C8BC501C5
:104F9000B4010F94562E6D877E878F87988B683764
:104FA00071058105910540F448E750E060E070E04C
:104FB0004D875E876F87788BF801EE5AFF4F4080F0
:104FC000518062807380C301B2010F941A266983F5
:104FD0007A838B839C8369897A898B899C890F94D6
:104FE00018266D8B7E8B8F8B988F20E030E0A90187
:104FF00069817A818B819C810F941326882309F41F
:10500000E1C1A7019601C701B6010F9479264B01B2
:105010005C012D893E894F89588DCA01B9010F94D1
:1050200079269B01AC01C501B4010F94E22C4B0120
:105030005C0129813A814B815C81CA01B9010F94DD
:10504000E32C9B01AC01C501B4010F94DD2D0F943D
:10505000C12D0F94562E6D837E838F83988766278C
:105060007727CB0164197509860997090F941A26C9
:105070004B015C016D857E858F8598890F9418267C
:105080002B013C0120E030E0A901C501B4010F94DF
:105090001326882309F49AC1A3019201C301B20126
:1050A0000F947926698F7A8F8B8F9C8FA701960139
:1050B000C701B6010F9479269B01AC01698D7A8DE9
:1050C0008B8D9C8D0F94E22C6B017C01A5019401CA
:1050D000C501B4010F94E32C9B01AC01C701B601DB
:1050E0000F94DD2D0F94852ED80195968D909D906F
:1050F000AD90BC909897750164012D813E814F81E0
:105100005885C21AD30AE40AF50A0F94562EC61A15
:10511000D70AE80AF90AF7FE8EC02D893E894F8921
:10512000588DCA01B9010F9479266B017C01298140
:105130003A814B815C81CA01B9010F94E32C6987E4
:105140007A878B879C8720E030E0A90169817A818A
:105150008B819C810F941326882309F43BC1C501E0
:10516000B4010F94182629853A854B855C850F94E8
:105170007926A70196010F94E22C6D837E838F839D
:105180009887A3019201C301B2010F9479269B0174
:10519000AC016D817E818F8198850F94E32C2B016A
:1051A0003C0120E030E040E850E469817A818B8165
:1051B0009C810F9479269B01AC01C301B2010F942D
:1051C000DD2D0F94C12D2B013C0120E030E0A90121
:1051D0000F94432F18161CF0412C512C3201C3019F
:1051E000B2010F94562E6D837E838F839887861627
:1051F0009706A806B90620F48D829E82AF82B886F3
:105200006D817E818F8198850F94182629853A8536
:105210004B855C850F947926A70196010F94E32CAA
:105220000F94912F0F94562E69877A878B879C87CE
:10523000C12CD12C760169857A858B859C8529893D
:105240003A894B895C89621B730B840B950B0F9415
:10525000182629813A814B815C810F94DD2D20E055
:1052600034E244EF59E40F9479260F94562E4B0103
:105270005C0169857A858B859C852D853E854F856A
:105280005889621B730B840B950B0F941826298188
:105290003A814B815C810F94DD2D20E034E244EFB4
:1052A00059E40F9479260F94562E2B013C013FE6CA
:1052B00083169104A104B10408F090C0F401EE0F2C
:1052C000FF1FEE0FFF1FE756F64E85919591A591B2
:1052D000B4918983292E3A2EBD8B4FE64416510492
:1052E0006104710408F083C0F201EE0FFF1FEE0F9E
:1052F000FF1FE756F64E45915591659174919A01BD
:10530000CB014D815E816F817885D80199964D934F
:105310005D936D937C939C974C0D5D1D6E1D7F1D61
:10532000F80145A756A767A770ABE65BFF4F498911
:105330005A896B897C894083518362837383D596B4
:105340008D929D92AD92BC92D897F80141AE52AE2B
:1053500063AE74AEFD9649814083218232825D89BD
:1053600053833496208331838283938369857A853E
:105370008B859C85D1966D937D938D939C93D497CB
:105380003D962D853E854F85588920833183428304
:1053900053836C960FB6F894DEBF0FBECDBFDF917E
:1053A000CF911F910F91FF90EF90DF90CF90BF9022
:1053B000AF909F908F907F906F905F904F903F90B5
:1053C0002F90089560E070E0CB0141CE60E070E086
:1053D000CB0188CE60E070E0CB01F3CEC501B40113
:1053E0000E94DD1A6983272E382E9D8B76CFC3014C
:1053F000B2010E94DD1A9B0184CF80917E129091B0
:105400007F12891B877019F490E080E008959091D5
:105410007B12992351F0833030F48FEF890F19F00C
:1054200080937B12F1CF10927B1280917F122CE53A
:10543000829FC00111248650974FFC01208120FDDE
:10544000E3CF20917F122F5F277020937C12309141
:105450007F1220917D12321304C020917C12209380
:105460007D12089590916F0081E091FD02C080E06F
:10547000089590916F009D7F90936F00089580FF35
:1054800004C09091920590FD8E7F81FF05C09091A0
:105490009205969590FD8D7F82FF06C090919205B2
:1054A0009695969590FD8B7F08958F929F92AF92DF
:1054B000BF92CF92DF92EF92FF92CF93DF93209132
:1054C0004502222309F49EC0EC0180919205C82E6A
:1054D000D12CF12CE12C80FF2CC0809047029090C1
:1054E0004802A0904902B0904A02288139814A813D
:1054F0005B81C501B4010F94432F181624F48882F0
:105500009982AA82BB828090530290905402A0900C
:105510005502B0905602288139814A815B81C501CC
:10552000B4010F94132687FF04C088829982AA824F
:10553000BB82D701C601B695A7959795879580FF41
:105540002CC080904B0290904C02A0904D02B090E5
:105550004E022C813D814E815F81C501B4010F94C3
:10556000432F181624F48C829D82AE82BF828090D5
:10557000570290905802A0905902B0905A022C8184
:105580003D814E815F81C501B4010F94132687FFD1
:1055900004C08C829D82AE82BF8282E0F694E79442
:1055A000D794C7948A95D1F7C0FE2CC0C0904F0203
:1055B000D0905002E0905102F09052022885398537
:1055C0004A855B85C701B6010F94432F181624F452
:1055D000C886D986EA86FB86C0905B02D0905C02C2
:1055E000E0905D02F0905E02288539854A855B85F2
:1055F000C701B6010F94132687FF04C0C886D98659
:10560000EA86FB86DF91CF91FF90EF90DF90CF90FD
:10561000BF90AF909F908F900895CF92DF92EF92BE
:10562000FF920F931F93C12CD12C76018C0128E29D
:105630003CE044E25CE060E27CE08CE19CE00E94C3
:10564000B5F41F910F91FF90EF90DF90CF900895E8
:105650000C94B9F580919906811105C08091780765
:10566000882309F463C080917F05659B59C08160E0
:1056700080937F059091030180917F0591FF52C037
:10568000826080937F0580917F054A9B4DC0846036
:1056900080937F058091E60580FF10C080919A0677
:1056A00080FF0CC080917F0580FF08C08091DC06E0
:1056B00081608093DC0680E00E948FC68091E605C1
:1056C000869580FF11C080919A06869580FF0CC058
:1056D00080917F0581FF08C08091DC068260809305
:1056E000DC0681E00E948FC68091E605869586954E
:1056F00080FF1CC080919A068695869580FF16C013
:1057000080917807882391F080917F0582FF0EC0F9
:105710008091DC0684608093DC0682E00C948FC666
:105720008E7FA6CF8D7FADCF8B7FB2CF0895809136
:105730009906811104C080917807882331F062E0D6
:1057400070E080E090E00C94322608950F931F9350
:1057500080911911813019F50E9472FD00919B050D
:1057600010919C0520919D0530919E05601B710B49
:10577000820B930B28EE33E040E050E00F94572C5F
:1057800060919F057091A0058091A1059091A2055F
:10579000620F731F841F951F1F910F9108956091D1
:1057A000A3057091A4058091A5059091A605D6CF7B
:1057B0001092191110929B0510929C0510929D0554
:1057C00010929E051092A3051092A4051092A505B3
:1057D0001092A60510929F051092A0051092A105A7
:1057E0001092A2050895CF92DF92EF92FF92CF938D
:1057F000DF93C62FFC01C080D180E280F38020E0DF
:1058000030E0A901C701B6010F94132620E030E073
:10581000A90187FD14C020E030E048EC52E4C70144
:10582000B6010F94432F24E630E040E050E0181614
:1058300034F0C701B6010F944F2E9B01AC01C2306A
:10584000A0F4D0E0CB50D74FAFEFB0E00F94982C3E
:1058500024E630E040E050E00F94792C2F3F3105F2
:1058600019F010F02FEF30E02883DF91CF91FF90F7
:10587000EF90DF90CF9008958091090180FD06C0E0
:105880008091261483FB882780F9089580E008958D
:10589000CF92DF92EF92FF92FC01C080D180E28034
:1058A000F380663019F510920B0610920C061092D8
:1058B0000D0610920E0610920F060E94B5BE20E053
:1058C00030E0A901C701B6010F94132687FF1DC060
:1058D000C12CD12C7601C701B6010F94502FCB01FA
:1058E000FF90EF90DF90CF900C9484220E94521F83
:1058F00020E030E0A901C701B6010F94132687FF0D
:1059000015C0C12CD12C760121C020E030E04CE044
:1059100053E4C701B6010F94432F1816E4F6C12CC7
:10592000D12C9CE0E92E93E4F92ED5CF20E030E095
:1059300046E953E4C701B6010F94432F181634F417
:10594000C12CD12C86E9E82E83E4F82EC701B601DC
:105950000F94502FCB01FF90EF90DF90CF900C94DD
:10596000461F90912C0C977081E0973009F080E0F1
:10597000089520917D0520FF14C020E83EE3629F3A
:10598000A001639F500D729F500D1124CA0196957E
:10599000879596958795009731F08A950000E9F7ED
:1059A00008950C9432260895CF93DF931092DB0B69
:1059B00010927C0C10927E0C10927D0C10927C0543
:1059C00010927B05CFEFDFEF8091261485FD07C095
:1059D0000E94CEAAD093A512C093A412F5CF8FEF48
:1059E0009FEF9093A5128093A412DF91CF91089519
:1059F0008F929F92AF92BF92CF92DF92EF92FF92DF
:105A00000F931F93CF93DF931092300510922F05C1
:105A10002FE320932A051092290510922805109251
:105A2000270510922B0510922C0510922D0510922F
:105A30002E059C01F90190812F5F3F4F9032D1F3E9
:105A40009E34C9F4818190ED980F9A3020F08D3208
:105A500011F08B3281F432969F012F5F3F4F80818E
:105A600080538A3008F47BC09F012F5F3F4F8081B5
:105A7000803209F476C0F0937B07E0937A078F01B8
:105A80000F5F1F4FC0816AE270E0C8010F94313090
:105A9000009731F0FC01319780818032E1F311826F
:105AA000CD3429F0C43519F0C73409F04BC0F801E2
:105AB00080810F5F1F4F8032D1F380538A3008F00E
:105AC00041C0C0932A0530E020E04AE0DF01119692
:105AD000429FC001439F900D11249C012053310926
:105AE0008081280F311D87FD3A95818190ED980FB7
:105AF0009A30C8F130932905209328058E3261F43D
:105B0000329690E04AE0DF0131968C9150ED580FCB
:105B10005A3058F190932705CD01DC0101964C9144
:105B20004032D9F3CD3489F52E31310539F018F5ED
:105B30002731310519F02C31310539F5B093300595
:105B4000A0932F05DF91CF911F910F91FF90EF90C0
:105B5000DF90CF90BF90AF909F908F900895F90104
:105B60007BCFF90181CFFD01B1CF949F800D11242E
:105B700090ED980FC8CF2537310538F0273731051C
:105B8000E8F2203A83E03807C9F2D0917A0740E082
:105B900050E0BA0110E000E0C12CD12C7601C39492
:105BA000FD0131968C91882309F47FC08132E1F4A4
:105BB000CD34D1F420323105B9F440932B05509304
:105BC0002C0560932D0570932E05F0933005E0931E
:105BD0002F0563E270E0CF010F943130009709F494
:105BE000B1CFFC011082AECF81548A3108F058C089
:105BF000DF019D91903291F0A0EDA90FAA30E8F05D
:105C00009E3271F4918190539A30B8F001151105CC
:105C100019F48F010150110990E013C0FD01E8CF84
:105C20009D3211F09B3291F79181A0EDA90FAA301E
:105C300020F09E3259F79281E6CF9E2F9D1B309720
:105C400059F3A82FB0E04601570104C0880C991CF5
:105C5000AA1CBB1C8A95D2F7482959296A297B2995
:105C6000A35FBA4F9C9380818154DF018A3108F48D
:105C700097CFDF018191882309F492CF90ED980F9F
:105C80009A30B8F393ED980F923098F38B3289F3F2
:105C9000CD010196EC91E03209F082CFDC01F8CF22
:105CA0000115110501F78D01DECF1093300500932A
:105CB0002F0540932B0550932C0560932D05709371
:105CC0002E0540CF4F925F926F927F928F929F925C
:105CD000AF92BF92CF92DF92EF92FF92CF93DF937A
:105CE00000D000D01F921F92CDB7DEB75C01DB0160
:105CF000CD90DD90ED90FC90E0917912F0917A12C8
:105D0000FE83ED8384819581A681B78189839A83FF
:105D1000AB83BC839C01AD01C701B6010F94E22C9B
:105D20002B013C01F50180809180A280B380AD8180
:105D3000BE818D919D910D90BC91A02D8D839E83F0
:105D4000AF83B88727E137EB41ED58EBC301B201D0
:105D50000F94432F87FDD1C023E030E041EE53E4A0
:105D6000C301B2010F94132618160CF4C6C02D817E
:105D70003E814F815885C501B4010F94E22C2B015F
:105D80003C0127E137EB41ED58EB0F94432F87FDA2
:105D9000B4C023E030E041EE53E4C301B2010F94FC
:105DA000132618160CF4A9C020E030E0A9016D817B
:105DB0007E818F8198850F94E32C2B013C0120E09C
:105DC00030E040E450E40F94132687FF05C0412CD7
:105DD000512C30E4632E762C27E137EB41ED58E36C
:105DE000C301B2010F94E22C9B01AC01C501B401C7
:105DF0000F94432F87FD81C020E030E041EE53E453
:105E00006D817E818F8198850F94E32C2B013C015D
:105E100020E030E84FED53E40F94432F18163CF484
:105E2000412C20E8522E2FED622E23E4722E27E122
:105E300037EB41ED58E3C301B2010F94E32C9B0112
:105E4000AC01C501B4010F94132618160CF455C00B
:105E500020E030E0A90169817A818B819C810F94D7
:105E6000E32C4B015C0120E030E040E951E40F9469
:105E7000132687FF06C0812C912C90E9A92E91E46E
:105E8000B92E27E137EB41ED58E3C501B4010F947A
:105E9000E22C9B01AC01C701B6010F94432F87FD93
:105EA0002CC020E030E041EE53E469817A818B819F
:105EB0009C810F94E32C4B015C0120E030E048ED25
:105EC00053E40F94432F181634F4812C912C88ED51
:105ED000A82E83E4B82E27E137EB41ED58E3C50146
:105EE000B4010F94E32C9B01AC01B1E0B983C7016D
:105EF000B6010F94132618160CF41982898128967E
:105F00000FB6F894DEBF0FBECDBFDF91CF91FF90EB
:105F1000EF90DF90CF90BF90AF909F908F907F9049
:105F20006F905F904F900895E6E0F8E082EBDF011C
:105F30001D928A95E9F708958091C105811104C0E9
:105F40000E94942F0C942FB88091261482FD0C94FB
:105F50007AF7089580910608882361F09091B70838
:105F6000891308C08091261483FF04C084E498E05C
:105F70000C94F9B680E00895FC01238121110C9462
:105F80002EB30895EFE6F0E080818260808308956B
:105F9000CF92DF92EF92FF92CF93DF93C82F0E94B0
:105FA000322A94E0C99FE0011124FE01EC50FA4F1F
:105FB000C080D180E280F38081110E94C22FC55A37
:105FC000DE4EC701B6010F941A26288139814A8115
:105FD0005B810F947926DF91CF91FF90EF90DF9056
:105FE000CF9008958F929F92AF92BF92CF92DF92FF
:105FF000EF92FF921F93CF93DF93CDB7DEB76097F9
:106000000FB6F894DEBF0FBECDBF182F80E00E9400
:10601000C82F4B015C018092800590928105A0926F
:106020008205B092830581E00E94C82F6B017C013C
:10603000C0928405D0928505E0928605F09287058E
:1060400082E00E94C82F6093880570938905809331
:106050008A0590938B051D861E861F86188A898265
:106060009A82AB82BC82CD82DE82EF82F88669871B
:106070007A878B879C8783E00E94C82F6D877E87F5
:106080008F87988B80912D0C882321F0CE0101966B
:106090000E9448211E3FD9F480E1FE013196ACE117
:1060A000BCE001900D928A95E1F760960FB6F894E6
:1060B000DEBF0FBECDBFDF91CF911F91FF90EF905C
:1060C000DF90CF90BF90AF909F908F90089584E025
:1060D000189FF0011124DF01A45EB34F81E090E02E
:1060E0008C0F9D1FE80FF91F4081518162817381E0
:1060F0004D935D936D937C931397D7CFCF92DF929F
:10610000EF92FF92CF93DF93C82F0E94322A94E040
:10611000C99FE0011124FE01E851FA4FC080D180EF
:10612000E280F38081110E94C22FC55ADE4EC70162
:10613000B6010F941A26288139814A815B810F9418
:106140007926DF91CF91FF90EF90DF90CF90089567
:106150000E94322A90917F1290937E1290937D122A
:1061600090937C1294E690937B1220ED33E0309371
:10617000F9082093F80881110E94C22F81E08093D2
:10618000E7050895CF93DF93CDB7DEB72C970FB611
:10619000F894DEBF0FBECDBF0E9497F60E94322A50
:1061A0009CE0E4EFF5E0DE01119601900D929A95E6
:1061B000E1F781110E94C22FCE0101960E946FC6A5
:1061C0002C960FB6F894DEBF0FBECDBFDF91CF91F6
:1061D00008952F923F924F925F926F927F928F928B
:1061E0009F92AF92BF92CF92DF92EF92FF920F9366
:1061F0001F93CF93DF9300D0CDB7DEB780901C0CF8
:1062000090901D0CA0901E0CB0901F0C4090200C84
:106210005090210C6090220C7090230CC090240CA4
:10622000D090250CE090260CF090270C0E94DB1BF0
:106230000E94291C09E71CE187E492E09B838A8382
:106240008DE6282E8CE1382E198289810E94CC1C83
:10625000C8010E94AF1DEA81FB8161937193819314
:106260009193FB83EA83C1010E94AF1DEA81FB8108
:106270006087718782879387F981FF5FF9830C5F5D
:106280001F4F84E0280E311CF330F9F682ED95E0C3
:106290000E94FCF60E94CB1E0E941027A5019401CB
:1062A00060911C0C70911D0C80911E0C90911F0C24
:1062B0000F94132681111CC0A30192016091200C40
:1062C0007091210C8091220C9091230C0F94132635
:1062D00081110EC02091240C3091250C4091260C88
:1062E0005091270CC701B6010F9413268823B9F0EB
:1062F0000F900F900F90DF91CF911F910F91FF9012
:10630000EF90DF90CF90BF90AF909F908F907F9055
:106310006F905F904F903F902F900C94C2300F90F1
:106320000F900F90DF91CF911F910F91FF90EF9001
:10633000DF90CF90BF90AF909F908F907F906F90A5
:106340005F904F903F902F90089580916F119091A2
:106350007011892B79F480916F1190917011892BB4
:1063600049F420916F113091701181E0232B19F4C1
:1063700080E0089581E008951092E1048091220266
:1063800090912302A0912402B09125028093DE0512
:106390009093DF05A093E005B093E10508959091F7
:1063A000861110928611923071F0943079F091300C
:1063B00099F4813089F48091E104882369F0109286
:1063C00026020C94BC3110921B0C089580E898E1D1
:1063D00090937B0C80937A0C08959091261493FBF4
:1063E000882780F993FF06C081E090918D15911167
:1063F00001C080E00895CF93C0917E05CF7739F535
:106400000E94ED31882319F180911E1490911F1480
:10641000A0912014B09121140097A105B105B9F005
:10642000BC01CD016D597F4F8F4F9F4F24E630E067
:1064300040E050E00F94572C609122147091231487
:1064400080912414909125140F94572CC22F8C2FD7
:10645000CF910895E5EFF8E010821182089581E070
:106460000895DC01EC918E2F90E0FC01EE0FFF1FF0
:10647000E80FF91FEF5DFD4E80818F7780830895CF
:106480008F929F92AF92BF92CF92DF92EF92FF9244
:106490000F93CF93DF931F92CDB7DEB75C017B01E3
:1064A00049016B01C40ED51EF501808191810F94C5
:1064B000312C8983002311F0F7018083BE016F5FC7
:1064C0007F4FC4010E9416E1F50180819181019600
:1064D00091838083FFEFEF1AFF0AEC14FD0421F78C
:1064E00080E00F90DF91CF910F91FF90EF90DF90C0
:1064F000CF90BF90AF909F908F9008950F93AB0176
:106500000091D60521E0022727ED35E0BC0187EB9D
:1065100095E00E9440320F910895009781F4109207
:10652000900082E080939100109295001092940068
:10653000C19A8091710082608093710008950197E3
:1065400061F41092A00082E08093A1001092A50057
:106550001092A40089BB8093720008957F928F925D
:106560009F92AF92BF92CF92DF92EF92FF920F93E2
:106570001F93CF93DF93EC017B018881883108F072
:10658000C3C090E0FC01EE0FFF1FE80FF91FEF5DA5
:10659000FD4E80818F770E9462E719821A8288817E
:1065A0002CE0622F0F94BA2C829FB001112430E0AE
:1065B00020E0AB01420F531FFA01EE0FFF1FE40F63
:1065C000F51FEF5DFD4E908197FD08C02F5F3F4F97
:1065D0002C30310571F790E00E948D327880072DC4
:1065E00010E06801CC0CDD1CF601E00FF11FEF5D3F
:1065F000FD4E80818068808377FC86C080E2E8164B
:1066000082E0F8060CF03FC08A8128E532E0281BC2
:10661000310987FD3395220F331F220F331F032EBD
:10662000000C440B550B898178E8872E912C881A31
:10663000910887FD9394880C991C880C991C092C4F
:10664000000CAA08BB0860E070E0CB01F7FC0AC0B0
:10665000B701653B710514F064EB70E0072E000C88
:10666000880B990B281939094A095B090F94472CA3
:1066700024EB30E040E050E00F94792C820E931E22
:10668000A41EB51E740187E18715D8F0298188E81A
:1066900090E0821B910927FD9395880F991F880F21
:1066A000991FE816F90604F502972FB7F894E6014A
:1066B000C00FD11FCF5DDD4E880F991F9A8389834C
:1066C0002FBF62E370E080E090E0DF91CF911F91F7
:1066D0000F91FF90EF90DF90CF90BF90AF909F9081
:1066E0008F907F900C9432262A8188E592E0821B5D
:1066F000910927FD9395880F991F880F991FE81618
:10670000F90694F6C701D0CFDF91CF911F910F9179
:10671000FF90EF90DF90CF90BF90AF909F908F90C1
:106720007F900895CF93DF93EB01682F70E08AE6A6
:1067300092E10E94AE32688179818A819B81643FB7
:1067400021E072078105910520F464EF71E080E09B
:1067500090E00E94322689B182FB882780F9DF9180
:10676000CF910895CF93DF9300D01F92CDB7DEB7BE
:106770008EEE92E0A0E0B0E089839A83AB83BC8385
:10678000BE016F5F7F4F8AE50E9492330F900F909A
:106790000F900F90DF91CF910895CF93DF9300D0AA
:1067A0001F92CDB7DEB78EEE92E0A0E0B0E0898315
:1067B0009A83AB83BC83BE016F5F7F4F8AE00E94E8
:1067C00092330F900F900F900F90DF91CF9108951B
:1067D000CF93DF9300D01F92CDB7DEB784EF91E067
:1067E000A0E0B0E089839A83AB83BC83BE016F5F76
:1067F0007F4F80EA0E9492330F900F900F900F907E
:10680000DF91CF9108951F920F920FB60F9211242E
:106810000BB60F922F933F934F935F936F937F939A
:106820008F939F93AF93BF93EF93FF9348EA50E00A
:1068300064EA70E081E090E00E945626FF91EF91BB
:10684000BF91AF919F918F917F916F915F914F9188
:106850003F912F910F900BBE0F900FBE0F901F9086
:1068600018951F920F920FB60F9211240BB60F922C
:106870002F933F934F935F936F937F938F939F9348
:10688000AF93BF93EF93FF9348E950E064E970E062
:1068900090E080E00E945626FF91EF91BF91AF916A
:1068A0009F918F917F916F915F914F913F912F9128
:1068B0000F900BBE0F900FBE0F901F9018959091E8
:1068C000D10095FD0CC09091D00095FF08C0809339
:1068D000D6008091D00080648093D00008952091EC
:1068E0000E042F5F2F770FB607FC27C090910F047F
:1068F000921328C09091D00095FF1EC090910F0474
:1069000040910E04941306C09091D1009F7D909306
:10691000D10012C0E92FF0E0E25FFB4F32819F5FB0
:106920009F773093D60090930F043091D00030645D
:106930003093D000491741F3D9CF90910F049213AF
:1069400001C0FBCFE0910E04F0E0E25FFB4F8283D9
:1069500020930E048091D10080628093D10008952D
:106960008F929F92AF92BF92CF92DF92EF92FF925F
:106970000F931F93CF93DF937C0121E5E20EF11C6F
:10698000D7014C914A3509F0A4C06C01B2E5CB0E99
:10699000D11CF6013081353A09F09BC0EC01C05B97
:1069A000DF4F2881233008F494C08C0100561F4F1C
:1069B000D8014C93E15BFF4F308331962083EF5435
:1069C000F1093081E05BFF4F30833038B1F431960C
:1069D000AC54B1093C913083E854F109AF5ABF4F30
:1069E00050E040E02250330B42175307CCF4808133
:1069F00032968D934F5F5F4FF7CF233031F53138AB
:106A000009F074C0FC01EC55FF4FDC01AC5ABF4FDC
:106A10002C9120833196885A9F4FDC018C91808382
:106A20004801B12CA12C888190E002968A159B0523
:106A30000CF43FC0F40181914F010E945F340E9429
:106A40002CE1FFEFAF1ABF0AEECF323821F5FC017F
:106A5000EC5AFF4F30814181E05BFF4F408331961C
:106A60003083DC01AA55BF4F50E040E02350330B88
:106A700042175307ACF6FA01EE7FE45AFF4FE80FD6
:106A8000F91F608171817C9311966C9311974E5F11
:106A90005F4F1296EDCF243019F6333809F6FC011A
:106AA000EC5AFF4F20813181E05BFF4F30833196FC
:106AB000B0CF80E5DE011D928A95E9F78AE1F80101
:106AC00011928A95E9F78AE5D7018C9385EAF60158
:106AD0008083DF91CF911F910F91FF90EF90DF9016
:106AE000CF90BF90AF909F908F900895323809F06B
:106AF00097CFADCFAF92BF92CF92DF92EF92FF923E
:106B00000F931F93CF93DF93EC0184E6C82E80E2AE
:106B1000D82EE12CF12C02E8A12C90E2B92E15E040
:106B20000093B313C092B413D092B513E092B6138E
:106B3000F092B713B092BD13A092BC131093B01390
:106B400080E693E10E94B0348FEFC81AD80AE80AB1
:106B5000F80A88E7C81680E2D806E104F10401F7D4
:106B600024E630E240E050E0BE0180E693E1DF91B0
:106B7000CF911F910F91FF90EF90DF90CF90BF903A
:106B8000AF900C9431E1CF92DF92EF92FF920F938E
:106B90001F93CF93DF93CDB7DEB77C01CDB6DEB6C2
:106BA0000F94602501962DB73EB7281B390B0FB601
:106BB000F8943EBF0FBE2DBF0DB71EB70F5F1F4F1E
:106BC000B701C8010F945925C8010E947A350FB644
:106BD000F894DEBE0FBECDBEDF91CF911F910F9115
:106BE000FF90EF90DF90CF9008958F929F92AF9299
:106BF000BF92CF92DF92EF92FF920F931F93CF93AA
:106C0000DF930E94D42C3AE0C32E30E2D32EE12C45
:106C1000F12C15E002E846015701CAE0D0E01092DD
:106C2000BD131092BC131093B0130093B313809252
:106C3000B4139092B513A092B613B092B71380E636
:106C400093E10E94B03421978FEF881A980AA80A1E
:106C5000B80A209721F78AE0C80ED11CE11CF11C6C
:106C600082EDC81680E2D806E104F104A1F6C12C39
:106C700020E2D22EE12CF12CD5E0C2E81092BD1317
:106C80001092BC13D093B013C093B313C092B4133B
:106C9000D092B513E092B613F092B71380E693E169
:106CA0000E94B0341092BD131092BC13D093B01355
:106CB000C093B313D701C6018C529F4FAF4FBF4F44
:106CC0008093B4139093B513A093B613B093B713F6
:106CD00080E693E10E94B0348FEFC81AD80AE80A20
:106CE000F80A8AE0C81680E2D806E104F10431F619
:106CF0009EEDC92E90E2D92EE12CF12CD5E0C2E810
:106D00001092BD131092BC13D093B013C093B31361
:106D1000C092B413D092B513E092B613F092B713A9
:106D200080E693E10E94B0348FEFC81AD80AE80ACF
:106D3000F80A86EEC81680E2D806E104F10401F7ED
:106D4000CC24C39482E1D82EE12CF12C0AE010E08F
:106D5000D5E0C2E81093BD130093BC13D093B013D9
:106D6000C093B313C092B413D092B513E092B6138C
:106D7000F092B71380E693E10E94B0341093BD13F4
:106D80000093BC13D093B013C093B313D701C601C3
:106D90008096A11DB11D8093B4139093B513A09359
:106DA000B613B093B71380E693E10E94B0348FEF2F
:106DB000C81AD80AE80AF80A85E1C81682E1D80696
:106DC000E104F10439F682E190E09093BD138093E1
:106DD000BC13D093B013C093B31384E190E1A0E04F
:106DE000B0E08093B4139093B513A093B613B0930F
:106DF000B71380E693E1DF91CF911F910F91FF9040
:106E0000EF90DF90CF90BF90AF909F908F900C94B9
:106E1000B0341F920F920FB60F9211240BB60F923F
:106E20002F938F939F93EF93FF9380910F04209163
:106E30000E04821306C08091D1008F7D8093D10013
:106E400012C0E82FF0E0E25FFB4F92818F5F8F77F7
:106E50009093D60080930F049091D000906490930B
:106E6000D000281741F3FF91EF919F918F912F91BF
:106E70000F900BBE0F900FBE0F901F9018951F9292
:106E80000F920FB60F9211240BB60F920F931F9310
:106E90002F933F934F935F936F937F938F939F9322
:106EA000AF93BF93CF93DF93EF93FF93C091D6003F
:106EB00000913205D091310511E01D0F1F739091A3
:106EC0000D04913108F09FC0E92FF0E08827E459C4
:106ED000F84C8F4F0D94DA2C7D37AC37BB37CA375F
:106EE000D1370338D5370338D937DD370338E137A1
:106EF000E537E937F0370338FB37C03229F028F59A
:106F0000CA3011F0CD3031F5011731F0ED2FF0E03E
:106F1000EF5CFA4FC283D12FD0933105FF91EF91EF
:106F2000DF91CF91BF91AF919F918F917F916F91A1
:106F30005F914F913F912F911F910F910F900BBE39
:106F40000F900FBE0F901F901895CD3481F081E007
:106F5000CE3471F080E10CC0CA3338F4C033A0F6EF
:106F6000C03291F2CD32B1F7CFCFCD3499F782E074
:106F700080930D04C9CFC13359F018F4C03221F207
:106F8000E9CF88E0C433A1F38BE0C83389F3E2CFC3
:106F900083E0EECF84E0C03359F386E0C13341F3A0
:106FA000D9CF85E0C833B1F6E3CF87E0C23391F69D
:106FB000DFCF89E0C13371F6DBCF8AE0C03351F611
:106FC000D7CF8CE0C73331F6D3CF8DE0C63311F67F
:106FD000CFCFC03209F498CF8EE0C33549F2BACF93
:106FE00080ED8C0F8A3008F08FCF9FE090930D04D6
:106FF00080930C0489CFCA3019F0CD3009F084CFCA
:1070000010920D0481CFCA3019F0CD3009F07CCF39
:1070100080911A148823A1F3973089F038F49530C1
:1070200079F710923C0210921B0CEACF9A3059F07B
:107030009F3031F780910C040E94CF31E1CF81E085
:1070400080930506DDCF81E080930406D9CF90912F
:10705000C00095FFFCCF8093C6000895CF93DF93C7
:10706000EC018991882319F00E942738FACF8DE02E
:107070000E9427388AE0DF91CF910C942738CF9275
:10708000DF92EF92FF92CF936B017C01C42F4A30C5
:1070900069F4F7FE0BC0F094E094D094C094C11C46
:1070A000D11CE11CF11C8DE20E9427384C2FC70136
:1070B000B601CF91FF90EF90DF90CF900C9467AA2C
:1070C000CF93DF93EC01FE0184912196882319F080
:1070D0000E942738F8CFDF91CF910895CF93DF93A7
:1070E000D091191185E59CE10E9460388AE00E94E8
:1070F00027388091980C873009F449C083E0809349
:10710000930C81E080936E0280E190E09093BD1338
:107110008093BC1385E08093B013C2E8C093B3138F
:1071200084E190E1A0E0B0E08093B4139093B513B4
:10713000A093B613B093B71380E693E10E94B034E6
:1071400061E070E080E090E00E94B92C81E09AE577
:107150009093BD138093BC1385E390E09093BF138D
:107160008093BE1387E08093B013C093B31384E879
:1071700090E0A0E0B0E08093B4139093B513A09397
:10718000B613B093B71380E693E10E94B0348091B8
:107190001911813089F1823061F50E94A62B60932C
:1071A0009F057093A0058093A1059093A20581E0AF
:1071B000809319110E9472FD60939B0570939C054A
:1071C00080939D0590939E05D23089F0809188062A
:1071D0009091890601969093890680938806109273
:1071E000A7051092A8051092A9051092AA0581E0A2
:1071F00004C00E94D82BDBCF80E0DF91CF910895AF
:10720000CF93C82FCB010E94603889EC98E10E948F
:1072100060388AEB98E1CC2311F08FEB98E10E9463
:1072200060388AE0CF910C942738CF93DF9300D059
:107230001F92CDB7DEB784EF91E0A0E0B0E0898384
:107240009A83AB83BC83BE016F5F7F4F8CE30E9448
:10725000923387EE98E10E9460388CB161EE78E15C
:1072600085FB882780F90E940039809103016BED2E
:1072700078E1869581700E94003989B165ED78E1E9
:1072800082FB882780F90E9400398CB16CEC78E190
:10729000829581700E9400394A9909C00E94CD33BD
:1072A0000F900F900F900F90DF91CF9108950E9453
:1072B000B2330F900F900F900F90DF91CF91089500
:1072C000809119118130C1F585E998E10E946038FB
:1072D0008AE00E94273881E09AE59093BD1380935D
:1072E000BC1387E590E09093BF138093BE1387E0B3
:1072F0008093B01382E88093B31384E890E0A0E019
:10730000B0E08093B4139093B513A093B613B093E9
:10731000B71380E693E10E94B03482E080931911A4
:107320000E9472FD6093A3057093A4058093A50548
:107330009093A60581E0089580E008950F931F9330
:107340000E9472FD009183061091840620918506AB
:1073500030918606011511052105310509F067C038
:1073600020919212222309F45FC0E09190122150E3
:107370002093921221E02E0F2093901230919312BD
:10738000231302C01092901224E0E29FF001112416
:10739000EC56FD4E008111812281338100937F06DE
:1073A000109380062093810630938206600F711F30
:1073B000811D911D609383067093840680938506DA
:1073C000909386068091810690918206892B61F1C7
:1073D0001FB7F89484E898E10E9460388AE00E9420
:1073E000273884E096E09093BD138093BC1380EA25
:1073F00090E89093BF138093BE1387E08093B013FF
:1074000082E88093B31380EA90E0A0E0B0E080933C
:10741000B4139093B513A093B613B093B71380E64B
:1074200093E10E94B0341FBF1F910F910895601B1C
:10743000710B820B930B97FDF7CF40981092830648
:10744000109284061092850610928606EDCF0F9357
:107450001F93CF93DF938C01EB01909192122091B7
:107460009312921305C00E949E390E942FC2F5CF3D
:107470008091911234E0839FF0011124EC56FD4E6F
:1074800011830083D383C2839F5F909392128F5F97
:10749000281739F080939112DF91CF911F910F91AE
:1074A000089510929112F8CFCF92DF92EF92FF924F
:1074B0001F93CF93DF93182F662351F01092E004AF
:1074C0001092DC041092DD041092DE041092DF04AE
:1074D0000E9472FD6B017C018091DC049091DD04BF
:1074E000A091DE04B091DF04A7019601281B390B9F
:1074F0004A0B5B0BDA01C901B7FD3DC02091E004E6
:1075000017FD13C0412F012E000C550B4C5F5F4F30
:10751000822F022E000C990B4817590764F184EF53
:1075200091E0A0E0B0E0211724F488EE93E0A0E021
:10753000B0E08C0D9D1DAE1DBF1D8093DC049093AB
:10754000DD04A093DE04B093DF042170C22F30E08D
:10755000D32F84E28C9FB0018D9F700D7C1B112472
:1075600060597C4F82E390E00E94273A8091E004CA
:107570008F5F8093E004DF91CF911F91FF90EF9098
:10758000DF90CF900895CF93DF9300D01F92CDB7B7
:10759000DEB78AE098E10E9460388AE00E942738CE
:1075A0008091980C8330D9F119821A821B821C8237
:1075B00060E0CE0101960E94F32B19821A821B8291
:1075C0001C8261E0CE0101960E94F32B81E0809342
:1075D0006D021092920C80936E0281E09AE5909376
:1075E000BD138093BC1383E390E09093BF1380930B
:1075F000BE1387E08093B01382E88093B31384E8CE
:1076000090E0A0E0B0E08093B4139093B513A09302
:10761000B613B093B71380E693E10E94B0340F9095
:107620000F900F900F90DF91CF9108956F927F92FE
:107630008F929F92AF92BF92CF92DF92EF92FF9282
:107640000F931F93CF93DF93CDB7DEB764970FB639
:10765000F894DEBF0FBECDBF1092D0008091D00055
:1076600082608093D0001092D50080E18093D40096
:107670008091D10080618093D1008091D100886099
:107680008093D1008091D10080688093D100809157
:10769000D1008F7D8093D1008AE58093B1138093D0
:1076A000611385EA8093B21380936213E0E0F4E102
:1076B0008AE1DF011D928A95E9F78091910C882378
:1076C00009F473C283E090E09093BD138093BC13E0
:1076D00085E08093B01382E88093B3138FE190E14B
:1076E000A0E0B0E08093B4139093B513A093B613C9
:1076F000B093B71380E693E10E94B03484E690E043
:107700009093BD138093BC1305E00093B01312E86F
:107710001093B31386E090E1A0E0B0E08093B4133F
:107720009093B513A093B613B093B71380E693E18B
:107730000E94B0348BE090E09093BD138093BC1313
:107740000093B0131093B31380E092E1A0E0B0E097
:107750008093B4139093B513A093B613B093B7135B
:1077600080E693E10E94B0341092BD131092BC13D6
:107770000093B0131093B31384E390E1A0E0B0E062
:107780008093B4139093B513A093B613B093B7132B
:1077900080E693E10E94B0341092BD131092BC13A6
:1077A0000093B0131093B3138AE390E1A0E0B0E02C
:1077B0008093B4139093B513A093B613B093B713FB
:1077C00080E693E10E94B0348091E0119091E11144
:1077D0009093BD138093BC130093B0131093B31315
:1077E00086E390E1A0E0B0E08093B4139093B513EA
:1077F000A093B613B093B71380E693E10E94B03420
:1078000080917511909176119093BD138093BC1364
:107810000093B0131093B3138CE390E1A0E0B0E0B9
:107820008093B4139093B513A093B613B093B7138A
:1078300080E693E10E94B03482E090E09093BD1323
:107840008093BC130093B0131093B3138EE190E1B7
:10785000A0E0B0E08093B4139093B513A093B61357
:10786000B093B71380E693E10E94B03481E0809337
:107870006D0270E6C72E70E1D72EE12CF12C10922C
:10788000BD131092BC130093B0131093B313C092A6
:10789000B413D092B513E092B613F092B71380E60A
:1078A00093E10E94B034BFEFCB1ADB0AEB0AFB0A6C
:1078B000E4E7CE16E0E1DE06E104F10401F7CE01D3
:1078C00001967C0184E1D7011D928A95E9F781E058
:1078D0008F9396ED9F938F9392EC9F938F939F93AB
:1078E0008BE893E09F938F93FF92EF920F946B300E
:1078F00020E630E140E050E068E973E080E693E1A3
:107900000E9431E12AE630E140E050E061EA73E0B4
:1079100080E693E10E9431E124E730E140E050E06D
:10792000B70180E693E10E9431E12EE730E140E0CB
:1079300050E06FEA73E080E693E10E9431E110923B
:10794000BD131092BC130093B0131093B3138EE0C9
:1079500090E1A0E0B0E08093B4139093B513A093AE
:10796000B613B093B71380E693E10E94B03410923F
:10797000BD131092BC130093B0131093B3138FE098
:1079800090E1A0E0B0E08093B4139093B513A0937E
:10799000B613B093B71380E693E10E94B0340FB6EC
:1079A000F894DEBF0FBECDBF4AE0C42E40E2D42E15
:1079B000E12CF12C55E0752E62E8662E4601570148
:1079C0000AE010E01092BD131092BC137092B01335
:1079D0006092B3138092B4139092B513A092B61331
:1079E000B092B71380E693E10E94B03401501109C0
:1079F000FFEF8F1A9F0AAF0ABF0A0115110511F791
:107A00008AE0C80ED11CE11CF11C92EDC91690E26F
:107A1000D906E104F10491F6C12C30E2D32EE12C19
:107A2000F12C05E012E81092BD131092BC130093E4
:107A3000B0131093B313C092B413D092B513E09265
:107A4000B613F092B71380E693E10E94B03410921F
:107A5000BD131092BC130093B0131093B313D7014E
:107A6000C6018C529F4FAF4FBF4F8093B41390937A
:107A7000B513A093B613B093B71380E693E10E94B9
:107A8000B034AFEFCA1ADA0AEA0AFA0ABAE0CB1639
:107A9000B0E2DB06E104F10431F62EEDC22E20E265
:107AA000D22EE12CF12C05E012E81092BD131092B9
:107AB000BC130093B0131093B313C092B413D092BD
:107AC000B513E092B613F092B71380E693E10E94EB
:107AD000B034EFEFCE1ADE0AEE0AFE0AF6EECF164B
:107AE000F0E2DF06E104F10401F7CC24C39482E163
:107AF000D82EE12CF12C9AE0A92EB12C05E012E849
:107B0000B092BD13A092BC130093B0131093B313A3
:107B1000C092B413D092B513E092B613F092B7139B
:107B200080E693E10E94B034B092BD13A092BC13E2
:107B30000093B0131093B313D701C6018096A11D13
:107B4000B11D8093B4139093B513A093B613B09363
:107B5000B71380E693E10E94B0348FEFC81AD80AB9
:107B6000E80AF80A95E1C91692E1D906E104F104A0
:107B700039F680E797E10E9460388AE00E94273852
:107B800064960FB6F894DEBF0FBECDBFDF91CF91E4
:107B90001F910F91FF90EF90DF90CF90BF90AF902B
:107BA0009F908F907F906F90089582E090E08CCDB1
:107BB0000E94163B10927A0581E080936E0282E269
:107BC00098E10E9460388AE00C9427380F931F9345
:107BD000CF938C01C62F80E294E10E946038C801E7
:107BE0000E9460388AE30E94273880E38C0F0E944D
:107BF00027388AE0CF911F910F910C94273883EAA0
:107C000095E10E94603860E083E995E10E94E63DDD
:107C100060E08EE795E10E94E63D61E087E795E14F
:107C20000E94E63D61E08CE695E10E94E63D61E060
:107C30008CE595E10E94E63D60E083E595E10E94D8
:107C4000E63D61E089E495E10E94E63D61E08FE375
:107C500095E10E94E63D61E088E395E10E94E63D02
:107C600061E080E395E10E94E63D61E082E295E11A
:107C70000E94E63D61E084E195E10E94E63D60E01E
:107C800085E095E10E94E63D60E087EF94E10E9487
:107C9000E63D60E081EE94E10E94E63D61E080ED2A
:107CA00094E10E94E63D61E081EC94E10E94E63DB2
:107CB00061E08AEB94E10E94E63D60E083EB94E1B1
:107CC0000E94E63D61E08AEA94E10E94E63D61E0BF
:107CD00085E994E10E94E63D61E087E894E10E9435
:107CE000E63D61E084E794E10E94E63D60E087E6DE
:107CF00094E10E94E63D61E082E694E10E94E63D67
:107D000061E085E594E10E94E63D60E081E494E174
:107D10000E94E63D60E08EE294E10E94E63D60E074
:107D200089E294E10E94921D682F617085E294E1DE
:107D30000C94E63D80912B05827149F480912D05CC
:107D40008C7829F480912E05837009F475C082E443
:107D50000E94701E882351F00E943E2460933E0CC6
:107D600070933F0C8093400C9093410C83E50E94EC
:107D7000701E882351F00E94C42460936E0C70938F
:107D80006F0C8093700C9093710C84E50E94701EB0
:107D9000882351F00E94C4246093720C7093730C7A
:107DA0008093740C9093750C88E50E94701E882354
:107DB00051F00E94C4246093D1087093D20880933C
:107DC000D3089093D40889E50E94701E882351F04F
:107DD0000E94C4246093D5087093D6088093D70876
:107DE0009093D8088AE50E94701E8823B1F00E9403
:107DF000C4246093D9087093DA088093DB089093C9
:107E0000DC082DEC3CEC4CEC5DE30F9413261816CB
:107E100024F088E99EE00E94603885E40E94701E8C
:107E2000882351F00E94C4246093DD087093DE081B
:107E30008093DF089093E0080895AF92BF92CF92AD
:107E4000DF92EF920F931F93CF93DF935B01EA01D1
:107E50006901882309F463C081E99EE00E946038CB
:107E6000F501608171818281938146E00E946FBA41
:107E7000E1100BC088E89EE00E946038688179813B
:107E80008A819B8146E00E946FBA81E89EE00E9451
:107E90006038F601608171818281938143E00E94A4
:107EA0006FBA8AE79EE00E946038F80160817181B4
:107EB0008281938143E00E946FBA81E79EE00E9435
:107EC0006038F6012081318142815381F80160815F
:107ED0007181828193810F94E22C43E00E946FBAFA
:107EE000EE20F9F08AE00E9427388CE59EE00E949F
:107EF0006038688179818A819B8146E00E946FBAEF
:107F00008AE00E9427388AE0DF91CF911F910F917C
:107F1000EF90DF90CF90BF90AF900C942738E11096
:107F2000E4CFDF91CF911F910F91EF90DF90CF9031
:107F3000BF90AF9008950F931F93CF938C01C62FDE
:107F400089E798E00E946038C8010E946038CC231D
:107F500031F08AE0CF911F910F910C942738CF9187
:107F60001F910F9108950E94CAE410921B0C109269
:107F70003C020E94ED31882351F08091261482FD4D
:107F800006C080E898E190937B0C80937A0C61E0C6
:107F900089E798E10E949B3F0C946E380F931F93E2
:107FA000CF93DF938C016F3F19F410925A1160E068
:107FB00020915A11862F062E000C990B28171906AE
:107FC00009F08CF560935A1160E083E498E10E9417
:107FD0009B3FC8010E9460388AE00E942738C80190
:107FE0000F946025800F911FEC01C01BD10BC03492
:107FF000D1053CF00197FC012491207C2038D1F37D
:10800000F3CFDD27AE01B8018AE191E10F9481251C
:10801000C65EDE4E18828AE191E1DF91CF911F9119
:108020000F910C947A35DF91CF911F910F910895A4
:1080300010921B0C10923C02809126148064809355
:10804000261461E081E598E10E949B3F46E658E1F5
:108050006EE678E185E00E944FE360E088E598E114
:108060000C94CE3F0F931F93CF938C01C62F60E0EB
:1080700083E898E00E949B3FC8010E946038CC23AF
:1080800031F08AE0CF911F910F910C942738CF9156
:108090001F910F91089561E08BE898E00C943240B5
:1080A000EF92FF920F931F93CF937C018B01C42F0C
:1080B00060E083E898E00E949B3FC7010E9460381F
:1080C00080E20E942738C8010E946038CC2319F052
:1080D0008C2F0E9427388AE0CF911F910F91FF903B
:1080E000EF900C942738DF92EF92FF920F931F933B
:1080F000CF93DF93D82E7B018A01E9010E944B4088
:10810000D092861140E0B70184E799E00E94504088
:108110000115110531F040E0B8018DE699E00E94AB
:108120005040209731F040E0BE018DE699E00E947A
:10813000504061E088E699E0DF91CF911F910F9167
:10814000FF90EF90DF900C943240AF92BF92CF92AD
:10815000DF92EF92FF920F931F93CF93DF9386EE00
:1081600097E00E946038C0E0D7E0D15021F080E273
:108170000E942738FACF8C2F0E9488E1CF5FC5304C
:1081800099F78AE00E94273804E817E0C0E080E20F
:108190000E9427388C2F0E9488E15801D5E080E2A8
:1081A0000E942738F501C080D180E280F380A701CA
:1081B0009601C701B6010F94D52F882369F180E29B
:1081C0000E9427388DE30E9427388DE30E942738CC
:1081D0008DE30E9427388DE30E9427388DE30E94AB
:1081E0002738D150F4E1AF0EB11CD111D8CF8AE0BD
:1081F0000E942738CF5F0C5F1F4FC53041F68AE0E1
:10820000DF91CF911F910F91FF90EF90DF90CF9072
:10821000BF90AF900C94273820E030E0A901C7014F
:10822000B6010F94432F87FD03C08BE20E942738CD
:1082300043E0C701B6010E946FBAD3CF811107C0D6
:108240008AEC9EE00E9460388AE00C9427388EEC1D
:108250009EE0F8CFCF93DF93EB010E946038CE0110
:10826000DF91CF910C9446E2CF93C62F0E946038E5
:108270008C2FCF910C9488E1CF92DF92EF92FF92F6
:108280006A017B010E94603842E0C701B601FF909D
:10829000EF90DF90CF900C946FBACF92DF92EF9275
:1082A000FF926A017B010E9460384AE0C701B60173
:1082B000FF90EF90DF90CF900C943F38CF93DF93F7
:1082C000EB010E946038CE01DF91CF910C948FE1D9
:1082D0004F925F926F927F928F929F92AF92BF92D6
:1082E000CF92DF92EF92FF920F931F93CF93DF9382
:1082F00000D000D01F921F92CDB7DEB780917905D4
:1083000081110AC480917705909178059C012F5FB7
:108310003F4F30937805209377058E3E924008F4C6
:10832000FBC38091E0119091E1119093BD13809374
:10833000BC1305E00093B01312E81093B31386E367
:1083400090E1A0E0B0E08093B4139093B513A093B4
:10835000B613B093B71380E693E10E94B0348091D6
:108360007511909176119093BD138093BC13009377
:10837000B0131093B3138CE390E1A0E0B0E08093CE
:10838000B4139093B513A093B613B093B71380E6CC
:1083900093E10E94B0348091E2119091E3119093A7
:1083A000BD138093BC130093B0131093B31384E3F5
:1083B00090E1A0E0B0E08093B4139093B513A09344
:1083C000B613B093B71380E693E10E94B034809166
:1083D0007711909178119093BD138093BC13009303
:1083E000B0131093B3138AE390E1A0E0B0E0809360
:1083F000B4139093B513A093B613B093B71380E65C
:1084000093E10E94B03481E0809379051092780561
:10841000109277058091980C882339F10E94241DD1
:10842000811123C0809176058F5F809376058091BE
:108430007605853620F0109276051092980CE09122
:10844000980CE150E73008F06AC00E2E000CFF0BCC
:108450008827E25DFD4B8F4F0D94DA2C384287421E
:1084600053447F44C044F8448B4210927605DFCFDA
:108470000E94B12C882309F452C081E080936E02DF
:108480008CEF97E10E9460388AE00E94273880E1F3
:1084900090E09093BD138093BC1385E08093B0135C
:1084A00012E81093B31384E190E1A0E0B0E0809370
:1084B000B4139093B513A093B613B093B71380E69B
:1084C00093E10E94B03481E09AE59093BD138093CC
:1084D000BC1386E390E09093BF138093BE1387E0B4
:1084E0008093B0131093B31384E890E0A0E0B0E061
:1084F0008093B4139093B513A093B613B093B713AE
:1085000080E693E10E94B0341092980C08C00E945B
:10851000B12C882321F00E94241D8823A9F3809187
:108520006E02882309F433C780917A058111C0C295
:1085300084E096E09093BD138093BC1380EA90E8AA
:108540009093BF138093BE1317E01093B01302E80B
:108550000093B31380EA90E0A0E0B0E08093B413FE
:108560009093B513A093B613B093B71380E693E13D
:108570000E94B0348091690290916A02A0916B02CE
:10858000B0916C020097A105B10509F03FC21092AD
:10859000BD131092BC1315E01093B0130093B313E6
:1085A0008AE890E1A0E0B0E08093B4139093B51313
:1085B000A093B613B093B71380E693E10E94B03452
:1085C00089E090E09093BD138093BC131093B01397
:1085D0000093B3138CE890E1A0E0B0E08093B41373
:1085E0009093B513A093B613B093B71380E693E1BD
:1085F0000E94B0348091690290916A02A0916B024E
:10860000B0916C020097F1E0AF07B10508F441C2E8
:10861000B093BD13A093BC139093BF138093BE136C
:1086200087E08093B01382E88093B31388E890E1E9
:10863000A0E0B0E08093B4139093B513A093B61369
:10864000B093B71380E693E10E94B0348091690241
:1086500090916A02A0916B02B0916C02BA2FA92F7F
:10866000982F8827009721E0A207B10508F417C2C8
:10867000B093BD13A093BC139093BF138093BE130C
:1086800087E08093B01312E81093B31381EA90E06F
:10869000A0E0B0E08093B4139093B513A093B61309
:1086A000B093B71380E693E10E94B03480912D0C13
:1086B000882309F4FAC183E090E09093BD1380937E
:1086C000BC1385E08093B0131093B31385E490E15D
:1086D000A0E0B0E08093B4139093B513A093B613C9
:1086E000B093B71380E693E10E94B03480917A058D
:1086F000875E80937A0520917A05822F90E0253657
:1087000008F021C29093BD138093BC1385E0809341
:10871000B01382E88093B31380E090E1A0E0B0E072
:108720008093B4139093B513A093B613B093B7137B
:1087300080E693E10E94B0340E94241D811114C28E
:108740000E94ED31811105C090917D0591FD0E943F
:10875000241D90917D0580FB91F990937D0591FDFD
:1087600003C28091261482FDFFC1809119118150AE
:10877000823008F4F9C16091771170917811072E59
:10878000000C880B990B0F941A266B017C0120E0DA
:1087900030E0A9010F941326882309F4BBC6609129
:1087A000751170917611072E000C880B990B0F94A0
:1087B0001A262B013C0120E030E040E850E4C701DC
:1087C000B6010F94E22CA30192010F94432F1816C7
:1087D0000CF4C2C66091E0117091E111072E000CFB
:1087E000880B990B0F941A266D837E838F8398874D
:1087F0006091E2117091E311072E000C880B990B28
:108800000F941A264B015C0120E030E040E251E475
:108810000F94E22C2D813E814F8158850F94432F78
:1088200018160CF499C620E030E040E850E4C70187
:10883000B6010F94E32CA30192010F94132687FD38
:1088400010C020E030E040E251E4C501B4010F94D3
:10885000E32C2D813E814F8158850F94132687FF8D
:108860006AC684E190E09093BD138093BC1385E0C9
:108870008093B01382E88093B31384E190E1A0E089
:10888000B0E08093B4139093B513A093B613B09354
:10889000B71380E693E10E94B0348091930C81116C
:1088A0007CC682E07AC68EEE97E10E9460388AE04C
:1088B0000E94273881E09AE59093BD138093BC1302
:1088C00080E490E09093BF138093BE1317E0109361
:1088D000B01382E88093B31384E890E0A0E0B0E0A6
:1088E0008093B4139093B513A093B613B093B713BA
:1088F00080E693E10E94B0341093980C10CE8091E2
:10890000820C882309F40BCE0E94B12C882309F431
:1089100006CE0E94241D811102CE80EE97E10E94B6
:1089200060388AE00E9427388091830C90E0B0E0A4
:10893000A0E0895B9F4FAE4FB54A21E03AE5309306
:10894000BD132093BC139093BF138093BE1387E095
:108950008093B01382E88093B31384E890E0A0E0A2
:10896000B0E08093B4139093B513A093B613B09373
:10897000B71380E693E10E94B0341092820CC4CD0C
:108980000E94B12C882309F4CACD0E94241D8111B4
:10899000C6CD81E080936E021092980C82ED97E133
:1089A0000E9460388AE00E94273881E09AE590931F
:1089B000BD138093BC138EE490E09093BF1380931B
:1089C000BE1387E08093B01382E88093B31384E8EA
:1089D00090E0A0E0B0E08093B4139093B513A0931F
:1089E000B613B093B71380E693E10E94B03497CDED
:1089F0000E94241D811193CD19821A821B821C8230
:108A000062E0CE0101960E9417F57ECD0196A11D70
:108A1000B11D35E0B695A795979587953A95D1F70D
:108A20000197A109B1090097E1E0AE07B10548F14E
:108A3000B093BD13A093BC139093BF138093BE1348
:108A40001093B01312E81093B3138AE890E1A0E0FA
:108A5000B0E08093B4139093B513A093B613B09382
:108A6000B71380E693E10E94B03488E090E09093E1
:108A7000BD138093BC1385E08093B0131093B313A0
:108A8000A9CD9093BD138093BC1385E08093B01360
:108A9000D9CF9093BD138093BC1385E0C2CD909342
:108AA000BD138093BC1385E0ECCD82E090E005CE51
:108AB0008A3F08F020CE8EEF80937A0581EC97E113
:108AC0000E9460388AE00E94273881E080936E021D
:108AD00081E09AE59093BD138093BC138DE290E002
:108AE0009093BF138093BE1387E08093B01382E806
:108AF0008093B31384E890E0A0E0B0E08093B413D7
:108B00009093B513A093B613B093B71380E693E197
:108B10000E94B0341092790528960FB6F894DEBF03
:108B20000FBECDBFDF91CF911F910F91FF90EF90BE
:108B3000DF90CF90BF90AF909F908F907F906F907D
:108B40005F904F900895845691099093BD13809340
:108B5000BC1385E08093B01382E88093B31381E067
:108B600090E1A0E0B0E0DCCD8CE090E09093BD130C
:108B70008093BC1315E01093B01382E88093B31375
:108B800084E190E1A0E0B0E08093B4139093B5133A
:108B9000A093B613B093B71380E693E10E94B0346C
:108BA0000E94A62B20E13EE040E050E00F94572CBD
:108BB0002115310581E04807510508F470C0509334
:108BC000BD134093BC133093BF132093BE1387E0B3
:108BD0008093B01312E81093B31380E190E1A0E00A
:108BE000B0E08093B4139093B513A093B613B093F1
:108BF000B71380E693E10E94B0340E94A62B20E1D7
:108C00003EE040E050E00F94572C2CE330E040E091
:108C100050E00F94572C3093BD132093BC1305E004
:108C20000093B0131093B31382E190E1A0E0B0E0A1
:108C30008093B4139093B513A093B613B093B71366
:108C400080E693E10E94B0340E94FB31882309F44E
:108C50005CC48F5F80937505E82EF12C833330F56B
:108C6000EE0CFF1CF092BD13E092BC130093B01306
:108C70001093B3138EE090E1A0E0B0E08093B413C2
:108C80009093B513A093B613B093B71380E693E116
:108C90000E94B0341092BD131092BC132BC03093BD
:108CA000BD132093BC131093B01394CF84E690E0CF
:108CB0009093BD138093BC130093B0131093B31320
:108CC0008EE090E1A0E0B0E08093B4139093B513F0
:108CD000A093B613B093B71380E693E10E94B0342B
:108CE000A2E3EA1AA0E8FA0AEE0CFF1CF092BD1308
:108CF000E092BC130093B0131093B3138FE090E194
:108D0000A0E0B0E08093B4139093B513A093B61392
:108D1000B093B71380E693E10E94B0340E94FB3118
:108D200090E09093BD138093BC1385E08093B013C3
:108D300082E88093B31386E190E1A0E0B0E08093F5
:108D4000B4139093B513A093B613B093B71380E602
:108D500093E10E94B03420E030E0A90160917512E7
:108D60007091761280917712909178120F94E32C83
:108D700020E030E048EC52E40F9479260F944F2E17
:108D80007093BD136093BC1305E00093B01312E819
:108D90001093B31386E290E1A0E0B0E08093B413A7
:108DA0009093B513A093B613B093B71380E693E1F5
:108DB0000E94B03480916502909166029093BD1339
:108DC0008093BC130093B0131093B31380E093E12E
:108DD000A0E0B0E08093B4139093B513A093B613C2
:108DE000B093B71380E693E10E94B03420E030E006
:108DF00040E251E46091420C7091430C8091440C2C
:108E00009091450C0F9479260F94562E7093BD13B4
:108E10006093BC130093B0131093B31382E492E1F8
:108E2000A0E0B0E08093B4139093B513A093B61371
:108E3000B093B71380E693E10E94B03420E030E0B5
:108E400040E251E46091460C7091470C8091480CCF
:108E50009091490C0F9479260F94562E7093BD1360
:108E60006093BC130093B0131093B31386E492E1A4
:108E7000A0E0B0E08093B4139093B513A093B61321
:108E8000B093B71380E693E10E94B03420E030E065
:108E900040E251E460914A0C70914B0C80914C0C73
:108EA00090914D0C0F9479260F94562E7093BD130C
:108EB0006093BC130093B0131093B3138AE492E150
:108EC000A0E0B0E08093B4139093B513A093B613D1
:108ED000B093B71380E693E10E94B03420E030E015
:108EE00040E251E460914E0C70914F0C8091500C17
:108EF0009091510C0F9479260F94562E7093BD13B8
:108F00006093BC130093B0131093B3138EE492E1FB
:108F1000A0E0B0E08093B4139093B513A093B61380
:108F2000B093B71380E693E10E94B03420E030E0C4
:108F300048EC52E460916D1270916E1280916F1244
:108F4000909170120F9479260F944F2E7093BD1349
:108F50006093BC130093B0131093B31386E392E1B4
:108F6000A0E0B0E08093B4139093B513A093B61330
:108F7000B093B71380E693E10E94B03420E030E074
:108F800048EC52E4609171127091721280917312E8
:108F9000909174120F9479260F944F2E7093BD13F5
:108FA0006093BC130093B0131093B3138AE392E160
:108FB000A0E0B0E08093B4139093B513A093B613E0
:108FC000B093B71380E693E10E94B03480917502AC
:108FD000909176029093BD138093BC130093B013CD
:108FE0001093B31382E592E1A0E0B0E08093B41354
:108FF0009093B513A093B613B093B71380E693E1A3
:109000000E94B03480917302909174029093BD13CA
:109010008093BC130093B0131093B31384E592E1D3
:10902000A0E0B0E08093B4139093B513A093B6136F
:10903000B093B71380E693E10E94B03420E030E0B3
:1090400040E251E46091E5117091E6118091E711E1
:109050009091E8110F9479260F94562E7093BD13BA
:109060006093BC130093B0131093B31386E592E1A1
:10907000A0E0B0E08093B4139093B513A093B6131F
:10908000B093B71380E693E10E94B0342CEA35EC3C
:1090900047E25EE36091E9117091EA118091EB1172
:1090A0009091EC110F94DD2D20E030E040E251E48E
:1090B0000F9479260F94562E7093BD136093BC13B2
:1090C0000093B0131093B3138AE592E1A0E0B0E0EF
:1090D0008093B4139093B513A093B613B093B713C2
:1090E00080E693E10E94B0342CEA35EC47E25EE37F
:1090F0006091ED117091EE118091EF119091F0114E
:109100000F94792620E030E040E251E40F94792674
:109110000F94562E7093BD136093BC130093B0133D
:109120001093B3138EE592E1A0E0B0E08093B41306
:109130009093B513A093B613B093B71380E693E161
:109140000E94B03420E030E040E251E460917A11B6
:1091500070917B1180917C1190917D110F947926F3
:109160000F94562E7093BD136093BC130093B013ED
:109170001093B31382E692E1A0E0B0E08093B413C1
:109180009093B513A093B613B093B71380E693E111
:109190000E94B0342CEA35EC47E25EE360917E1128
:1091A00070917F1180918011909181110F94DD2D2C
:1091B00020E030E040E251E40F9479260F94562EDF
:1091C0007093BD136093BC130093B0131093B3134B
:1091D00086E692E1A0E0B0E08093B4139093B513DB
:1091E000A093B613B093B71380E693E10E94B03416
:1091F0002CEA35EC47E25EE36091821170918311B5
:1092000080918411909185110F94792620E030E0AF
:1092100040E251E40F9479260F94562E7093BD13BB
:109220006093BC130093B0131093B3138AE692E1DA
:10923000A0E0B0E08093B4139093B513A093B6135D
:10924000B093B71380E693E10E94B03480918C0C08
:10925000811105C080918E0C882309F46DC0609146
:10926000E0117091E111072E000C880B990B0F94FF
:109270001A2620E030E048EC52E40F9479266B0186
:109280007C016091E2117091E311072E000C880BB4
:10929000990B0F941A269B01AC01C701B6010F94DC
:1092A000DD2D0F94562E6536710510F064E670E0E2
:1092B0007093BD136093BC1305E00093B01312E8E4
:1092C0001093B31384E290E1A0E0B0E08093B41374
:1092D0009093B513A093B613B093B71380E693E1C0
:1092E0000E94B0346091E0117091E111072E000CE2
:1092F000880B990B0F941A266B017C0120E030E05B
:109300004AE253E40F94432F181624F480918C0CF6
:10931000811146C16091E2117091E311072E000C9A
:10932000880B990B0F941A269B01AC01C701B6015B
:109330000F94432F87FFAFC18091820C882339F1AE
:109340008091810C91E0980F9093810C90E0909324
:10935000BD138093BC1385E08093B01382E88093A3
:10936000B31382E490E1A0E0B0E08093B413909353
:10937000B513A093B613B093B71380E693E10E94A0
:10938000B0348091810C8A3010F01092810C0E94D0
:109390003C2C882309F4B5C16091960C7091970C10
:1093A000EE24E394F12C61157105A9F090E080E0C2
:1093B0000F94182620E030E040E85EE30F94792611
:1093C0000F94C12D20E030E040E85FE30F94E32CE0
:1093D0000F94562E7B0101E010E080917C0C8111EE
:1093E00002C010E000E08091A4129091A5128F3F7E
:1093F000980711F40E94C4B39093A5128093A4120D
:10940000080F191FB80190E080E00F94182620E0A3
:1094100030E040E85EE30F9479260F94C12D4B01B4
:109420005C01F092BD13E092BC1305E00093B01311
:1094300012E81093B31380E193E1A0E0B0E08093D1
:10944000B4139093B513A093B613B093B71380E6FB
:1094500093E10E94B034C501B4010F94562E70936D
:10946000BD136093BC130093B0131093B31382E148
:1094700093E1A0E0B0E08093B4139093B513A09370
:10948000B613B093B71380E693E10E94B03400E0C6
:1094900014E1AAE1FA2E80913105909132052091D4
:1094A000730530917405891B8F7309F449C12A3102
:1094B00031050CF0DBC190913105809132054FEF01
:1094C0005FEF981749F0E82FF0E0EF5CFA4F428128
:1094D0008F5F8F7380933205F901E050FC4E40831B
:1094E000809100148A3509F0B3C162E070E080E039
:1094F00090E00E94B92C80917305909174050196BB
:109500009093740580937305C6CF1092BD1310928B
:10951000BC13ACCB6091E2117091E311072E000CEB
:10952000880B990B0F941A2620E030E0A9010F94C4
:109530001326811134C98CE090E09093BD13809381
:10954000BC1385E08093B01382E88093B31384E169
:1095500090E1A0E0B0E0F3CB8DE090E09093BD13FC
:109560008093BC1385E08093B01382E88093B3139B
:1095700084E190E1A0E0B0E08093B4139093B51340
:10958000A093B613B093B71380E693E10E94B03472
:109590008091930C811101C081E08093930CDBCB0F
:1095A00010928C0C20E030E040E251E46091840C99
:1095B0007091850C8091860C9091870C0F94792680
:1095C0000F944F2E7093BD136093BC130093B01390
:1095D0001093B31384E590E1A0E0B0E08093B4135E
:1095E0009093B513A093B613B093B71380E693E1AD
:1095F0000E94B03420E030E040E251E46091880CF9
:109600007091890C80918A0C90918B0C0F94792623
:109610000F944F2E7093BD136093BC130093B0133F
:109620001093B31388E590E1A0E0B0E08093B41309
:109630009093B513A093B613B093B71380E693E15C
:109640000E94B03480EA97E10E9460388AE00E946C
:10965000273881E09AE59093BD138093BC1381E491
:1096600090E09093BF138093BE1387E08093B01374
:109670001093B31384E890E0A0E0B0E08093B413BB
:109680009093B513A093B613B093B71380E693E10C
:109690000E94B03451CE60918E0C662309F44CCEFA
:1096A000062E000C770B87E897E10E945E418AE066
:1096B0000E94273810928E0C84E090E09093BD13A6
:1096C0008093BC1385E08093B01312E81093B3131A
:1096D0008EE890E1A0E0B0E08093B4139093B513CE
:1096E000A093B613B093B71380E693E10E94B03411
:1096F00081E09AE59093BD138093BC1383E590E0DD
:10970000B0CF1092BD131092BC1305E00093B013BC
:1097100012E81093B31380E193E1A0E0B0E08093EE
:10972000B4139093B513A093B613B093B71380E618
:1097300093E10E94B0341092BD131092BC1393CEEB
:10974000121613060CF492C0809164139091651365
:10975000A0916613B09167138C34E0E19E07A105D8
:10976000B10509F4D7C98A349041A105B10509F4BE
:10977000D1C920E030E040E251E460911C0C7091CE
:109780001D0C80911E0C90911F0C0F9479260F9444
:109790004F2E7093BD136093BC1305E00093B0137C
:1097A00012E81093B31388E490E1A0E0B0E0809356
:1097B000B4139093B513A093B613B093B71380E688
:1097C00093E10E94B03420E030E040E251E4609147
:1097D000200C7091210C8091220C9091230C0F94FD
:1097E00079260F944F2E7093BD136093BC13009392
:1097F000B0131093B3138AE490E1A0E0B0E080933B
:10980000B4139093B513A093B613B093B71380E637
:1098100093E10E94B03420E030E040E251E46091F6
:10982000240C7091250C8091260C9091270C0F949C
:1098300079260F944F2E7093BD136093BC13009341
:10984000B0131093B3138CE490E1A0E0B0E056C9DC
:10985000121613060CF01FCEF8012F2D11922A9527
:10986000E9F7109274051092730515CE909161136B
:1098700080910014981321C090916213809101147B
:1098800098131BC023303105C4F0909102149093BB
:10989000601380910314809363139330D1F4982F55
:1098A0009D7F9038B1F4909104149F3409F059C011
:1098B000909105149B3409F054C0E0E0F4E18AE192
:1098C000DF011D928A95E9F71092740510927305D5
:1098D0003BCF833809F045C0809104149091051462
:1098E000982789279827B0E0A0E08093641390938D
:1098F0006513A0936613B0936713C0900614D12C20
:10990000F12CE12CC0926813D0926913E0926A1393
:10991000F0926B1327E034E140E050E0BA014C15BF
:109920005D056E057F0508F04AC0DB01CA01B695EA
:10993000A795979587950696880F991FFC01E05A81
:10994000FC4ED9018C9111969C91892798278927E3
:10995000918380834E5F5F4F6F4F7F4F2E5F3F4FEE
:10996000DECF813861F58091041490E0B0E0A0E092
:109970008093641390936513A0936613B093671359
:1099800080910514482F50E070E060E04093681328
:109990005093691360936A1370936B13A6E0B4E15C
:1099A000ECE6F3E190E030E020E08217930739F035
:1099B0004D9150E0419351932F5F3F4FF6CFE0E040
:1099C000F4E18AE1DF011D928A95E9F710927405AE
:1099D000109273050E9422FEB7CE3F924F925F9283
:1099E0006F927F928F929F92AF92BF92CF92DF92AF
:1099F000EF92FF920F931F93CF93DF9380912D05EA
:109A000087FD38C080912E058370A1F5C091791231
:109A1000D0917A12488159816A817B8181E197E1F5
:109A20000E943C414C815D816E817F8184E69FE292
:109A30000E943C41409175125091761260917712CC
:109A40007091781281E69FE20E943C418AE0DF91AA
:109A5000CF911F910F91FF90EF90DF90CF90BF902B
:109A6000AF909F908F907F906F905F904F903F90BE
:109A70000C94273860906D1270906E1280906F1267
:109A800090907012A0907112B090721200917312A7
:109A900010917412C0907512D0907612E0907712E7
:109AA000F090781288E50E94BE1EC82F882309F422
:109AB0009AC00E94C424362E472E582ED92F20E05B
:109AC00030E041EE53EC0F94432F87FD0DC020E0B2
:109AD00030E041EE53E4632D742D852D9D2F0F94BE
:109AE000132618160CF081C062EC71E08EEF96E13F
:109AF0000E945E4162EC71E089EF96E10E945E4156
:109B000086EF96E10E946038C0E089E50E94BE1EA3
:109B1000882361F10E94C424362E472E582ED92F57
:109B200020E030E041EE53EC0F94432F87FD0DC051
:109B300020E030E041EE53E4632D742D852D9D2F00
:109B40000F94132618160CF055C062EC71E083EEEA
:109B500096E10E945E4162EC71E08EED96E10E941A
:109B60005E418BED96E10E946038C0E08AE50E947C
:109B7000BE1E882309F443C00E94C4246B017C01EB
:109B800020E030E040E151EC0F94432F87FD0AC004
:109B900020E030E040E151E4C701B6010F94132604
:109BA00018166CF567EF7FEF89EC96E10E945E4135
:109BB00069E070E084EC96E10E945E4181EC96E100
:109BC000DF91CF911F910F91FF90EF90DF90CF9099
:109BD000BF90AF909F908F907F906F905F904F90CD
:109BE0003F900C946038C1E090CF632C742C852C8E
:109BF0009D2E8BCFA32CB42C052D1D2FB7CFCC239E
:109C0000E1F0C301D40180936D1290936E12A09382
:109C10006F12B0937012C501D801809371129093A6
:109C20007212A0937312B0937412C0927512D092F4
:109C30007612E0927712F0927812DF91CF911F9115
:109C40000F91FF90EF90DF90CF90BF90AF909F90DB
:109C50008F907F906F905F904F903F9008958FED21
:109C600097E00C94603889ED97E00C94603884E6B6
:109C700090E09093B8058093B7051092D8051092A4
:109C8000D7050C94F5DBEF92FF920F931F93CF93C0
:109C9000DF93CDB7DEB762970FB6F894DEBF0FBE85
:109CA000CDBF0E943F2A882309F43FC04EED53E008
:109CB00082FF02C042EC53E02EED33E081FF02C090
:109CC00024EC33E080FD2EC08EED93E05F934F9344
:109CD0003F932F939F938F938BE399E19F938F9360
:109CE0008E010F5F1F4F1F930F930F94AA250E94A1
:109CF000334EC8010E942E38C8010E9492E40FB66C
:109D0000F894DEBF0FBECDBF81E062960FB6F89427
:109D1000DEBF0FBECDBFDF91CF911F910F91FF909E
:109D2000EF90089586EC93E0D1CF80E0EECFCF9214
:109D3000DF92EF92FF928AE50E94BE1E882309F40B
:109D40005AC00E94C42420E030E040E050EC0F9460
:109D50001326C12CD12CE12C90ECF92E87FD0FC0DD
:109D60000E94C42420E030E040E050E40F94432FF0
:109D700018160CF462C00E94C4246B017C0120916F
:109D80004A0C30914B0C40914C0C50914D0CC7013A
:109D9000B6010F9479260F944F2ECB010E94ABFD94
:109DA00080E50E94701E81114EC0A701960160914E
:109DB00075127091761280917712909178120F94AB
:109DC000E32C6093751270937612809377129093C0
:109DD00078120E94334E4091751250917612609124
:109DE00077127091781282EB96E10E943C418AE0F2
:109DF0000E94273805C083E50E94BE1E8111A1CFB5
:109E000080912D0587FD24C080912E05837001F57A
:109E10000E94334E409175125091761260917712E4
:109E20007091781283EA96E10E943C418AE0FF90AB
:109E3000EF90DF90CF900C942738C12CD12CE12CDF
:109E400080E4F82E9CCF0E948C248111AECFD8CF15
:109E500082E50E94701E8111DBCFFF90EF90DF90B2
:109E6000CF900895CF9384E50E94BE1EC0E0882362
:109E7000D9F00E946C24C82F1816B4F40E94334EF7
:109E80008DE40E94273880912805909129050E9431
:109E900046E26C2FCC0F770B88EA9FE00E945E4170
:109EA0008AE00E942738CFEF8C2FCF9108954F92F0
:109EB0005F926F927F928F929F92AF92BF92CF925A
:109EC000DF92EF92FF92CF93DF93CDB7DEB72C975F
:109ED0000FB6F894DEBF0FBECDBF4090C4085090BF
:109EE000C5086090C6087090C7082091470230915D
:109EF00048024091490250914A02C301B2010F94B5
:109F0000E32C69837A838B839C838090C80890902C
:109F1000C908A090CA08B090CB0820914B0230919C
:109F20004C0240914D0250914E02C501B4010F9474
:109F3000E32C6D837E838F839887C090CC08D0906C
:109F4000CD08E090CE08F090CF0820914F023091DC
:109F500050024091510250915202C701B6010F9434
:109F6000E32C69877A878B879C87209153023091F5
:109F700054024091550250915602C301B2010F9410
:109F8000E32C2B013C012091570230915802409163
:109F9000590250915A02C501B4010F94E32C4B01B0
:109FA0005C0120915B0230915C0240915D02509116
:109FB0005E02C701B6010F94E32C6B017C010E9485
:109FC000334E83EE9EE00E94603883E50E94701E4F
:109FD000882321F00E948C248093450280914502C1
:109FE000811151C08AEC9EE00E9460388BED9EE0AA
:109FF0000E94603849815A816B817C8189E09EE1B1
:10A000000E943C414D815E816F81788584E69FE2AC
:10A010000E943C4149855A856B857C8581E69FE29B
:10A020000E943C4189ED9EE00E94603881ED9EE0F7
:10A030000E946038B301A20189E09EE10E943C4188
:10A04000B501A40184E69FE20E943C41B701A6014C
:10A0500081E69FE20E943C418AE02C960FB6F8947C
:10A06000DEBF0FBECDBFDF91CF91FF90EF90DF90AD
:10A07000CF90BF90AF909F908F907F906F905F90A8
:10A080004F900C9427388EEC9EE0AECF5F926F928B
:10A090007F928F929F92AF92BF92CF92DF92EF9278
:10A0A000FF920F931F93CF93DF931F92CDB7DEB72D
:10A0B0007C0139018B015B01A40EB51ED12CC12C92
:10A0C000A016B10609F450C0F70180809180F80114
:10A0D00051908F015982C4010F94312C5816B9F157
:10A0E000652DC4010F94392CFFEFCF1ADF0AC6018A
:10A0F0008F779927892B21F162E070E080E090E072
:10A100000E943FFDC4010F94312C99818917F9F009
:10A110000E94334E8FE694E00E94603881E00F90F9
:10A12000DF91CF911F910F91FF90EF90DF90CF9033
:10A13000BF90AF909F908F907F906F905F900895A9
:10A1400062E070E080E090E00E943226DBCFBE014A
:10A150006F5F7F4FC3010E9416E1F70180819181FB
:10A16000019691838083ACCF80E0D9CFDF92EF92CC
:10A17000FF920F931F93CF93DF93CDB7DEB7CA5AE9
:10A18000D1090FB6F894DEBF0FBECDBFCF55DF4F5C
:10A19000188219821A821B82C15AD0408091C8034A
:10A1A0009091C903A091CA03B091CB03CB55DF4F67
:10A1B00088839983AA83BB83C55AD04084E690E004
:10A1C0009093B8058093B7051092D8051092D705E3
:10A1D0001092D90527ED35E044E050E0BE016B5503
:10A1E0007F4F87EB95E00E9446508091B705909194
:10A1F000B80502969093B8058093B7051092D805DC
:10A200001092D70581E0C655DF4F8883CA5AD040E7
:10A21000CE0186559F4F0E94DBD127ED35E048E403
:10A2200050E06EE27CE087EB95E00E94465027ED1F
:10A2300035E040E150E061ED78E087EB95E00E9489
:10A2400046508AE097EDA3EABCE3CF55DF4F888301
:10A250009983AA83BB83C15AD040CE018F559F4FAB
:10A260000E94D2D18AEF97E00E94EDD186E292E07F
:10A270000E94E4D182E292E00E94D2D18091C00893
:10A280009091C108A091C208B091C30889839A83B4
:10A29000AB83BC838E010F5F1F4FC8010E94D2D1D8
:10A2A000CF55DF4F188219821A821B82C15AD040C3
:10A2B0007E018DE6E80EF11C83E0D7018C93898343
:10A2C000CE018F559F4F0E94D2D1C7010E94DBD192
:10A2D000C8010E94DBD14AE0D42EDA94DD2031F0AF
:10A2E000CE018F559F4F0E94D2D1F7CF8DE692E1DC
:10A2F0000E94EDD1CF55DF4F188219821A821B823E
:10A30000C15AD0403AE0D32EDA94DD2031F0CE01AC
:10A310008F559F4F0E94D2D1F7CF85E0D82ED9829A
:10A32000F701D082C8010E94DBD1C7010E94DBD1B6
:10A3300027ED35E048E050E06AEC75E087EB95E00A
:10A340000E94465027ED35E048E050E062EC75E0B1
:10A3500087EB95E00E94465027ED35E044E650E05B
:10A3600064E877E087EB95E00E94465019828FEF12
:10A37000D7018C93C8010E94E4D1C7010E94DBD1B0
:10A3800027ED35E044E050E064EE72E087EB95E0C5
:10A390000E94465080919B068983C8010E94E4D1A7
:10A3A000198A1A8A1B8A1C8A80E090E0A0E8BFE321
:10A3B0008D879E87AF87B88B8091E5119091E611CC
:10A3C000A091E711B091E81189839A83AB83BC8394
:10A3D0002CEA35EC47E25EE36091E9117091EA11F5
:10A3E0008091EB119091EC110F94DD2D6D837E83A4
:10A3F0008F8398872CEA35EC47E25EE36091ED119C
:10A400007091EE118091EF119091F0110F947926D7
:10A4100069877A878B879C8727ED35E044E150E098
:10A42000B80187EB95E00E94465084E190E09A8362
:10A430008983C8010E94C0D180917A1190917B11CB
:10A44000A0917C11B0917D1189839A83AB83BC83E9
:10A450002CEA35EC47E25EE360917E1170917F114A
:10A4600080918011909181110F94DD2D6D837E83F9
:10A470008F8398872CEA35EC47E25EE36091821186
:10A480007091831180918411909185110F94792698
:10A4900069877A878B879C87C8010E94C9D18CE025
:10A4A000EBE7F2E0D80101900D928A95E1F7C8013F
:10A4B0000E94C9D11982C8010E94DBD18FE790E0C8
:10A4C0009A838983C8010E94C0D1E7E8F2E0D801ED
:10A4D00001900D92DA94E1F727ED35E045E050E088
:10A4E000B80187EB95E00E9446508091C1058983B1
:10A4F000C8010E94E4D180E2ECE8F2E0D8010190CA
:10A500000D928A95E1F727ED35E040E250E0B80181
:10A5100087EB95E00E944650F7011082C7010E9428
:10A52000E4D18DEE97E00E94E4D189EE97E00E949D
:10A53000D2D1CF55DF4F188219821A821B82C15A9D
:10A54000D040CE018F559F4F0E94D2D180E2D801DA
:10A550001D928A95E9F727ED35E040E250E0B80119
:10A5600087EB95E00E944650FE01F99688E0DF01F6
:10A570001D928A95E9F744E650E060E070E0498377
:10A580005A836B837C834D835E836F83788783E0FC
:10A5900090E0A0E0B0E089879A87AB87BC874D87C1
:10A5A0005E876F87788B498B5A8B6B8B7C8B8D8BFF
:10A5B0009E8BAF8BB88F898F9A8FAB8FBC8F8D8F0F
:10A5C0009E8FAF8FB8A38EE190E0A0E0B0E089A3AA
:10A5D0009AA3ABA3BCA38DA39EA3AFA3B8A789A73F
:10A5E0009AA7ABA7BCA78DA79EA7AFA7B8AB89AB0F
:10A5F0009AABABABBCAB8DAB9EABAFABB8AF27ED03
:10A6000035E040E450E0B80187EB95E00E94465009
:10A6100090E1D92EF8018D2D11928A95E9F727ED59
:10A6200035E040E150E0B80187EB95E00E944650EC
:10A63000D8011D92DA94E9F727ED35E040E150E0CA
:10A64000B80187EB95E00E944650CF55DF4F188246
:10A6500019821A821B82C15AD040CE018F559F4F5A
:10A660000E94D2D12CE0D22EF8018D2D11928A9524
:10A67000E9F727ED35E04CE050E0B80187EB95E0D5
:10A680000E9446508CE6D8011D928A95E9F727ED85
:10A6900035E04CE650E0B80187EB95E00E9446506B
:10A6A0008BEA95E00E94C9D127ED35E048E050E003
:10A6B00069EB75E087EB95E00E944650F701119237
:10A6C000DA94E9F7C755DF4F1882C95AD04080E0C5
:10A6D00090E0A0E4B0E4C356DF4F88839983AA8357
:10A6E000BB83CD59D040C7010E94EDD1CE01875523
:10A6F0009F4F0E94DBD1CE0183569F4F0E94D2D143
:10A7000080E3D7011D928A95E9F785E89CE10E94D4
:10A7100060388AE00E94273827ED35E040E350E0BA
:10A72000B70187EB95E00E9446508091D9058111D1
:10A7300028C00091B7051091B8058091D705909178
:10A74000D805F7019183808384E690E09093B80563
:10A750008093B70527ED35E044E050E068EE72E005
:10A7600087EB95E00E944650C7010E94C0D191E05E
:10A770000536134009F490E08091D905892B809328
:10A78000D9058091D905811105C060E089EB9CE174
:10A790000E94CE3F89E99CE10E9460388AE00E94D5
:10A7A00027389091D90581E08927C655DF4F0FB62C
:10A7B000F894DEBF0FBECDBFDF91CF911F910F91F7
:10A7C000FF90EF90DF900895CF93DF9300D01F921A
:10A7D000CDB7DEB7809187068823C1F083E390E090
:10A7E0009C838B831A8219829E012F5F3F4F40E129
:10A7F00050E068E876E0CE0103960E94465089E971
:10A800009CE10E9460388AE00E9427380F900F90E8
:10A810000F900F90DF91CF910895CF92DF92EF923A
:10A82000FF92CF93C82F809119118150823008F088
:10A8300069C00E94C33A109219110E9472FD609380
:10A84000A3057093A4058093A5059093A605C090D9
:10A85000A705D090A805E090A905F090AA050E9450
:10A86000A62BAB01BC014093A7055093A8056093AC
:10A87000A9057093AA0580918C0690918D06A091F0
:10A880008E06B0918F068C199D09AE09BF09840F01
:10A89000951FA61FB71F80938C0690938D06A093DB
:10A8A0008E06B0938F06C1110AC0C1E00E94E45326
:10A8B0008C2FCF91FF90EF90DF90CF9008958091F3
:10A8C0008A0690918B06019690938B0680938A0658
:10A8D0000E94A62BC0909006D0909106E090920620
:10A8E000F0909306C616D706E806F906F0F60E9421
:10A8F000A62B609390067093910680939206909396
:10A900009306D3CFC0E0D2CF81E00C940D540E94C7
:10A91000E2BE0E94845480E00E9441F98091DD06ED
:10A920008130A1F40E942F4E82E697E00E946038A9
:10A9300060E088E597E00E94CE3F6EE571E080E040
:10A9400090E00E94322688E08093DD060895CF9241
:10A95000DF92EF92FF921F93CF93DF9300D01F926D
:10A96000CDB7DEB78EEEC82E82E0D82EE12CF12CCA
:10A97000C982DA82EB82FC82BE016F5F7F4F8AE57B
:10A980000E94923381110EC010E0812F0F900F9022
:10A990000F900F90DF91CF911F91FF90EF90DF907C
:10A9A000CF9008950E94E833C982DA82EB82FC825C
:10A9B000BE016F5F7F4F8AE50E949233182F882374
:10A9C00019F30E942F4E8CE398E00E9460380E9499
:10A9D0008754DBCFCF92DF92EF92FF921F93CF93FA
:10A9E000DF9300D01F92CDB7DEB78EEEC82E82E087
:10A9F000D82EE12CF12CC982DA82EB82FC82BE01D6
:10AA00006F5F7F4F8AE00E94923381110EC010E089
:10AA1000812F0F900F900F900F90DF91CF911F918A
:10AA2000FF90EF90DF90CF9008950E94E8330E944E
:10AA3000B2330E94CD330E94B233C982DA82EB82F4
:10AA4000FC82BE016F5F7F4F8AE00E949233182F15
:10AA50008823E9F20E942F4E8FEF97E00E94603822
:10AA60000E948754D5CFCF93DF9300D01F921F92BF
:10AA7000CDB7DEB781E08093870680E1E8E8F6E0B5
:10AA8000DF011D928A95E9F70E94E45386E18D83E8
:10AA900082E390E09C838B831A8219829E012F5F50
:10AAA0003F4F41E050E0BE016B5F7F4FCE01039608
:10AAB0000E9446500F900F900F900F900F90DF91D3
:10AAC000CF910895CF93DF93CDB7DEB7A8970FB698
:10AAD000F894DEBF0FBECDBF8C01F42E0E94E2BE03
:10AAE0000E942F4E88E397E00E94603801151105FF
:10AAF00011F40FE217E080917D0580FD79C081603F
:10AB000080937D058BE197E00E9460388AE00E9487
:10AB10002738CC24C3948AE5D82ED092BD13C09296
:10AB2000BC138FE090E09093BF138093BE1397E027
:10AB3000792E7092B01322E8E22EE092B31334E83B
:10AB4000832E912CA12CB12C8092B4139092B5132A
:10AB5000A092B613B092B71380E693E10E94B0348E
:10AB6000D092BD13C092BC1388E590E09093BF13C0
:10AB70008093BE137092B013E092B3138092B4131B
:10AB80009092B513A092B613B092B71380E693E1FA
:10AB90000E94B0348AE289838A838B838C83F80194
:10ABA000DE011596BE016F5F7F4FCD01861B970BAF
:10ABB0002491319621110CC0FB01E80FF91F8AE2A4
:10ABC0009F01261B370B2832310524F48193F8CFDF
:10ABD0002D93EBCF20E630E140E050E080E693E1BA
:10ABE0000E9431E16AE070E080E090E00E94B92CC0
:10ABF00061E086E297E00E949B3F89EE93E030E6B9
:10AC0000019729F0232F2A950000E9F7F9CFF8944E
:10AC100089EE93E038EE019729F0232F2A95000062
:10AC2000E9F7F9CF0E94E2BEFF2031F00E942A1F0F
:10AC30000E94431FA895FECF0E94281FF9CF809144
:10AC4000DC06882319F01092DC06089540E070E0DD
:10AC500060E08CEA98E10E9462558091990C909195
:10AC60009A0C2FEF3FEF981751F0E92FF0E0E756DD
:10AC7000F34F228130E09F5F9F7790939A0CC90138
:10AC800008951F920F920FB60F9211240F900FBECE
:10AC90000F901F9018951F920F920FB60F921124CC
:10ACA0000BB60F920F931F932F933F934F935F9386
:10ACB0006F937F938F939F93AF93BF93CF93DF93C4
:10ACC000EF93FF93C091C60000919A0CD091990C1C
:10ACD00011E01D0F1F7790910B04913108F09FC078
:10ACE000E92FF0E08827E858F94A8F4F0D94DA2CC5
:10ACF0008956B856C756D656DD560F57E1560F57E8
:10AD0000E556E9560F57ED56F156F556FC560F57D6
:10AD10000757C03229F028F5CA3011F0CD3031F58F
:10AD2000011731F0ED2FF0E0E756F34FC283D12F3A
:10AD3000D093990CFF91EF91DF91CF91BF91AF919B
:10AD40009F918F917F916F915F914F913F912F9143
:10AD50001F910F910F900BBE0F900FBE0F901F9081
:10AD60001895CD3481F081E0CE3471F080E10CC0D3
:10AD7000CA3338F4C033A0F6C03291F2CD32B1F705
:10AD8000CFCFCD3499F782E080930B04C9CFC13384
:10AD900059F018F4C03221F2E9CF88E0C433A1F3AE
:10ADA0008BE0C83389F3E2CF83E0EECF84E0C03399
:10ADB00059F386E0C13341F3D9CF85E0C833B1F60A
:10ADC000E3CF87E0C23391F6DFCF89E0C13371F67C
:10ADD000DBCF8AE0C03351F6D7CF8CE0C73331F6F2
:10ADE000D3CF8DE0C63311F6CFCFC03209F498CF60
:10ADF0008EE0C33549F2BACF80ED8C0F8A3008F06F
:10AE00008FCF9FE090930B0480930C0489CFCA30BE
:10AE100019F0CD3009F084CF10920B0481CFCA30E5
:10AE200019F0CD3009F07CCF80911A148823A1F35A
:10AE3000973089F038F4953079F710923C021092EF
:10AE40001B0CEACF9A3059F09F3031F780910C04F7
:10AE50000E94CF31E1CF81E080930506DDCF81E014
:10AE600080930406D9CF8EBD0DB407FEFDCF0895A3
:10AE70008FEF8EBD0DB407FEFDCF8EB50895909176
:10AE800064009B7F90936400982F906A96959CBD78
:10AE900080FD03C091E0863009F490E09DBD0895E7
:10AEA000CF93DF93EB010E946038CE01DF91CF9109
:10AEB0000C942CAF2F923F924F925F926F927F92A1
:10AEC0008F929F92AF92BF92CF92DF92EF92FF92BA
:10AED0000F931F93CF93DF93009709F0AAC11092AD
:10AEE0007E0C10927D0C90937C0580937B05BAE0DC
:10AEF000CB2EB0E2DB2EE12CF12C15E002E846016E
:10AF00005701C4E1D0E01092031310920213109382
:10AF1000F6120093F9128092FA129092FB12A0920C
:10AF2000FC12B092FD1286EA92E10E94B0342197A1
:10AF30002FEF821A920AA20AB20A209721F744E15F
:10AF4000C40ED11CE11CF11C8AE5C81680E2D806AB
:10AF5000E104F104A1F6C12CA0E2DA2EE12CF12CDF
:10AF6000D5E0C2E81092031310920213D093F612A8
:10AF7000C093F912C092FA12D092FB12E092FC1226
:10AF8000F092FD1286EA92E10E94B034109203130F
:10AF900010920213D093F612C093F912D701C60192
:10AFA0008C529F4FAF4FBF4F8093FA129093FB127A
:10AFB000A093FC12B093FD1286EA92E10E94B03495
:10AFC000EFEFCE1ADE0AEE0AFE0AFAE0CF16F0E242
:10AFD000DF06E104F10431F6FEEDCF2EF0E2DF2EC4
:10AFE000E12CF12CD5E0C2E8109203131092021369
:10AFF000D093F612C093F912C092FA12D092FB12BB
:10B00000E092FC12F092FD1286EA92E10E94B034C6
:10B010002FEFC21AD20AE20AF20A46EEC41640E242
:10B02000D406E104F10401F7CC24C394E2E1DE2E5E
:10B03000E12CF12C0AE010E0D5E0C2E810930313F4
:10B0400000930213D093F612C093F912C092FA1231
:10B05000D092FB12E092FC12F092FD1286EA92E18D
:10B060000E94B0341093031300930213D093F6128E
:10B07000C093F912D701C6018096A11DB11D80931E
:10B08000FA129093FB12A093FC12B093FD1286EA81
:10B0900092E10E94B0348FEFC81AD80AE80AF80A81
:10B0A000E5E0CE16E2E1DE06E104F10439F60091B6
:10B0B0007D0C10917E0C0115110509F0D6C0809110
:10B0C0007C0C882309F4E1C02AE030E240E050E043
:10B0D0006CEC73E086EA92E10E9431E1C1E0D0E0DD
:10B0E00003E010E0E0907D0CF0907E0C35E0332E14
:10B0F00042E8242E44244A94542C64E0662E712C99
:10B100007FE1C72E74E0D72E80917D0C90917E0C4C
:10B11000800F911FE816F90608F0D5C0C7010E94FC
:10B120004CE2882309F481C08091941167E871E1B1
:10B13000882311F064E971E1FB0101900020E9F737
:10B14000CF010197861B970BF4E1FC9F9001FD9FB7
:10B15000300D1124265F3F4D50E040E0459710F040
:10B16000FB01128A86EA92E10E9431E1CE018F5FF3
:10B170009D4EB0E0A0E021964E0124E0880C991C81
:10B180002A95E1F7FDEF8F1AFFE99F0AB12CA12C58
:10B190002091261424FF7EC0709203136092021344
:10B1A0003092F6122092F9128093FA129093FB12C9
:10B1B000A093FC12B093FD1286EA92E10E94B03493
:10B1C000D0920313C09202133092F6122092F91219
:10B1D0008092FA129092FB12A092FC12B092FD1291
:10B1E00086EA92E10E94B034B70181E498E10E94BE
:10B1F0002A418091941164E971E1811102C067E8EC
:10B2000071E18EE398E10E9450576BED7BE08AE399
:10B2100098E10E94505767E871E189E398E10E9444
:10B22000505785E398E10E9460382FEFE21AF20A46
:10B230006BCF20917D0C30917E0CA90141505109BA
:10B2400060917B0570917C056817790738F42C5F55
:10B250003F4F30937E0C20937D0C45CE44305105FA
:10B2600008F43DCE24503109F4CF0430110569F4BF
:10B2700080917C0C882331F083E090E090937E0CE9
:10B2800080937D0CD0E0C0E02DCFD0E0C0E004E0A2
:10B2900010E028CF10920313109202133092F6128E
:10B2A0002092F9128093FA129093FB12A093FC1251
:10B2B000B093FD1286EA92E10E94B03450920313DB
:10B2C0004092021381CFDF91CF911F910F91FF9098
:10B2D000EF90DF90CF90BF90AF909F908F907F9036
:10B2E0006F905F904F903F902F900895AF92BF92D4
:10B2F000CF92DF92EF92FF920F931F93CF93DF9342
:10B30000CDB7DEB7E6970FB6F894DEBF0FBECDBF60
:10B3100000912F0510913005F80101900020E9F708
:10B3200031976F01C01AD10AF801CF01801B910B30
:10B330008C159D053CF481918F32B9F7DF0111978F
:10B340001C92F3CF8BE1E6E4F4E1DE015C96019020
:10B350000D928A95E1F7F12CE12CEC14FD040CF030
:10B360005DC0F801EE0DFF1D8081811103C08FEFDC
:10B37000E81AF80A5801AE0CBF1CF5018081882339
:10B3800009F44CC0FFEFEF1AFF0AF801EE0DFF1DA4
:10B390007F01E01AF10A81918111FACFCE014C961A
:10B3A0000E94BFB38BE1FE017C96DE0111960190F5
:10B3B0000D928A95E1F7B501CE0101960E94CDABC1
:10B3C000CE0101960E94BC2F8FE20E942738809107
:10B3D000941181113BC089ED93E00E942CAF8091C4
:10B3E000261484FF1BC019821C8221E0A501BE0126
:10B3F000645E7F4FCE0101960E9401B6811129C083
:10B400008AE00E9427380E94334EB50180E297E11E
:10B410000E945057CE0101960E94BC2F8AE00E94E4
:10B420002738CE014C960E94BC2FE6960FB6F894B2
:10B43000DEBF0FBECDBFDF91CF911F910F91FF9067
:10B44000EF90DF90CF90BF90AF90089584E991E1A5
:10B45000C4CFCE014C960E942EB38BE1FE013196F3
:10B46000DE015C9601900D928A95E1F7CE0101967E
:10B470000E94BC2F72CF2F923F924F925F926F9299
:10B480007F928F929F92AF92BF92CF92DF92EF9274
:10B49000FF920F931F93CF93DF9300D000D000D083
:10B4A0001F921F92CDB7DEB7B82E8091860D8430E3
:10B4B00008F0D1C10E9472FD6B017C018091860D64
:10B4C000811108C08091990C90919A0C891B8F77FB
:10B4D00009F4A4C681E6A82E13C08A3019F08D3075
:10B4E00009F0F6C01092810D80911F0D9091200DF2
:10B4F000FC01E55EF24F1682892BF1F40E942FC207
:10B500008091860D843008F0ECC08091990C909168
:10B510009A0C891B8F7709F4E4C00E942D5697FF7F
:10B52000DCCF0E942F4E85EB95E00E946038809121
:10B53000990C80939A0CE4CF1092200D10921F0D5D
:10B5400001E21DE0F8018191803209F446C08E3499
:10B5500009F0A9C060EB75E0C8010F9490254C017B
:10B56000892B41F06EE470E0C80104960F943130ED
:10B57000009709F4C8014AE050E070E060E00196ED
:10B580000F9400232B013C0180911B0D90911C0D09
:10B59000A0911D0DB0911E0D0196A11DB11D481663
:10B5A00059066A067B0629F060E08DE795E0892858
:10B5B00051F16AE270E0C8010F9460309C0100977D
:10B5C00029F1982F901B912C992349F09150F80163
:10B5D000E90FF11D80819826F7CF8F01B3CF4AE0A4
:10B5E00050E070E060E0C90101960F940023292D1E
:10B5F00030E050E040E0621773078407950751F090
:10B6000060E08EE595E00E94C7E77ACF60E084E3D2
:10B6100095E0F9CF40921B0D50921C0D60921D0DCC
:10B6200070921E0D8091DD068130E1F067E470E0DC
:10B63000C8010F9431300097A9F04AE050E070E063
:10B6400060E001960F940023643071058105910537
:10B6500048F483E994E00E94603860E089E894E06F
:10B660000E94CE3FC0927C07D0927D07E0927E0779
:10B67000F0927F078091210D8B3309F441CF8091A7
:10B68000860D843008F03CCF8091880D8A9DC001E2
:10B69000112461E27DE08757924F0F943C3080E0A7
:10B6A0000E9481E72DCF8091261480FFBBCF67E8F1
:10B6B0007DE2C8010F949025009731F0FC01838151
:10B6C00080538A3008F0AECF60E08AE095E09BCFEF
:10B6D0002FE13DE041E25DE061E87DE00E943E1D3A
:10B6E0000FCF8091261482FFB6C01A82198271E6AC
:10B6F000F72EE0E1EE2EF9E6DF2E8091860D843004
:10B7000008F0A9C00E94761D8111A5C041E050E05B
:10B71000BE016B5F7F4F8AE895E10E9481B10D8188
:10B7200010E0019711F00FEF1FEF809192159091AB
:10B730009315A0919415B091951580932214909330
:10B740002314A0932414B09325140E94761D0F3F58
:10B75000100749F4811107C00E942F4E83ED95E038
:10B760000E946038CACF4091880D242F30E00A3003
:10B7700061F00D3051F0882309F45FC089819A810E
:10B78000009719F001969A83898310929204898117
:10B790009A81F29EF001F39EF00D1124EA57F24FC8
:10B7A000E80FF91F1382892B69F50E942FC20E94AE
:10B7B000761D882309F4A1CF0E94A5618AE895E14E
:10B7C0000E942EB380911D14882391F181508093A3
:10B7D0001D148D9DC001112462E08B5E994F0E9463
:10B7E00083B8E0911D1424E0E29FF0011124EF5E84
:10B7F000F94F60817181828193810E948F220E9422
:10B8000036AB7BCF1A82198281E00E9481E780915A
:10B81000221490912314A0912414B09125148093A4
:10B82000820D9093830DA093840DB093850DBFCFAF
:10B830000E9437B3E092DD0660CF4F9DA001112436
:10B840004757524F9E012F5F3F4F62E974E0802FB0
:10B850000E943E1D52CF0E9472FD6B017C01B1100F
:10B8600004C080911811882351F0C0926B11D092BE
:10B870006C11E0926D11F0926E11BB24B394809123
:10B88000070590910805A0910905B0910A05009758
:10B89000A105B105B1F040916B1150916C1160910F
:10B8A0006D1170916E11840F951FA61FB71FA70110
:10B8B0009601281B390B4A0B5B0BDA01C901B7FF54
:10B8C00092C18091130290911402A0911502B0913F
:10B8D0001602892B8A2B8B2B09F099C10E9472FDCD
:10B8E0004B015C0180911B0C811108C020917E12DC
:10B8F00090917F1281E0291301C080E02091E01136
:10B900003091E11191E089272A3A31050CF480E069
:10B9100091E040919704509198046091990470913E
:10B920009A04452B462B472B09F490E0981789F091
:10B93000882309F4BDC1D501C40180569444A24FA7
:10B94000BF4F8093970490939804A0939904B09369
:10B950009A044090280C5090290C60902A0C70900A
:10B960002B0C2091930430919404409195045091B4
:10B970009604C301B2010F941326882319F1809114
:10B98000970490919804A0919904B0919A044092E0
:10B990009304509294046092950470929604892BBB
:10B9A0008A2B8B2B09F449C0D501C40180569444DD
:10B9B000A24FBF4F8093970490939804A09399044B
:10B9C000B0939A048091970490919804A09199045F
:10B9D000B0919A040097A105B10579F1881A990AE6
:10B9E000AA0ABB0AB7FC29C01092970410929804C7
:10B9F0001092990410929A0483E396E00E946038B2
:10BA000060E08FE196E00E94CE3F8091E21190913C
:10BA1000E3111816190624F490E080E00E94461FF6
:10BA200080917711909178111816190634F41092BC
:10BA30007811109277110E94B5BE80919F04909169
:10BA4000A004A091A104B091A20446015701881A54
:10BA5000990AAA0ABB0AD501C401B7FDB9C1209150
:10BA60007E1290917F1240912D0280912C02291319
:10BA700023C19091F508899FC0011124880F892F57
:10BA8000881F990B91958D838091F608489FC0017E
:10BA90001124880F892F881F990B91958E830E94FE
:10BAA00072FD69837A838B839C8340E0BE016F5F64
:10BAB0007F4FCE0105960E94901C6D8170E089E059
:10BAC0000E9469FC41E0BE016F5F7F4FCE01059689
:10BAD0000E94901C6E8170E087E00E9469FC80915A
:10BAE0001006882309F467C10091200210912102F9
:10BAF000C80102972091E2113091E311281739070C
:10BB00000CF459C180907F128F82188619861A868C
:10BB10001B8680917E129F80891509F4E7C0892DCC
:10BB200090E03CE5A32EA89EF001A99EF00D112403
:10BB3000E650F74F458956896789708D452B462B0E
:10BB4000472B81F4418D528D638D748D452B462B8F
:10BB5000472B41F4458D568D678D70A1452B462BA3
:10BB6000472BE1F12CE5B22EB89E9001B99E300D25
:10BB70001124A9014650574F1A01FA0161817281BF
:10BB8000838194810F94912F4B015C01F10161A19C
:10BB900072A183A194A10F9418262B013C01F101FD
:10BBA00065A176A187A190A50F9418269B01AC01F1
:10BBB000C301B2010F94DD2DA50194010F947926E4
:10BBC0004B015C01288539854A855B850F94432F9D
:10BBD000181624F488869986AA86BB868F818F5F83
:10BBE00087708F8396CF0E942F4E60917A07709155
:10BBF0007B0782EE95E00E9450578AE00E9427382A
:10BC000040E070E060E090E080E00E94625590913A
:10BC10007E1280917F12981749F0C0926B11D092DA
:10BC20006C11E0926D11F0926E1158CEBB2019F09C
:10BC30001092A30453CE0E9472FD00916B111091DB
:10BC40006C1120916D1130916E11809013029090C3
:10BC50001402A0901502B0901602080D191D2A1D9D
:10BC60003B1D601B710B820B930B97FDE1CF809105
:10BC7000A304811133CE81E08093A3045F9A809165
:10BC80002C0C8E7F80932C0C8A9A80912C0C8D7FAB
:10BC900080932C0C8091080180958170809306011F
:10BCA00080912C0C8B7F80932C0C0E94281F16CE29
:10BCB00080E090E0DC0145CE20917F125CE5259F7D
:10BCC000900111242650374FF901EA5AFF4F908115
:10BCD000899FC0011124880F892F881F990B919586
:10BCE0008D83295A3F4FF9018081D0CE20911A02CD
:10BCF00030911B0240911C0250911D02688579858C
:10BD00008A859B850F9479264B015C01B801012E31
:10BD1000000C880B990B0F941A269B01AC01C501EE
:10BD2000B4010F94E32C69837A838B839C834091C5
:10BD30001E0250911F02B801CE0101960E94EDC172
:10BD400089809A80AB80BC8040909B0450909C047A
:10BD500060909D0470909E04A3019201C501B401FE
:10BD60000F94132687FF16C028E431EE4AE75FE3FD
:10BD7000C301B2010F94792620E037ED43EA5CE37A
:10BD80000F94E32CA50194010F94792669837A839B
:10BD90008B839C8369817A818B819C8160939B04D6
:10BDA00070939C0480939D0490939E040F944F2E57
:10BDB000CB010E94461FF4E6CF0ED11CE11CF11C02
:10BDC000C0929F04D092A004E092A104F092A20439
:10BDD0000E942FC28091DD06882309F4E0C1809182
:10BDE0002602882309F4A3C08091E10481119FC039
:10BDF00080911811811108C080911911813021F0B2
:10BE00008091261482FF93C0F894649B10C08091A7
:10BE1000220290912302A0912402B09125028093E6
:10BE2000DE059093DF05A093E005B093E1056091F6
:10BE3000DE057091DF058091E0059091E105789431
:10BE400020E030E0A9010F94132687FF70C001E0C5
:10BE50000093E10480911811811167C088E496E095
:10BE60000E9460388AE00E94273884E08093930C17
:10BE700082E080937F0C81E09AE59093BD138093DC
:10BE8000BC138EE490E09093BF138093BE1387E0C1
:10BE90008093B01382E88093B31384E890E0A0E02D
:10BEA000B0E08093B4139093B513A093B613B093FE
:10BEB000B71380E693E10E94B0340E944B40009398
:10BEC000861140E36CE876E084E799E00E945040F8
:10BED00061E088E699E00E94324010910B0560E035
:10BEE00010278CE399E069F48AE796E00E949B3F73
:10BEF00080E30E9427388AE00E94273860E08DE5C1
:10BF000096E00E949B3F88E696E00E94603880E3BE
:10BF10000E9427388AE00E942738112331F083E6F7
:10BF200096E090937B0C80937A0C0E94A56190918F
:10BF30000901892F80958170109100021817C9F0AE
:10BF4000209126142062209326148093000290FDF5
:10BF50003FC164EF71E080E090E00E9432260E94D1
:10BF600059B38091261483FD7CC1111133C10E9405
:10BF7000F5350E9472FD6B017C01109117021123AF
:10BF8000F1F080910C058823D1F04091A4045091E8
:10BF9000A5046091A6047091A70446015701841A74
:10BFA000950AA60AB70AB501A40177FD1AC0833025
:10BFB00009F42FC10CF01EC181300CF023C1212FD8
:10BFC00030E0A8EEB3E00F94AB2CC60ED71EE81EEF
:10BFD000F91EC092A404D092A504E092A604F092A7
:10BFE000A70480911911813009F073C00E9472FD7D
:10BFF0006B017C018091AC049091AD04A091AE04E2
:10C00000B091AF04A7019601281B390B4A0B5B0BBB
:10C01000DA01C901B7FD3AC0D701C601805F984D6A
:10C02000AF4FBF4F8093AC049093AD04A093AE0488
:10C03000B093AF048090A7059090A805A090A905A3
:10C04000B090AA050E94A62BAB01BC014093A705A6
:10C050005093A8056093A9057093AA0580918C065A
:10C0600090918D06A0918E06B0918F06881999093E
:10C07000AA09BB09840F951FA61FB71F80938C06C2
:10C0800090938D06A0938E06B0938F068091A8049E
:10C090009091A904A091AA04B091AB044601570164
:10C0A000881A990AAA0ABB0AD501C401B7FD11C0B2
:10C0B00020E8C20E2EEED21E26E3E21EF11CC09234
:10C0C000A804D092A904E092AA04F092AB040E94C2
:10C0D000E4530E949E390E9468418091060588239E
:10C0E00079F10E9472FD6B017C01809102059091B3
:10C0F0000305A0910405B091050546015701881A72
:10C10000990AAA0ABB0AD501C401B7FD19C020913A
:10C11000060530E0A8EEB3E00F94AB2CC60ED71E98
:10C12000E81EF91EC0920205D0920305E0920405B4
:10C13000F092050580E00E9413BB8AE00E94273838
:10C1400080910105882359F10E9472FD6B017C01E9
:10C150008091FD049091FE04A091FF04B091000530
:10C16000A7019601281B390B4A0B5B0BDA01C901A9
:10C17000B7FD15C02091010530E0A8EEB3E00F94A3
:10C18000AB2CC60ED71EE81EF91EC092FD04D0923D
:10C19000FE04E092FF04F09200050E94F4AA2B96A0
:10C1A0000FB6F894DEBF0FBECDBFDF91CF911F91C8
:10C1B0000F91FF90EF90DF90CF90BF90AF909F9046
:10C1C0008F907F906F905F904F903F902F90089549
:10C1D0000E9448B3123008F0CCCE0E94F53560E0E2
:10C1E00085EC96E056C083ED96E090937B0C8093AF
:10C1F0007A0CBFCE843009F0E2CE0E94334E8AED35
:10C2000096E004C00E94334E89E097E00E946038B7
:10C21000D6CE0E94334E82EF96E0F8CF80917C0715
:10C2200090917D07A0917E07B0917F07A7019601AD
:10C23000281B390B4A0B5B0BDA01C901885E93405E
:10C24000A109B109B7FD46C98DEC95E00E9460389F
:10C25000C0927C07D0927D07E0927E07F0927F0724
:10C2600039C91230C8F48DE996E00E9460388AE03E
:10C270000E9427380E94D42C90E080E00E945A57F8
:10C280001092970C1092960C1092950C60E086EB31
:10C2900096E00E94CE3F6DCE123009F06ACE0E9429
:10C2A000B3B7882379F081E00E9489B742EB50E070
:10C2B00066E078E08BE294E10E9481B18BE294E148
:10C2C0000E942EB30E94AA2F81118DCF0E94942F1D
:10C2D0000E942FB80E9484B74CCECF93DF938091F9
:10C2E0007E1290917F12891B8095877019F40E94AD
:10C2F0003B5AF5CF80917E128F5F8770A0917E129E
:10C300009CE5A99FD0011124FD01E650F74FEF01F4
:10C3100019929A95E9F798E09083A15FB64F90E162
:10C32000E0E8F2E101900D929A95E1F720917E12FA
:10C3300090917F12291303C094E690937B1280930F
:10C340007E12DF91CF910C94C22F90917E1280913A
:10C350007F12981306C08091F8089091F908892BF4
:10C3600021F080E00E943B5AF0CF0895FC0120812B
:10C3700031814281538160914E0C70914F0C8091BC
:10C38000500C9091510C0F9479260F94502F60937C
:10C390008C1270938D1280938E1290938F129091C5
:10C3A0007E1280917F1298130C946D610E94A5619A
:10C3B0000E94322A40918C1250918D1260918E12FF
:10C3C00070918F124093000650930106609302060D
:10C3D0007093030681110C94C22F08954F925F92BF
:10C3E0006F927F928F929F92AF92BF92CF92DF9285
:10C3F000EF92FF920F931F93CF93DF93EC018B018A
:10C400005A01F90120914E0C30914F0C4091500C83
:10C410005091510C60817181828193810F947926B2
:10C420000F94502F6B017C0120914A0C30914B0CE2
:10C4300040914C0C50914D0CF501608171818281CD
:10C4400093810F9479260F94502F4B015C0120911A
:10C45000460C3091470C4091480C5091490CF80122
:10C4600060817181828193810F9479260F94502F7E
:10C470002B013C012091420C3091430C4091440C23
:10C480005091450C688179818A819B810F9479262E
:10C490000F94502F609380127093811280938212B8
:10C4A0009093831240928412509285126092861269
:10C4B000709287128092881290928912A0928A12AA
:10C4C000B0928B12C0928C12D0928D12E0928E128A
:10C4D000F0928F1290917E1280917F12981791F0B6
:10C4E000DF91CF911F910F91FF90EF90DF90CF9050
:10C4F000BF90AF909F908F907F906F905F904F9084
:10C500000C946D610E94A5610E94322A40918812AC
:10C510005091891260918A1270918B12009184124D
:10C52000109185122091861230918712C09080124E
:10C53000D0908112E0908212F0908312C092F405A4
:10C54000D092F505E092F605F092F7050093F80514
:10C550001093F9052093FA053093FB054093FC05F1
:10C560005093FD056093FE057093FF0540918C127A
:10C5700050918D1260918E1270918F12409300062F
:10C58000509301066093020670930306882391F08E
:10C59000DF91CF911F910F91FF90EF90DF90CF909F
:10C5A000BF90AF909F908F907F906F905F904F90D3
:10C5B0000C94C22FDF91CF911F910F91FF90EF90BC
:10C5C000DF90CF90BF90AF909F908F907F906F90B3
:10C5D0005F904F9008953F924F925F926F927F923B
:10C5E0008F929F92AF92BF92CF92DF92EF92FF9283
:10C5F0000F931F93CF93DF93CDB7DEB768970FB636
:10C60000F894DEBF0FBECDBFD82E2A013B014801F2
:10C6100059013E2C20E030E0A901C501B8010F947A
:10C620001326811110C081E08D1508F0B6C060E0BE
:10C6300070E080E793E420E030E040E752E40F94BC
:10C64000DD2D4B015C018D8A9E8AAF8AB88E0D2D3F
:10C6500010E0F801EA56F64EE491BB24B3941E169E
:10C660000CF4B12CCC24C39420E030E0A901C30128
:10C67000B2010F94432F18160CF0C12CBC1471F0AA
:10C6800092E0D9120BC0332049F081E00E9441F9B9
:10C6900069E170E080E090E00E94322680E00E9434
:10C6A000C82F69837A838B839C8381E00E94C82F83
:10C6B0006D837E838F83988782E00E94C82F69876D
:10C6C0007A878B879C8783E00E94C82F6D877E873F
:10C6D0008F87988B000F111F000F111FE1E0F0E012
:10C6E000EC0FFD1F0E0F1F1FF80110821182128226
:10C6F00013829E01235F3F4FAE01475F5F4FBE0134
:10C700006B5F7F4FCE0101960E94EE61F80140827F
:10C71000518262827382198A1A8A1B8A1C8A8091CA
:10C72000F8089091F908892B91F4CE0141967C018B
:10C730008E010B5E1F4F9E01235F3F4FAE01475F8F
:10C740005F4FBE016B5F7F4F40970E94EBE70E94F7
:10C75000A561BC1451F092E0D91205C0332019F044
:10C7600080E00E9441F90E941F5668960FB6F89427
:10C77000DEBF0FBECDBFDF91CF911F910F91FF9014
:10C78000EF90DF90CF90BF90AF909F908F907F9071
:10C790006F905F904F903F90089560E070E88BE35A
:10C7A00095E449CF4F925F926F927F928F929F92C2
:10C7B000AF92BF92CF92DF92EF92FF920F931F93AF
:10C7C000CF93DF93CDB7DEB72C970FB6F894DEBFCB
:10C7D0000FBECDBF2B013C0129873A874B875C8771
:10C7E00047015801F601E080F1800281138120E0C9
:10C7F00030E0A901B701C8010F941326882309F47A
:10C8000088C05E2D4F2D302F212F852F942FA32FE1
:10C81000B22F89839A83AB83BC8320E030E0A901E7
:10C82000B701C8010F941326811108C0E0903D02A2
:10C83000F0903E0200913F0210914002C701D801E2
:10C840008D839E83AF83B887A50194016091240CEA
:10C850007091250C8091260C9091270C0F94132633
:10C8600087FF0CC08092240C9092250CA092260C7D
:10C87000B092270CCE0101960E940D2B40921C0C09
:10C8800050921D0C60921E0C70921F0C89859A8527
:10C89000AB85BC858093200C9093210CA093220C37
:10C8A000B093230CCE0105960E940D2BA501940197
:10C8B0006091240C7091250C8091260C9091270C8E
:10C8C0000F94432F181664F48092240C9092250C38
:10C8D000A092260CB092270CCE0101960E940D2B3F
:10C8E0000E94A5612C960FB6F894DEBF0FBECDBF97
:10C8F000DF91CF911F910F91FF90EF90DF90CF903C
:10C90000BF90AF909F908F907F906F905F904F906F
:10C91000089550E040E030E820E477CFCF92DF92F6
:10C92000EF92FF920F931F936A01E090240CF09016
:10C93000250C0091260C1091270CFB0120813181E0
:10C9400042815381FC0160817181828193810E94C7
:10C95000D2631F910F91FF90EF90DF90CF900895D9
:10C96000CF92DF92EF92FF920F931F936B01FC0126
:10C97000E080F18002811381ECE1FCE024813581CB
:10C980004681578160817181828193810E94D26347
:10C990001F910F91FF90EF90DF90CF9008950F932C
:10C9A0001F93CF93DF93EC018B0181E00E9441F94B
:10C9B00069E170E080E090E00E943226B801CE018B
:10C9C0000E94B064C091DC0680E00E9441F91092A0
:10C9D000DC0682E00E94F22F0E94282BC2FBCC27AB
:10C9E000C0F981E08C27DF91CF911F910F910895BD
:10C9F000AF92BF92CF92DF92EF92FF920F931F936D
:10CA0000CF93DF9300D01F92CDB7DEB7FC01E0805B
:10CA1000F18002811381611112C0A090240CB090AA
:10CA2000250CC090260CD090270C9501A601B701CB
:10CA3000C8010F94132687FF02C07501860120E00C
:10CA400030E04BEE53E4B701C8010F94132687FD85
:10CA500004C0E12CF12C0BEE13E4C701D80189834B
:10CA60009A83AB83BC8360EE72E0CE0101960E9494
:10CA7000B0640F900F900F900F90DF91CF911F91A6
:10CA80000F91FF90EF90DF90CF90BF90AF900895FF
:10CA90003F924F925F926F927F928F929F92AF924E
:10CAA000BF92CF92DF92EF92FF920F931F93CF939B
:10CAB000DF9300D01F92CDB7DEB7382E80E090E034
:10CAC000A0E2B1E489839A83AB83BC83C0907512E2
:10CAD000D0907612E0907712F090781220E030E05B
:10CAE000A901C701B6010F94132687FF0CC0A70147
:10CAF000960160E070E080E291E40F94E22C69839B
:10CB00007A838B839C8360E0CE0101960E94F86457
:10CB100040901C0C50901D0C60901E0C70901F0CCF
:10CB20008090200C9090210CA090220CB090230CAF
:10CB3000332089F10E94EA5419821A821B821C82D6
:10CB4000E090240CF090250C0091260C1091270CFD
:10CB5000CE0101966C01A5019401C301B2010E94AE
:10CB6000D263309278070E94972B0F900F900F900E
:10CB70000F90DF91CF911F910F91FF90EF90DF9079
:10CB8000CF90BF90AF909F908F907F906F905F906D
:10CB90004F903F9008950E94A754CECF8091780780
:10CBA000882319F080E00E94486580E008952F9264
:10CBB0003F924F925F926F927F928F929F92AF922D
:10CBC000BF92CF92DF92EF92FF920F931F93CF937A
:10CBD000DF93CDB7DEB766970FB6F894DEBF0FBE12
:10CBE000CDBFF82E282E312CF101EA56F64ED49006
:10CBF00022E0821335C080917807811103C081E063
:10CC00000E9448650E94EA54811139C182E999E184
:10CC10000E94AF1D20E030E0A9010F941326882365
:10CC2000F9F06D2DDD0C770B880B990B0F941A26FC
:10CC30002B013C0182E999E10E94AF1D4B015C018F
:10CC400020E030E040EA50E40F94132611E087FF23
:10CC50001CC0812C912C90EAA92E90E4B92E15C00D
:10CC60006D2DDD0C770B880B990B0F941A262B0179
:10CC70003C01C101880F991F880F991F8657964E56
:10CC80000E94AF1D4B015C0110E0A3019201C501A0
:10CC9000B4010F9479264B015C016101CC0CDD1CC1
:10CCA000CC0CDD1CC6018258964E0E94AF1DEE24AE
:10CCB000E394E12620E030E040EC5FE30F94792636
:10CCC000A30192010F947926AB01BC0100E010E0B2
:10CCD00098018F2D0E94EB6220E030E0A901C50190
:10CCE000B4010F941326F601EE58F64EFA8BE98B39
:10CCF000882309F44DC0F2E000E010E020E431E4C4
:10CD0000FF1619F000E010E09801B501A401705879
:10CD1000E12C8F2D0E94EB62A5019401C501B401A5
:10CD20000F94E32C6B8B7C8B8D8B9E8B22E0F21609
:10CD3000E9F0F101E159F64E6491611107C00E94DA
:10CD4000334E8DE499E10E9460386AE070E090E033
:10CD500080E00F9418269B01AC0160E070E088E44D
:10CD600092E40F94DD2D8B019C0104C000E010E0E3
:10CD700020EC30E4EE24E3944B895C896D897E8954
:10CD80008F2D0E94EB6232E0F312D0C00E94A754B4
:10CD900081E090E0A0E0B0E00F2C04C0880F991F64
:10CDA000AA1FBB1F0A94D2F720912C0C282B20938A
:10CDB0002C0C20919205822B8093920589899A8967
:10CDC0000E94AF1DF601E45EF34F6083718382839E
:10CDD000938382E0F8121AC0209175123091761276
:10CDE00040917712509178126091240C7091250C2B
:10CDF0008091260C9091270C0F94E22C6093240CC8
:10CE00007093250C8093260C9093270CF601E25129
:10CE1000F84F10821182128213828F2D0E94CC1C37
:10CE20000E94282BF601E45EF34F80819181A2815C
:10CE3000B381F601E859F84F80839183A283B383CD
:10CE400092E0F916A9F18CE0ECEAF2E0DE0111962D
:10CE500001900D928A95E1F7E1E0F0E0EC0FFD1F03
:10CE6000EC0DFD1D80809180A280B38020E030E039
:10CE7000A901C501B4010F94132681111EC0669645
:10CE80000FB6F894DEBF0FBECDBFDF91CF911F91DB
:10CE90000F91FF90EF90DF90CF90BF90AF909F9059
:10CEA0008F907F906F905F904F903F902F9008955C
:10CEB0000E94CE658111E3CFC6CF20E030E0A9010A
:10CEC000C501B4010F94432F87FF04C0B7FAB09493
:10CED000B7F8B094F601E45EF34F6F01A30192013D
:10CEE000C501B4010F9479269B01AC01F601608164
:10CEF0007181828193810F94E22CF60160837183AA
:10CF000082839383F2E080E090E0A0E4B1E4FF1636
:10CF100021F080E090E0A8E4B2E48D879E87AF879F
:10CF2000B88BCE010D960E940D2BA9CF81E090E029
:10CF3000A0E0B0E00F2C04C0880F991FAA1FBB1FF0
:10CF40000A94D2F720912C0C282B20932C0C2091A2
:10CF50009205822B8093920589899A890E94AF1D40
:10CF6000F601E45EF34F60837183828393834ECF37
:10CF7000CF93DF9300D01F92CDB7DEB780E090E073
:10CF8000A0EAB0E489839A83AB83BC8361E0CE01DD
:10CF900001960E94F8640F900F900F900F90DF9110
:10CFA000CF9108958F929F92AF92BF92CF92DF92CE
:10CFB000EF92FF920F931F93CF93DF93CDB7DEB71E
:10CFC0002C970FB6F894DEBF0FBECDBF8B0140E0AB
:10CFD00050E068E472E44D835E836F83788740E0BD
:10CFE00050E060EA70E449875A876B877C8781301C
:10CFF000B9F1823009F459C020E030E040E050E45B
:10D000006091240C7091250C8091260C9091270C36
:10D010000F94E32C4B017C0120E030E04BEE53E415
:10D020000F94432F181634F4812C912C8BEEE82E9C
:10D0300093E4F92EF801A084B184C284D3849401CE
:10D04000A701B501C6010F94432F181614F054011F
:10D050006701C501D60189839A83AB83BC8348C02D
:10D06000BE01675F7F4FC80108960E94B064B80197
:10D070006C5F7F4FAE014B5F5F4FC8010E948E64B3
:10D080000E94C2302C960FB6F894DEBF0FBECDBF03
:10D09000DF91CF911F910F91FF90EF90DF90CF9094
:10D0A000BF90AF909F908F900895F80120853185B3
:10D0B000428553856091240C7091250C8091260C3B
:10D0C0009091270C0F94E32C6B017C0120E030E061
:10D0D0004BEE53E40F94132687FD06C0C12CD12CD0
:10D0E0002BEEE22E23E4F22EC982DA82EB82FC825E
:10D0F000BE01675F7F4FCE010196B7CFEF92FF92DF
:10D100000F931F93CF93DF937C018B010E94BC315F
:10D11000CCE1DCE020916102309162024091630237
:10D1200050916402F70160817181828193810F9433
:10D13000DD2D2C853D854E855F850F94E32C6C8716
:10D140007D878E879F87C8010E940D2BDF91CF912D
:10D150001F910F91FF90EF900C94A5614F925F92F9
:10D160006F927F92AF92BF92CF92DF92EF92FF9237
:10D170000F931F93CF93DF9300D000D01F921F9285
:10D18000CDB7DEB75C0180E090E0A0E7B2E4898330
:10D190009A83AB83BC8380E090E0A0E8B0EC8D8301
:10D1A0009E83AF83B887BE016F5F7F4FCE01059628
:10D1B0000E947E6868E873E180E090E00E94322679
:10D1C000C12CD12C88ECE82E81E4F82EC982DA82B9
:10D1D000EB82FC8280E090E0A0E8B0E48D839E8347
:10D1E000AF83B887BE016F5F7F4FCE0105960E9467
:10D1F0007E680EE21CE0F80140AC51AC62AC73AC4E
:10D20000C0AED1AEE2AEF3AE80E090E0A0EAB1E411
:10D2100089839A83AB83BC83F50180819181A2814C
:10D22000B3818D839E83AF83B887BE016F5F7F4FCD
:10D23000CE0105960E947E68F80140AE51AE62AE06
:10D2400073AE129A64E670E080E090E00E943226AD
:10D2500081E028960FB6F894DEBF0FBECDBFDF91F8
:10D26000CF911F910F91FF90EF90DF90CF90BF90E3
:10D27000AF907F906F905F904F9008951F93CF93E2
:10D28000DF93CDB7DEB72C970FB6F894DEBF0FBE95
:10D29000CDBF182F882379F020E030E0A9016091FC
:10D2A000CA057091CB058091CC059091CD050F9466
:10D2B00013268823F9F080912D0C8117D9F00E9454
:10D2C000A5618CE0E8EBF2E0DE01119601900D9291
:10D2D0008A95E1F7CE0101960E945B1F80912D0C8B
:10D2E000882391F08CE19CE00E94342710922D0C51
:10D2F0000E94282B2C960FB6F894DEBF0FBECDBF30
:10D30000DF91CF911F91089581E080932D0C8CE1E6
:10D310009CE00E944821ECCF2F923F924F925F9267
:10D320006F927F928F929F92AF92BF92CF92DF9235
:10D33000EF92FF920F931F93CF93DF93CDB7DEB79A
:10D34000CB54D1090FB6F894DEBF0FBECDBF2DB7B9
:10D350003EB739AF28AF87E00E94434E81110BC022
:10D3600061E086E50E9480248DA3853060F087E32C
:10D370009EE00E946038A8ADB9AD0FB6F894BEBF6C
:10D380000FBEADBF40C33DA1332321F087E19EE036
:10D390000E9460386AE080E50E948024182F8CEF9C
:10D3A000810F8F3218F083EF9DE0E3CF60E085E4DA
:10D3B0000E949C24882309F448C081E08FABE09050
:10D3C0007912F0907A12D7012D913D914D915C9197
:10D3D00060911C0C70911D0C80911E0C90911F0C83
:10D3E0000F94E32CAB01BC0188E50E94EE24698711
:10D3F0007A878B879C87F701248135814681578105
:10D400006091200C7091210C8091220C9091230C42
:10D410000F94E32CAB01BC0189E50E94EE246D87DB
:10D420007E878F87988BBE01635F7F4FCE01099601
:10D430000E94622E382E81110BC063E68FED9DE0B5
:10D440000E94CE3F87EC9DE094CF92E09FABB7CF98
:10D450008CE40E94701E082F882309F431C10E94B9
:10D460006C248EA3803118F080EA9DE082CFFEA16B
:10D47000F13009F427C160E083E50E949C248AAF63
:10D48000882321F0011102C037E03EA38DA1833033
:10D4900020F086E89DE00E94603890912D0C9DAFB1
:10D4A00080E00E943E690E94051D1D8A1E8A1F8A17
:10D4B000188E198E1A8E1B8E1C8E83EF9FE4A3ECA0
:10D4C000B7E48D8F9E8FAF8FB8A383EF9FE4A3EC5B
:10D4D000B7EC89A39AA3ABA3BCA3A12FB0E0BCA7D0
:10D4E000ABA7EDB7FEB724E0129FE019F1091124B4
:10D4F0000FB6F894FEBF0FBEEDBF8DB79EB7019675
:10D500009CAF8BAF2DA14FA9BE01635F7F4FCE01B2
:10D5100009960E94D0F99B01AC010F94D52F81117F
:10D5200062C20E9472FD611571058105910511F0BD
:10D530000F949921212C1BAA1CAA1DAA1EAAAEA1D8
:10D54000A150BB0B2C96BFAFAEAF2C97E22DF0E0F5
:10D55000F8A7EFA32BA53CA5E217F3070CF074C2C4
:10D560003196FEA7EDA73F932F93FF93EF9382E7AA
:10D570009DE09F938F938CE79DE09F938F931F92E5
:10D580000E945FF98DB79EB709960FB6F8949EBFBB
:10D590000FBE8DBF9EA1992309F458C10F944A2153
:10D5A0002AE030E040E050E00F94792C0F941A26E6
:10D5B00020E030E040EA50E40F94432F0FEF1FEFDC
:10D5C000181614F001E010E00F944A2128E631E02B
:10D5D00040E050E00F94792C0F941A262B013C0167
:10D5E0000F944A2123E330E040E050E00F94792C7F
:10D5F0006B5F7F4F8F4F9F4F0F941A264B015C013B
:10D60000ADA1A430D1F4BC01A40184E69DE00E9448
:10D610003C41B301A2018CE59DE00E943C4186E5BE
:10D620009DE00E9460380130110519F483E40E94E6
:10D63000273882E59DE00E946038312CC801110F27
:10D64000AA0BBB0B2A968CAF9DAFAEAFBFAF2A978C
:10D650002C96AEADBFAD2C973A161B060CF0F6C05B
:10D660002A966CAD7DAD8EAD9FAD2A970F941A268C
:10D670006B017C01BAADBB2341F1AC019B010F945E
:10D68000E32C20E030E040E952E40F9479269B013E
:10D69000AC01C301B2010F94E32C2B013C0120E04B
:10D6A00030E044EB53E40F94432F1816FCF420E0D1
:10D6B00030E044EB53E4C301B2010F94E22CEDCF10
:10D6C0001EA2D9CE22E02EA3D6CE0F944A2124E169
:10D6D00030E040E050E00F94792C675E7F4F8F4F31
:10D6E0009F4F0F941A26A7019601CFCF20E030E07C
:10D6F000A901C301B2010F94132687FF0BC020E0DC
:10D7000030E044EB53E4C301B2010F94E32C2B014E
:10D710003C01ECCF0091791210917A12F80124812A
:10D720003581468157816D857E858F8598890F94D7
:10D73000E22C22966CAF7DAF8EAF9FAF22972BED80
:10D740003FE049E450E4C301B2010F94792620E0A0
:10D7500030E044E353E40F94DD2D6B017C010F9422
:10D76000D82D6FA778AB89AB9AABD8012D913D919D
:10D770004D915C9169857A858B859C850F94E22C0F
:10D7800026966CAF7DAF8EAF9FAF2697A501940113
:10D790006FA578A989A99AA90F9479269B01AC0154
:10D7A00026966CAD7DAD8EAD9FAD26970F94E32C84
:10D7B00069837A838B839C83C701B6010F94832F7F
:10D7C000A50194010F94792622962CAD3DAD4EAD66
:10D7D0005FAD22970F94E32C6D837E838F839887B0
:10D7E00042EC51E070E060E0CE0101960E94EDC194
:10D7F00042EC51E070E060E0CE0105960E94EDC180
:10D80000BDA1B43099F449815A816B817C8186E451
:10D810009DE00E943C414D815E816F81788584E668
:10D820009FE20E943C418AE00E942738198A1A8AA6
:10D830001B8A1C8AAE014F5E5F4FBE016B5F7F4F3C
:10D84000CE0101960E948E64339402CF20E04FA94E
:10D85000BE01635F7F4FCE0109960E94D0F94B0154
:10D860005C01312CAC019B010F94D52F811102C0BA
:10D8700033243394A5019401C501B4010F94D52F2D
:10D880008111E2C0EFA1F8A5EE0FFF1FEE0FFF1F01
:10D890002BAD3CADE20FF31F80829182A282B38256
:10D8A000A50194016D8D7E8D8F8D98A10F94432FCE
:10D8B000181624F48D8E9E8EAF8EB8A2A501940109
:10D8C00069A17AA18BA19CA10F94132687FF04C0A4
:10D8D00089A29AA2ABA2BCA2A50194016BA97CA9C2
:10D8E0008DA99EA90F94E32C6BAB7CAB8DAB9EAB4B
:10D8F000ADA5BEA5BD01BB0F880B990B0F941A26D1
:10D900006FA378A789A79AA79B01AC016BA97CA9F3
:10D910008DA99EA90F94DD2D2B013C014D8A5E8AB5
:10D920006F8A788EEBADFCADF8ABEFA710E0C12CA1
:10D93000D12C7601AFA5B8A96D917D918D919D9166
:10D94000B8ABAFA7A30192010F94E22C9B01AC01ED
:10D950000F9479269B01AC01C701B6010F94E32C0B
:10D960006B017C011F5F211628F72FA138A549A55F
:10D970005AA50F94DD2D0F94912F698F7A8F8B8F7D
:10D980009C8FBDA1B23068F18DA59EA50E948FE14C
:10D990006BA57CA581E49DE00E945E418BE39DE048
:10D9A0000E94603843E0C501B4010E946FBA80E272
:10D9B0000E94273881E0EDA1E3300CF480E0E12CF7
:10D9C0008E010F5D1F4F9E01235E3F4FAE01475EEC
:10D9D0005F4FBE016B5E7F4F0E941D3F8AE00E9439
:10D9E00027382394B3CD0E94CE650E94EC1C8DADE8
:10D9F0000E943E690E94C23088AD99AD0FB6F8947E
:10DA00009EBF0FBE8DBFE8ADF9AD0FB6F894FEBF57
:10DA10000FBEEDBFC55BDF4F0FB6F894DEBF0FBE84
:10DA2000CDBFDF91CF911F910F91FF90EF90DF90CD
:10DA3000CF90BF90AF909F908F907F906F905F90AE
:10DA40004F903F902F9008950E94CE65332069F249
:10DA500080E39DE00E94603881E0FDA11F160CF07C
:10DA600080E0EE24E3948E010F5D1F4F9E01235E44
:10DA70003F4FAE01475E5F4FBE016B5E7F4F0E941E
:10DA80001D3F698D7A8D8B8D9C8D0052110926E08A
:10DA900042E00F94E0209F938F938FE19DE09F934E
:10DAA0008F9389E29DE09F938F931F920E945FF96D
:10DAB0002DB73EB7295F3F4F0FB6F8943EBF0FBE5C
:10DAC0002DBF93CF2F923F924F925F926F927F9292
:10DAD0008F929F92AF92BF92CF92DF92EF92FF927E
:10DAE0000F931F93CF93DF93CDB7DEB76A970FB62F
:10DAF000F894DEBF0FBECDBF83E50E94701E182FC5
:10DB000030902D0C882319F00E948C24382E4090E0
:10DB10001C0C50901D0C60901E0C70901F0C80917E
:10DB2000200C9091210CA091220CB091230C8B8B96
:10DB30009C8BAD8BBE8B8091240C9091250CA09179
:10DB4000260CB091270C8F8B988FA98FBA8F112339
:10DB500029F0311003C080E00E943E6986E50E94F2
:10DB6000701E8A8B20E030E0A9016091CA05709197
:10DB7000CB058091CC059091CD050F941326882379
:10DB800009F4C9C083E40E94701E882309F49DC073
:10DB90000E94C4246B017C01A4E8B7E0B987A88780
:10DBA000BF83AE83F5E0FD831D861E8628EC2F879C
:10DBB00002EC1A86212C88EC8B8792E49C87AE813C
:10DBC000BF81B98BA88B15E0E889F9898190919084
:10DBD000A190B190F98BE88B2A85322D4B855C851D
:10DBE000C501B4010F94132687FF04C08A86292C2F
:10DBF000AB86BC862D853E854F85502FC501B4016F
:10DC00000F94432F181624F48D869E86AF860B2D15
:10DC10001150D1F6FD81F150FD838E819F81449694
:10DC20009F838E83F111CBCF2D853E854F85502F5D
:10DC30006A85722D8B859C850F94E32C20E030E063
:10DC400040E05FE30F947926A70196010F94E32C3F
:10DC50004B015C012DEB37E346E855EB0F94432F66
:10DC600087FD0AC02DEB37E346E855E3C501B40153
:10DC70000F94132618164CF580E00E943E6910E0C0
:10DC8000E884F98400E0D7016D917D918D919D919B
:10DC90007D016D01B4E0CB1AD108A50194010F9468
:10DCA000E22CF6016083718382839383602F812F3E
:10DCB0000E9434F80F5F053031F71F5F8885998522
:10DCC0004496998788871530D9F6AA89AA2381F0C6
:10DCD00020E030E0A9016091CA057091CB058091E8
:10DCE000CC059091CD050F94132681110E94A5407B
:10DCF0008AE50E94701E882351F00E94C424698323
:10DD00007A838B839C83CE0101960E94FCF6832D3F
:10DD10000E943E690BC0311003C09A89992341F3D8
:10DD20000E94334E80E69CE00E946038332051F020
:10DD300080912D0C811106C00E942F4E81E49CE041
:10DD40000E9460380E94334E83E39CE00E9460385A
:10DD500080912D0C0E941E410E94334E86E29CE071
:10DD60000E946038C090C008D090C108E090C208FE
:10DD7000F090C30820E030E0A901C701B6010F947C
:10DD8000432F18160CF053C042E0C701B6010E94A1
:10DD90006FBA8DE00E9427388AE00E942738A301DD
:10DDA000920160911C0C70911D0C80911E0C909141
:10DDB0001F0C0F94132681111FC02B893C894D899C
:10DDC0005E896091200C7091210C8091220C9091C1
:10DDD000230C0F94132681110FC02F89388D498D84
:10DDE0005A8D6091240C7091250C8091260C909195
:10DDF000270C0F94132681110E94C2306A960FB629
:10DE0000F894DEBF0FBECDBFDF91CF911F910F9170
:10DE1000FF90EF90DF90CF90BF90AF909F908F904A
:10DE20007F906F905F904F903F902F90089581E288
:10DE30009CE00E946038B3CF8F929F92AF92BF92C6
:10DE4000EF92FF920F931F93CF93DF9380E00E9496
:10DE50003E691092C6051092C7051092C80510922F
:10DE6000C9051092C2051092C3051092C405109204
:10DE7000C5051092CE051092CF051092D0051092D4
:10DE8000D1051092CA051092CB051092CC051092C4
:10DE9000CD0504E817E0C0E0812C912C80ECA82E81
:10DEA0008FE7B82E7801D0E0F70181929192A1928C
:10DEB000B1927F016D2F8C2F0E9434F8DF5FD53037
:10DEC00099F7CF5F0C5E1F4FC53061F7DF91CF919F
:10DED0001F910F91FF90EF90BF90AF909F908F9008
:10DEE000089590917E1280917F12981308C08091BE
:10DEF000F8089091F908892B11F40C942A1F80E0FE
:10DF00000E943B5AEECF83E50E94BE1E8823E9F0B3
:10DF10000E9472FD60936B1170936C1180936D1170
:10DF200090936E110E94C42420E030E04AE754E44C
:10DF30000F9479260F94562E609313027093140257
:10DF40008093150290931602089580912B0584FD0D
:10DF50000AC080912D0587FD06C080912E05837033
:10DF600011F40C94716F0E94A56188E50E94701EE7
:10DF7000882331F05F9A80912C0C8E7F80932C0C3B
:10DF800089E50E94701E882331F08A9A80912C0CBA
:10DF90008D7F80932C0C8AE50E94701E882359F097
:10DFA00080910801809581708093060180912C0CEE
:10DFB0008B7F80932C0C85E40E94701E81110C9441
:10DFC000281F08952F923F924F925F926F927F92F7
:10DFD0008F929F92AF92BF92CF92DF92EF92FF9279
:10DFE0000F931F93CF93DF93CDB7DEB7A6970FB6EE
:10DFF000F894DEBF0FBECDBF88E697E00E94552A99
:10E000008091DA0B83FD7EC02091280C3091290C81
:10E0100040912A0C50912B0C6091740770917507F8
:10E0200080917607909177070F941326882309F43F
:10E0300069C01091F708111161C080915F02909141
:10E04000600201972091E0113091E1112817390702
:10E050003CF40E94334E80E299E10E94603811E066
:10E060002091280C3091290C40912A0C50912B0CB6
:10E07000609174077091750780917607909177078A
:10E080000F94E22C6B017C0120E030E0A9010F9499
:10E09000432F87FF04C0F7FAF094F7F8F09420912B
:10E0A0006102309162024091630250916402C701A3
:10E0B000B6010F94792620E030E84BE354E40F9446
:10E0C000432F1816ECF40E94334E81E099E10E9430
:10E0D00060388091740790917507A0917607B09190
:10E0E00077078093280C9093290CA0932A0CB09367
:10E0F0002B0C84E797E00E94B66104C010E0B0CF1B
:10E100001111E7CF2AE037ED43E25CE36091410271
:10E110007091420280914302909144020F947926BB
:10E120006B017C016091670270916802072E000C00
:10E13000880B990B0F941A269B01AC01C701B601FD
:10E140000F947926698B7A8B8B8B9C8B80912D0C0D
:10E15000882309F18090C0089090C108A090C2085F
:10E16000B090C308C0907007D0907107E09072071C
:10E17000F090730720E030E0A901C501B4010F94CD
:10E1800013268823D1F1A7019601C501B4010F948C
:10E19000432F181694F1C12CD12C76018E010F5EFD
:10E1A0001F4F24E737E040E757E06CE677E088E66A
:10E1B00097E00E94B5F480E1E8E6F7E0ACE1BCE06E
:10E1C00001900D928A95E1F7A6960FB6F894DEBFFE
:10E1D0000FBECDBFDF91CF911F910F91FF90EF90B8
:10E1E000DF90CF90BF90AF909F908F907F906F9077
:10E1F0005F904F903F902F90089520911C0C30918C
:10E200001D0C40911E0C50911F0C6091680770917D
:10E21000690780916A0790916B070F94E22C6D8BD0
:10E220007E8B8F8B988F2091200C3091210C409108
:10E23000220C5091230C60916C0770916D078091B6
:10E240006E0790916F070F94E22C698F7A8F8B8FF6
:10E250009C8F2091240C3091250C4091260C5091DC
:10E26000270CC701B6010F94E22C6D8F7E8F8F8F24
:10E2700098A32091280C3091290C40912A0C5091A0
:10E280002B0C6091740770917507809176079091BF
:10E2900077070F94E22C6B017C0120E030E0A901AC
:10E2A0006D897E898F89988D0F94132681110CC0FA
:10E2B00020E030E0A901698D7A8D8B8D9C8D0F94C3
:10E2C0001326882309F467CF2D893E894F89588DFD
:10E2D000CA01B9010F9479264B015C01298D3A8D51
:10E2E0004B8D5C8DCA01B9010F9479269B01AC015D
:10E2F000C501B4010F94E32C4B015C012D8D3E8DC3
:10E300004F8D58A1CA01B9010F9479269B01AC0128
:10E31000C501B4010F94E32C4B015C01A7019601E8
:10E32000C701B6010F9479269B01AC01C501B40168
:10E330000F94E32C0F94912F4B015C012DEB37E3ED
:10E3400046E855E30F94132687FF0FC020E030E026
:10E35000A901C701B6010F94432F4601570187FF5A
:10E3600004C0B7FAB094B7F8B0942DEB37E346E8A1
:10E3700055E3C501B4010F94132687FD1CCF20E09F
:10E3800030E040EA51E4C501B4010F94DD2D0F9453
:10E39000562E1B01672B19F422242394312CB10132
:10E3A00090E080E00F9418269B01AC0160E070E0E3
:10E3B00080E89FE30F94DD2D2B013C01AC019B0114
:10E3C000C501B4010F9479264B015C01A3019201B0
:10E3D0006D897E898F89988D0F9479266D8B7E8BC0
:10E3E0008F8B988FA3019201698D7A8D8B8D9C8D77
:10E3F0000F947926698F7A8F8B8F9C8FA30192015E
:10E400006D8D7E8D8F8D98A10F9479266D8F7E8F67
:10E410008F8F98A3A3019201C701B6010F947926AB
:10E4200069A37AA38BA39CA380E1ECE1FCE08E01BD
:10E430000F5F1F4FD80101900D928A95E1F70E945E
:10E4400072FD2B013C0128EC420E511C611C711C19
:10E450000DA31EA381E0281A310809F460C00E94B0
:10E4600072FD8B019C01041915092609370937FD36
:10E4700059C02B013C0128EC420E511C611C711C3F
:10E4800080E00E943B5A2D893E894F89588D6981D1
:10E490007A818B819C810F94E32C69837A838B83AF
:10E4A0009C83298D3A8D4B8D5C8D6D817E818F8112
:10E4B00098850F94E32C6D837E838F8398872D8DB1
:10E4C0003E8D4F8D58A169857A858B859C850F94EB
:10E4D000E32C69877A878B879C8729A13AA14BA176
:10E4E0005CA16D857E858F8598890F94E32C6D875F
:10E4F0007E878F87988B750164018E010F5E1F4F99
:10E500009E01235F3F4FAE01475F5F4FBE016B5FD0
:10E510007F4F8DA19EA10E94B5F481119BCF750103
:10E5200064013CCE0E942FC2AECF8F929F92AF92D9
:10E53000BF92CF92DF92EF92FF92CF93DF938090C2
:10E54000410290904202A0904302B0904402FC012C
:10E55000C080D180E280F38020E030E0A901C701D3
:10E56000B6010F941326882341F0C0924102D09245
:10E570004202E0924302F0924402C0916702D091BD
:10E58000680284E690E09093680280936702C090EE
:10E590006102D0906202E0906302F090640280E039
:10E5A00090E0A0E8BFE38093610290936202A093A1
:10E5B0006302B09364020E94E26F809241029092E3
:10E5C0004202A0924302B0924402D0936802C093E8
:10E5D0006702C0926102D0926202E0926302F092FE
:10E5E0006402DF91CF91FF90EF90DF90CF90BF90CA
:10E5F000AF909F908F9008950F931F93CF93DF93C9
:10E6000000D01F92CDB7DEB79C0108E617E090E17D
:10E61000ECE1FCE0D80101900D929A95E1F7F90147
:10E620002081318142815381F80160857185828525
:10E6300093850F94E32CF801608771878287938715
:10E6400080E090E0A0EAB0E489839A83AB83BC8346
:10E65000CE0101960E9495720F900F900F900F902F
:10E66000DF91CF911F910F9108952F923F924F927A
:10E670005F926F927F928F929F92AF92BF92CF9252
:10E68000DF92EF92FF921F93CF93DF93CDB7DEB768
:10E690002C970FB6F894DEBF0FBECDBF7A011901DB
:10E6A000DC012D913D914D915C912D833E834F83F3
:10E6B0005887FB01408051806280738080901C0CE1
:10E6C00090901D0CA0901E0CB0901F0CA501940101
:10E6D0006D817E818F8198850F94132681110EC0E4
:10E6E00011E0A30192016091200C7091210C8091A6
:10E6F000220C9091230C0F941326811110E0D1016C
:10E700002D913D914D915C9129873A874B875C878C
:10E71000F701C080D180E280F38020910B0230911C
:10E720000C0240910D0250910E02C701B6010F94E8
:10E730001326882309F44EC0C0920B02D0920C021B
:10E74000E0920D02F0920E028091280C9091290C1B
:10E75000A0912A0CB0912B0C4091200C5091210CCF
:10E760006091220C7091230C809268079092690747
:10E77000A0926A07B0926B0740936C0750936D07A5
:10E7800060936E0770936F07C0927007D092710705
:10E79000E0927207F0927307809374079093750765
:10E7A000A0937607B093770720E030E040E05FE386
:10E7B00060915A0C70915B0C80915C0C90915D0C97
:10E7C0000F94792669837A838B839C83CE0101968B
:10E7D0000E9495722D813E814F8158852093680754
:10E7E0003093690740936A0750936B0740926C0718
:10E7F00050926D0760926E0770926F07D1012D9154
:10E800003D914D915C916091740770917507809175
:10E810007607909177070F94E32C609374077093B9
:10E820007507809376079093770711112FC020E02A
:10E8300030E0A90169857A858B859C850F94132624
:10E84000811133C060E070E088EC92E469837A83E0
:10E850008B839C83CE0101960E9495722C960FB6F5
:10E86000F894DEBF0FBECDBFDF91CF911F91FF9017
:10E87000EF90DF90CF90BF90AF909F908F907F9060
:10E880006F905F904F903F902F9008952AEF3EE752
:10E890004AE25FE360915E0C70915F0C8091600CC6
:10E8A0009091610C0F947926D1CF60E070E080EAFE
:10E8B00091E4CCCF0F931F93CF93DF9300D000D080
:10E8C0001F921F92CDB7DEB78B01FC0123A521114A
:10E8D00002C00E94BDFB1D821E821F82188620E09E
:10E8E00030E040E05FE36091240C7091250C809152
:10E8F000260C9091270C0F94E32C69837A838B83E9
:10E900009C839E012B5F3F4FAE014F5F5F4F60E2E4
:10E910007CE08CE19CE00E9435731D821E821F8288
:10E92000188620E030E040E05FE3F8016085718503
:10E93000828593850F94E32C69837A838B839C83F0
:10E94000B8016C5F7F4F9E012B5F3F4FAE014F5F61
:10E950005F4FC8010E94357328960FB6F894DEBF4A
:10E960000FBECDBFDF91CF911F910F9108959B01F5
:10E97000AC01485F5F4FBC016C5F7F4F0C943573F7
:10E980002F923F924F925F926F927F928F929F92BF
:10E99000AF92BF92CF92DF92EF92FF920F931F93AD
:10E9A000CF93DF93CDB7DEB7A6970FB6F894DEBF4F
:10E9B0000FBECDBF8C011B015A87498740901C0CAC
:10E9C00050901D0C60901E0C70901F0C8090200CBD
:10E9D0009090210CA090220CB090230CDB018D9123
:10E9E0009D910D90BC91A02D8B8B9C8BAD8BBE8B84
:10E9F0009C01AD01C301B2010F94E22C6B017C01BB
:10EA0000D10114968D919D910D90BC91A02D8F8B6D
:10EA1000988FA98FBA8F9C01AD01C501B4010F94E5
:10EA2000E22C6B8F7C8F8D8F9E8FA985BA858D91FF
:10EA30009D910D90BC91A02D8B879C87AD87BE8743
:10EA40009C01AD01C301B2010F94E22C6F8F78A33A
:10EA500089A39AA3A985BA8514968D919D910D904D
:10EA6000BC91A02D8F87988BA98BBA8B9C01AD018F
:10EA7000C501B4010F94E22C6BA37CA38DA39EA3CC
:10EA8000A7019601C701B6010F9479266B017C019D
:10EA90002B8D3C8D4D8D5E8DCA01B9010F94792669
:10EAA0009B01AC01C701B6010F94E32C4B015C0143
:10EAB0002B893C894D895E896B857C858D859E85FA
:10EAC0000F94E22C2B013C012F89388D498D5A8DF2
:10EAD0006F85788989899A890F94E22C6B017C0172
:10EAE000A3019201C301B2010F9479262B013C01CD
:10EAF000A7019601C701B6010F9479269B01AC01CD
:10EB0000C301B2010F94E32C0F94912F6B017C0190
:10EB10002F8D38A149A15AA1CA01B9010F947926B4
:10EB20002B013C012BA13CA14DA15EA1CA01B90161
:10EB30000F9479269B01AC01C301B2010F94E32C21
:10EB40009B01AC01C501B4010F94432F1816B4F515
:10EB500020E030E0A901C701B6010F94432F87FFE1
:10EB60002AC0C701B601905820E030E040EA50E4E6
:10EB70000F94432F181614F5A10169857A85C801F1
:10EB80000E94C074A6960FB6F894DEBF0FBECDBF2C
:10EB9000DF91CF911F910F91FF90EF90DF90CF9079
:10EBA000BF90AF909F908F907F906F905F904F90AD
:10EBB0003F902F900895C701B601D6CF20E030E0F6
:10EBC00040E050E4C501B4010F94432F181624F41B
:10EBD000B101C8010E945A7419821A821B821C82D8
:10EBE000BE016F5F7F4FC1010E94B7742DEC3CECFA
:10EBF0004CEC5CE3C701B6010F9479269B01AC0194
:10EC0000F80160817181828193810F9479266D83EF
:10EC10007E838F839887D8019B968C919B978823BE
:10EC2000C9F02AE939E949E95FE314966D917D91CC
:10EC30008D919C9117970F94792669837A838B83A2
:10EC40009C83BE016F5F7F4F88E697E00E94B77498
:10EC5000F80113A6BE016B5F7F4F89859A850E94DC
:10EC6000B77490CF3F924F925F926F927F928F9244
:10EC70009F92AF92BF92CF92DF92EF92FF920F934B
:10EC80001F93CF93DF93CDB7DEB76C970FB6F89491
:10EC9000DEBF0FBECDBFDB010C91142F100F15305E
:10ECA00008F067C11196DC90C22ECD0CB4E0BC1503
:10ECB00008F45FC1ED2DF0E0EE50FB4F8080912C09
:10ECC000B12CA12C002E04C0B694A79497948794DD
:10ECD0000A94D2F780FE4DC1EC2DF0E0EE50FB4FD0
:10ECE0008080912CB12CA12C012E04C0B694A79445
:10ECF000979487940A94D2F780FE3BC1322E642FFA
:10ED00007C014090C2055090C3056090C40570908E
:10ED1000C5058091CA059091CB05A091CC05B09115
:10ED2000CD05898F9A8FAB8FBC8F660F770B072E1F
:10ED3000000C880B990B0F941A264B015C01602F75
:10ED4000000F770B880B990B0F941A26298D3A8D9B
:10ED50004B8D5C8D0F947926A30192010F94E32CC7
:10ED6000A50194010F94E32C6D877E878F87988B84
:10ED7000612F110F770B880B990B0F941A26298D91
:10ED80003A8D4B8D5C8D0F947926A30192010F94DF
:10ED9000E32CA50194010F94E22C69837A838B8381
:10EDA0009C834090C6055090C7056090C805709040
:10EDB000C9058091CE059091CF05A091D005B09165
:10EDC000D105898F9A8FAB8FBC8F632D660F770B20
:10EDD000072E000C880B990B0F941A264B015C012F
:10EDE0006D2DDD0C770B880B990B0F941A26298D4E
:10EDF0003A8D4B8D5C8D0F947926A30192010F946F
:10EE0000E32CA50194010F94E32C698B7A8B8B8BF7
:10EE10009C8B6C2DCC0C770B880B990B0F941A26BE
:10EE2000298D3A8D4B8D5C8D0F947926A30192012B
:10EE30000F94E32CA50194010F94E22C6D837E8343
:10EE40008F839887F70180859185A285B38589870F
:10EE50009A87AB87BC878D8B9E8BAF8BB88F41EC2D
:10EE600051E061E070E0CE0141960E94EDC141ECBD
:10EE700051E061E070E0CE0105960E94EDC141ECE9
:10EE800051E061E070E0CE010D960E94EDC141ECD1
:10EE900051E061E070E0CE0101960E94EDC18988E9
:10EEA0009A88AB88BC8827E137EB41ED58EBC50168
:10EEB000B4010F94432F87FD5CC023E030E041EEA6
:10EEC00053E4C501B4010F94132618160CF451C075
:10EED0008D849E84AF84B88827E137EB41ED58EBF1
:10EEE000C501B4010F94432F87FD43C023E030E0F8
:10EEF00041EE53E4C501B4010F9413261816CCF16A
:10EF00008D809E80AF80B88427E137EB41ED58EBD0
:10EF1000C501B4010F94432F87FD2BC023E030E0DF
:10EF200041EE53E4C501B4010F94132618160CF1F9
:10EF300089809A80AB80BC8027E137EB41ED58EBAC
:10EF4000C501B4010F94432F87FD13C023E030E0C7
:10EF500041EE53E4C501B4010F94132618164CF08A
:10EF6000AE014F5F5F4FBE01635F7F4FC7010E94DD
:10EF7000C0746C960FB6F894DEBF0FBECDBFDF91A4
:10EF8000CF911F910F91FF90EF90DF90CF90BF90A6
:10EF9000AF909F908F907F906F905F904F903F9039
:10EFA00008952F923F924F925F926F927F928F922D
:10EFB0009F92AF92BF92CF92DF92EF92FF920F9308
:10EFC0001F93CF93DF93CDB7DEB7CC58D1090FB6DF
:10EFD000F894DEBF0FBECDBF80E19CE00E94603898
:10EFE00087E00E94434E81116EC084E50E94BE1EE0
:10EFF000882329F00E94B12481110E945DBA80E02B
:10F0000090E0A0E8BFE389839A83AB83BC838D83C0
:10F010009E83AF83B8878DEC9CECACE4BEE389871C
:10F020009A87AB87BC8780E090E0A0E2B1E48D874F
:10F030009E87AF87B88B8CE390E09A8B898B8DECA1
:10F0400090E09C8B8B8B8DEC9CECACECBEE38D8BC1
:10F050009E8BAF8BB88F80E090E0A0EEBFE3898FEE
:10F060009A8FAB8FBC8F1BA61CA64AE959E969E9A8
:10F070007EE38FE40E94EE246D8F7E8F8F8F98A3A6
:10F0800060E083E40E949C2489A360E08BE40E94FA
:10F090009C248AA382E40E94BE1E882381F10E94E0
:10F0A000B124009761F19C012852310925363105C0
:10F0B00020F16CE870E082EE9BE00E945E418DEDF5
:10F0C0009BE00E946038C457DF4F0FB6F894DEBF54
:10F0D0000FBECDBFDF91CF911F910F91FF90EF90A9
:10F0E000DF90CF90BF90AF909F908F907F906F9068
:10F0F0005F904F903F902F9008959A8B898B8CE46E
:10F100000E94BE1E8823E1F00E94C4246B017C0192
:10F11000C986DA86EB86FC8620E030E0A9010F94F0
:10F12000432F87FD0AC020E030E040E050E4C701F3
:10F13000B6010F94132618161CF485EB9BE0C1CF83
:10F1400081E50E94701E882331F18091FB0490912B
:10F15000FC04892BE9F00E94C4246B017C01CD8260
:10F16000DE82EF82F8862DEC3CEC4CE45DE30F94FC
:10F17000432F87FD0AC020E030E040E751E4C7019B
:10F18000B6010F941326181634F484E89BE099CF47
:10F1900089E59BE096CF83E50E94BE1E8823E9F0B7
:10F1A0000E94C4246B017C01CD8ADE8AEF8AF88E2E
:10F1B0002DEC3CEC4CEC5DE30F94432F87FD0AC033
:10F1C00020E030E040E050E4C701B6010F94132680
:10F1D00018161CF482E39BE074CF80E50E94701E39
:10F1E000882341F18091FB049091FC04892B19F450
:10F1F0008AEF9AE066CF8BA58F5F8BA70E94C4240D
:10F200006B017C01CD86DE86EF86F88A20E030E057
:10F21000A9010F94432F87FD0AC020E030E048EC9D
:10F2200051E4C701B6010F94132618161CF482EDA1
:10F230009AE047CF86E40E94BE1E8823E9F00E9430
:10F24000C4246B017C01C98EDA8EEB8EFC8E20E02B
:10F2500030E040E85FE30F94432F87FD0AC020E0D1
:10F2600030E040E850E4C701B6010F9413261816A9
:10F270001CF489EA9AE025CFC98CDA8CEB8CFC8CE3
:10F280008D889E88AF88B88CA7019601C701B6010A
:10F290000F9479269B01AC0160E070E084E490E477
:10F2A0000F94DD2D29813A814B815C810F94792661
:10F2B0002B013C01A5019401C501B4010F947926ED
:10F2C000A70196010F9479262CEE31E548EB5DE31A
:10F2D0000F94DD2D9B01AC01C301B2010F9479267F
:10F2E00069837A838B839C8388E40E94BE1E882373
:10F2F00079F00E94B124009759F09C01255A3109F8
:10F300002838310518F08BE79AE0DBCE9C8B8B8B8D
:10F3100085E50E94701E8823C9F00E9472FD611568
:10F3200071058105910511F00F9499218091FB04DD
:10F330009091FC04892B91F00E94C4246093F704FF
:10F340007093F8048093F9049093FA0482E50E9484
:10F35000701E811108C087E49AE0B3CE60E070E0CF
:10F3600088E492E4EBCF8091FB049091FC04892B1C
:10F3700061F00E94B124AD969FAF8EAFAD97181685
:10F3800019064CF083E19AE09CCE2AE130E0AD967C
:10F390003FAF2EAFAD9789E50E94BE1E882381F155
:10F3A0000E94C4242091C8083091C9084091CA081D
:10F3B0005091CB080F94E22C6B017C0188E50E94F0
:10F3C000BE1E882331F10E94C4242091C4083091CC
:10F3D000C5084091C6085091C7080F94E22C6BA352
:10F3E0007CA38DA39EA3CFA2D8A6E9A6FAA6CE01A0
:10F3F00083960E942F1E811115C089EE99E061CE7F
:10F40000C090200CD090210CE090220CF090230CA6
:10F41000D5CF60911C0C70911D0C80911E0C9091A9
:10F420001F0CDDCF84E40E94701E91E089270E94AA
:10F430003E6980E090E0A0EAB0E48DA79EA7AFA768
:10F44000B8AB60E0CE018D960E94F8643091ED0774
:10F45000CD57DF4F3883C358D0401092ED070E943C
:10F46000291C88EC99E00E94603889899A898A3140
:10F4700091050CF044C08B899C890E94461F61E075
:10F4800080E00E94FDBC811142C06FEF8DED99E0DC
:10F490000E94CE3F8CA5811104C0CE0101960E942E
:10F4A000BDFB80E090E0A0EAB0E480937007909309
:10F4B0007107A0937207B09373071DA61EA61FA61F
:10F4C00018AABE01635D7F4F88E697E00E94B7747B
:10F4D000CD57DF4F5881C358D0405093ED070E945D
:10F4E000291C8AA18111EFCD109278111092771109
:10F4F0000E94B5BE90E080E00E94461FE4CD0E94CD
:10F50000842281E00E9486BB8111B5CFBECF1092CC
:10F51000280C1092290C10922A0C10922B0C88E2C5
:10F520009CE00E94B6618BA5882309F452C020E0BC
:10F5300030E040E751E460915E0C70915F0C809187
:10F54000600C9091610C0F94DD2D6DA77EA78FA7A5
:10F5500098AB80E1ECE1FCE0A8E6B7E001900D9209
:10F560008A95E1F72D853E854F855889609174070E
:10F570007091750780917607909177070F94E32C2F
:10F58000609374077093750780937607909377075D
:10F59000CE018D960E9495722D853E854F855889A6
:10F5A0006091740770917507809176079091770745
:10F5B0000F94E22C6093740770937507809376071D
:10F5C000909377078CA5811104C0CE0101960E940B
:10F5D000BDFBE2EFF4E085E0DF011D928A95E9F7DB
:10F5E00080E1ECE1FCE0A8E6B7E001900D928A959D
:10F5F000E1F789859A85AB85BC85809370079093E8
:10F600007107A0937207B09373071DA61EA61FA6CD
:10F6100018AABE01635D7F4F88E697E00E94B77429
:10F62000BE01635E7F4F88E697E00E94B77489A1B0
:10F63000882309F41CC420911C0C30911D0C4091AE
:10F640001E0C50911F0CE5962CAF3DAF4EAF5FAF37
:10F65000E5978091200C9091210CA091220CB09103
:10F66000230CE1968CAF9DAFAEAFBFAFE197312CCD
:10F67000212C9FEFA4969FAFA497AFEFA896AFAFB2
:10F68000A897BFEFC158DF4FB883CF57D040EFE402
:10F69000C058DF4FE883C058D040F3ECCF57DF4F5E
:10F6A000F883C158D04027E4CE57DF4F2883C25893
:10F6B000D04081E090E0A0E0B0E0022C04C0880FD0
:10F6C000991FAA1FBB1F0A94D2F7CC57DF4F88831C
:10F6D0009983AA83BB83C458D040A2EFB4E0E796D5
:10F6E000BFAFAEAFE79710E000E09101032C000C34
:10F6F000440B550BC857DF4F288339834A835B83FC
:10F70000C858D040C457DF4F2882CC58D040E79625
:10F71000AEADBFADE7978D91E796BFAFAEAFE797C0
:10F7200090E0B0E0A0E0CC57DF4F288139814A81DA
:10F730005B81C458D04082239323A423B523892B13
:10F740008A2B8B2B09F024C1C857DF4F6881798140
:10F750008A819B81C858D0400F941A262091CA05EF
:10F760003091CB054091CC055091CD050F94792671
:10F770002091C2053091C3054091C4055091C50543
:10F780000F94E32CEB966CAF7DAF8EAF9FAFEB97F2
:10F79000B801012E000C880B990B0F941A262091AA
:10F7A000CE053091CF054091D0055091D1050F94F1
:10F7B00079262091C6053091C7054091C805509122
:10F7C000C9050F94E32C6B017C01EB962CAD3DAD8C
:10F7D0004EAD5FADEB97E5966CAD7DAD8EAD9FAD5B
:10F7E000E5970F94E22C2B013C01A7019601E196CD
:10F7F0006CAD7DAD8EAD9FADE1970F94E22C4B01CA
:10F800005C01A3019201C301B2010F9479262B017F
:10F810003C01A5019401C501B4010F9479269B0117
:10F82000AC01C301B2010F94E32C0F94912F4B0153
:10F830005C01EB962CAD3DAD4EAD5FADEB976BA192
:10F840007CA18DA19EA10F94E22C2B013C01A7016C
:10F8500096016FA178A589A59AA50F94E22C6B015A
:10F860007C01A3019201C301B2010F9479262B01FF
:10F870003C01A7019601C701B6010F9479269B01AF
:10F88000AC01C301B2010F94E32C0F94912F20E03F
:10F8900030E040E751E40F94DD2DA50194010F9471
:10F8A000E32C6B017C018090F7049090F804A09009
:10F8B000F904B090FA0420E030E040E85FE3C501CD
:10F8C000B4010F94432F1816F4F4C501B4010F943A
:10F8D0004F2E4B015C0160E070E0CB01181419045D
:10F8E0001A041B0434F40F944A21A50194010F94C7
:10F8F000792C0F941A269B01AC01B601C7010F9415
:10F90000E32C6B017C01C158DF4F2881CF57D040D9
:10F91000C058DF4F3881C058D040CF57DF4F4881A3
:10F92000C158D040CE57DF4F5881C258D040B601A1
:10F93000C7010F94132687FF2BC0A4960FAFA4977F
:10F94000C457DF4F3881CC58D040A8963FAFA89716
:10F95000EC96CFAEEC97ED96DFAEED97EE96EFAE70
:10F96000EE97EF96FFAEEF97C158DF4FC882CF57A3
:10F97000D040C058DF4FD882C058D040CF57DF4F5B
:10F98000E882C158D040CE57DF4FF882C258D040ED
:10F990000F5F1F4F0530110509F0B9CE4FEF241A44
:10F9A000340A55E02516310409F083CEA4968FADB4
:10F9B000A497E82FF0E0EE50FB4F208181E090E02B
:10F9C000A0E0B0E0A8960FACA89704C0880F991FDC
:10F9D000AA1FBB1F0A94D2F7822B8083A8969FADE3
:10F9E000A8976A969FAF6A97A496AFADA4976B96B7
:10F9F000AFAF6B97EC968FADEC97ED969FADED9713
:10FA0000EE96AFADEE97EF96BFADEF976F968CAFDA
:10FA10009DAFAEAFBFAF6F97A896BFADA897BF3FE2
:10FA200009F409C2A496EFADA497EF3F09F403C20D
:10FA30006B2FBB0F770B880B990B0F941A26209115
:10FA4000CA053091CB054091CC055091CD050F945E
:10FA500079262091C2053091C3054091C40550918B
:10FA6000C5050F94E32C162F072F382E292E862F2D
:10FA7000902FA32DB22D65968CAF9DAFAEAFBFAFCB
:10FA80006597A496FFADA4976F2FFF0F770B880B98
:10FA9000990B0F941A262091CE053091CF054091F5
:10FAA000D0055091D1050F9479262091C60530914B
:10FAB000C7054091C8055091C9050F94E32C6B010F
:10FAC0007C016996CCAEDDAEEEAEFFAE6997CE019D
:10FAD0008F5A9F4F0E942F1E882309F4B0C120E047
:10FAE00030E040EA50E4612F702F832D922D0F9467
:10FAF000E32C4B015C01CB01D50121968CAF9DAF6E
:10FB0000AEAFBFAF21972596CCAEDDAEEEAEFFAE69
:10FB10002597A8962FADA8972111E3C1A4963FADD4
:10FB2000A4973111B3C120E030E040EA50E4C701AE
:10FB3000B6010F94E32C6B017C01A4964FADA49702
:10FB4000442309F4C5C1A4968FADA49784300CF06A
:10FB5000BFC122ED422E23E5522E2BE7622E21E477
:10FB6000722E21968CAC9DACAEACBFAC2197259685
:10FB70008CAD9DADAEADBFAD2597A7968CAF9DAFBB
:10FB8000AEAFBFAFA7979C01AD0169966CAD7DADDF
:10FB90008EAD9FAD69970F94E22CAB966CAF7DAFA5
:10FBA0008EAF9FAFAB97A501940165966CAD7DAD0F
:10FBB0008EAD9FAD65970F94E22C2D966CAF7DAF07
:10FBC0008EAF9FAF2D97AB962CAD3DAD4EAD5FADDB
:10FBD000AB9761962CAF3DAF4EAF5FAF6197A5017C
:10FBE000940160911C0C70911D0C80911E0C9091E1
:10FBF0001F0C0F94E22C4B015C01A7962CAD3DAD80
:10FC00004EAD5FADA7976091200C7091210C809153
:10FC1000220C9091230C0F94E22CA7966CAF7DAF31
:10FC20008EAF9FAFA797812F902FA32DB22D8DA7B9
:10FC30009EA7AFA7B8ABC9AADAAAEBAAFCAAC98447
:10FC4000DA84EB84FC84CDAADEAAEFAAF8AE2DEC10
:10FC50003CEC4CEC5CE3C301B2010F9479262981A2
:10FC60003A814B815C810F9479262091280C309148
:10FC7000290C40912A0C50912B0C0F94E32C69AF66
:10FC80007AAF8BAF9CAFA5019401C501B4010F946D
:10FC900079264B015C01A7962CAD3DAD4EAD5FAD15
:10FCA000A797CA01B9010F9479269B01AC01C50140
:10FCB000B4010F94E32C20E030E040E050E40F94D6
:10FCC000432F1816ACF420E030E040E05FE3C701BA
:10FCD000B6010F94E32C29966CAF7DAF8EAF9FAF2A
:10FCE0002997BE01635C7F4FCE0101960E945A7432
:10FCF00089859A85AB85BC8529968CAF9DAFAEAFC3
:10FD0000BFAF2997A3961CAE1DAE1EAE1FAEA39724
:10FD1000BE01615A7F4FCE01CD960E94B7748CA56B
:10FD20008823C1F02AE939E949E95FE36D817E81E1
:10FD30008F8198850F947926A3966CAF7DAF8EAF97
:10FD40009FAFA397BE01615A7F4F88E697E00E945C
:10FD5000B7741CA6E090560CF090570C0091580C0C
:10FD60001091590CA090520CB090530CC090540CB0
:10FD7000D090550C9501A601B701C8010F94432FEF
:10FD8000181614F475018601809041029090420289
:10FD9000A0904302B09044022DEC3CEC4CEC5DE3AF
:10FDA000B701C8010F947926609341027093420213
:10FDB000809343029093440240E0BE01675B7F4F13
:10FDC000CE018D960F944B1580E1ECE1FCE0A8E6A6
:10FDD000B7E001900D928A95E1F7809241029092EE
:10FDE0004202A0924302B092440220E04FEFBE01D3
:10FDF000675A7F4FCE0101960E94327620E041E0A3
:10FE0000BE01675A7F4FCE0101960E9432762FEFD6
:10FE100040E0BE01675A7F4FCE0101960E943276C4
:10FE200021E040E0BE01675A7F4FCE0101960E945B
:10FE300032760E94A5618091990C80939A0CAD96C0
:10FE40004EAD5FADAD9741505109AD965FAF4EAF2E
:10FE5000AD97452B09F419CB6A968FAD6A9787FD4C
:10FE600014CB6B968FAD6B9787FFE1CB0ECB2BA19D
:10FE70003CA14DA15EA1E5962CAF3DAF4EAF5FAF6B
:10FE8000E5978FA198A5A9A5BAA5EBCB812F902FB7
:10FE9000A32DB22D21968CAF9DAFAEAFBFAF2197F2
:10FEA00020E030E040EA50E4C701B6010F94E22CB4
:10FEB00025966CAF7DAF8EAF9FAF2597A4965FADB3
:10FEC000A49754300CF42FCE182D092D3A2C2B2C3E
:10FED00092ED492E93E5592E9BEF692E90E4792EF1
:10FEE00040CEA8969FADA89794300CF452C0A4962B
:10FEF000AFADA497A4300CF120E030E040EA50E42C
:10FF0000612F702F832D922D0F94E22C21966CAFD0
:10FF10007DAF8EAF9FAF219720E030E040EA50E404
:10FF2000C701B6010F94E22C6B017C01A496EFADE2
:10FF3000A497E4300CF40DCECBCF812F902FA32DBE
:10FF4000B22D21968CAF9DAFAEAFBFAF219720E011
:10FF500030E040EA50E4C701B6010F94E32C259647
:10FF60006CAF7DAF8EAF9FAF2597A496BFADA49722
:10FF7000B111D2CF20E030E040EA50E4612F702F81
:10FF8000832D922D0F94E22C162F072F382E292E19
:10FF90009FCFA496FFADA497F1110DC020E030E0F3
:10FFA00040E251E4B401C5010F94E22C162F072F53
:10FFB000382E292ECECDA4962FADA49724309CF0B8
:10FFC00020E030E040E251E4B401C5010F94E22C9E
:10FFD00021966CAF7DAF8EAF9FAF2197182D092D65
:10FFE0003A2C2B2CB6CD182D092D3A2C2B2C82ED2A
:10FFF000482E83E5582E8BEF682E81E4782EB1CD04
:020000021000EC
:100000002F923F924F925F926F927F928F929F9228
:10001000AF92BF92CF92DF92EF92FF920F931F9316
:10002000CF93DF93CDB7DEB7EE970FB6F894DEBF70
:100030000FBECDBF80912D0C888B87E50E94701E6E
:10004000882309F423C120E030E0A9016091CA05AA
:100050007091CB058091CC059091CD050F9413261E
:10006000811108C00E942F4E8DE09DE00E946038F3
:1000700010E01FC18AE50E94BE1E882339F10E944C
:10008000C4242091CC083091CD084091CE085091E5
:10009000CF080F94E22C6B017C0120E030E040E2BD
:1000A00051ECC701B6010F94432F87FD0AC020E031
:1000B00030E040E251E4C701B6010F941326181650
:1000C00074F40E942F4E80E09DE0D0CFC090240CAD
:1000D000D090250CE090260CF090270CDECF40E06D
:1000E00050E060EC7FE788E50E94EE242091C40890
:1000F0003091C5084091C6085091C7080F94E22C72
:100100002B013C0140E050E060EC7FE789E50E9474
:10011000EE242091C8083091C9084091CA08509136
:10012000CB080F94E22C4B015C016FEF89E40E9435
:100130008024182F6FEF8AE40E948024082FA301E7
:100140009201C301B2010F94D52F81116EC0A50198
:100150009401C501B4010F94D52F811166C08BA104
:100160009CA1ADA1BEA18BAB9CABADABBEAB2091B6
:10017000C2053091C3054091C4055091C505C30126
:10018000B2010F94E22C2B013C0120E030E040E072
:100190005FE36BA97CA98DA99EA90F9479269B0189
:1001A000AC01C301B2010F94E32C2BA93CA94DA9CA
:1001B0005EA90F94DD2D0F944F2E162F4FA058A43B
:1001C00069A47AA42091C6053091C7054091C8055D
:1001D0005091C905C501B4010F94E22C4B015C019B
:1001E00020E030E040E05FE3C301B2010F947926E4
:1001F0009B01AC01C501B4010F94E32CA301920152
:100200000F94DD2D0F944F2E062F812F012E000C01
:10021000990B97FD33C005979CF5802F002E000C9D
:10022000990B97FD2FC005977CF5153008F020CF6E
:10023000053008F01DCF80E00E943E6995E019026C
:10024000F0011124E00FF11D07FDFA95EE0FFF1FDD
:10025000EE0FFF1FEC57F84FC082D182E282F3828B
:10026000602F812F0E9434F888890E943E69888916
:10027000882309F4FDCE0E94C230FACE10E0CDCF23
:1002800014E0CBCF00E0D1CF04E0CFCF8AE40E94CE
:10029000701E182F811127C070E060E086E50E9473
:1002A000B5249A838983059708F18BED9CE00E9421
:1002B0006038812FEE960FB6F894DEBF0FBECDBF2B
:1002C000DF91CF911F910F91FF90EF90DF90CF9032
:1002D000BF90AF909F908F907F906F905F904F9066
:1002E0003F902F9008950E941C6FC2CE60E084E47E
:1002F0000E949C248F8740E050E0BA018AE50E946A
:10030000EE246BA77CA78DA79EA740E050E86BE387
:1003100076E483E50E94EE2420E030E040E752E4FA
:100320000F94DD2D60933D0270933E0280933F0257
:1003300090934002E0907912F0907A12D7018D905C
:100340009D90AD90BC9020E030E0A901C501B401C2
:100350000F94E32C6BAF7CAF8DAF9EAF20E030E00D
:1003600040E450E40F94132687FF06C01BAE1CAE7A
:10037000B0E4BDAFE0E4EEAF20E030E041EE53E4A6
:10038000C501B4010F94E32C662E7BAB8FAB98AF05
:1003900020E030E84FED53E40F94432F18163CF45F
:1003A000612CF0E8FBAB2FED2FAB33E438AFD70176
:1003B00014968D909D90AD90BC90179720E030E002
:1003C000A901C501B4010F94E32CD62EE72EF82E17
:1003D000092F20E030E040E951E40F94132687FF15
:1003E00005C0D12CE12CF0E9FF2E01E420E030E043
:1003F00041EE53E4C501B4010F94E32CB62EC72E91
:1004000089AF9AAF20E030E048ED53E40F94432FDA
:10041000181634F4B12CC12CB8EDB9AFE3E4EAAF4F
:1004200088E40E94701E882309F416C20E94C42426
:100430000F944F2E1B0177FF02C06F5F7F4F7595A2
:1004400067957195619571096F517F4F072E000C6B
:10045000880B990B0F941A26762E872E982EA92E8C
:100460002D2D3E2D4F2D502F0F94432F18161CF479
:10047000D72C74010A2D2BAD3CAD4DAD5EAD672D73
:10048000782D892D9A2D0F94432F181624F07BACCC
:100490008CAC9DACAEAC872D982DA92DBA2D8B8B35
:1004A0009C8BAD8BBE8B8D2D9E2DAF2DB02F8F8B4A
:1004B000988FA98FBA8FB101330C880B990B0F94C9
:1004C0001A261B012C01AC019B016D2D7E2D8F2D59
:1004D000902F0F94E32CD62EE72EF82E092F2B2DDC
:1004E0003C2D49AD5AAD0F94132687FF04C0BD2C97
:1004F000CE2CF9AE0AAFA2019101672D782D892D7E
:100500009A2D0F94E32CD62EE72EF82E092F262DA8
:100510003BA94FA958AD0F94132687FF04C06D2C3B
:10052000EBAAFFAA08AF862D9BA9AFA9B8AD8B8F08
:100530009C8FAD8FBE8F8B2D9C2DA9ADBAAD8F8FAB
:1005400098A3A9A3BAA3BE01695E7F4FCE014396CB
:100550000E94622E882309F4B0C1BE01615E7F4F04
:10056000CE014B960E94622EE82E882309F4A5C185
:100570002F89388D498D5A8D6F8D78A189A19AA1C7
:100580000F94E22C20E030E040E85EE30F947926FF
:100590004B015C012B893C894D895E896B8D7C8D7B
:1005A0008D8D9E8D0F94E22C20E030E040E85EE3DC
:1005B0000F9479266BA37CA38DA39EA38FA298A6EC
:1005C000A9A6BAA689819A811816190674F489EA2F
:1005D0009CE00E9460388F85882321F08FE99CE0A1
:1005E0000E9460388AE00E9427380E94A5610E941C
:1005F000051D80E00E943E6980E090E0A0E2B1E449
:100600008FA798ABA9ABBAAB60E0CE018F960E94E2
:10061000F8642091CA053091CB054091CC055091EA
:10062000CD056BA17CA18DA19EA10F9413268111F4
:1006300030C02091CE053091CF054091D00550912A
:10064000D1056FA178A589A59AA50F9413268111CC
:1006500020C02091C2053091C3054091C40550913E
:10066000C5056B897C898D899E890F94132681111C
:1006700010C02091C6053091C7054091C805509122
:10068000C9056F89788D898D9A8D0F9413268823DB
:10069000A9F00E941C6F88E0FE01B396AAECB5E0B9
:1006A00001900D928A95E1F788E0FE017396A2EC25
:1006B000B5E001900D928A95E1F7188A60E085E433
:1006C0000E949C24882309F4FBC0F1E0FBAB1B864D
:1006D0001C861D861E861A8A9E2C4FE6C42E4CE070
:1006E000D42E5DE7A52E5CE0B52E1A8915300CF0EE
:1006F000F7C06B857C858D859E859B01AC010F9431
:10070000D52F8111EDC0992009F4DDC031E03FAB58
:1007100035E0232E91E09926F12EFF0CFF0CF10E0F
:10072000F394898B19896A89121509F4D5C0062EAC
:10073000000C770B880B990B0F941A262FA138A564
:1007400049A55AA50F9479262F89388D498D5A8D40
:100750000F94E32C2B013C01612F110F770B880BB9
:10076000990B0F941A262BA13CA14DA15EA10F94C9
:1007700079262B893C894D895E890F94E32C6B8304
:100780007C838D839E834F82588669867A86898191
:100790009A81892B79F06F2D8BE89CE00E9434417F
:1007A00069E170E089E89CE00E945E4186E89CE097
:1007B0000E9460381F9299E19F931F92FF92DF92EF
:1007C000CF92BF92AF921F920E945FF929814BA9ED
:1007D000BE01695F7F4FCE0103960E94D0F92B01C5
:1007E0003C014B865C866D867E860FB6F894DEBF34
:1007F0000FBECDBFAC019B010F94D52F811169C0F5
:1008000089883A8825E0382D320380011124030DB0
:10081000111D37FC1A95000F111F000F111F0C57E7
:10082000184FA30192016BA57CA58DA59EA50F94E1
:10083000E32CD8016D937D938D939C931397632D37
:10084000882D0E9434F8188A81E00E943B5AF39464
:100850008989BFA98B0F65CF4D2D5E2D6F2D702F10
:1008600086E40E94EE241B012C014BAD5CAD6DAD06
:100870007EAD8CE40E94EE246B8B7C8B8D8B9E8BEB
:100880002F8A388E498E5A8E4B2D5C2D69AD7AADEC
:1008900082E40E94EE246B017C01462D5BA96FA9C6
:1008A00078AD82E50E94EE246B8F7C8F8D8F9E8FBA
:1008B000CF8ED8A2E9A2FAA246CE8FEB9CE0F7CC6D
:1008C00022E02BAB04CF8FEF8FAB22242A9484E05D
:1008D00021CF88890E943E698A898F5F8A8B05CFE4
:1008E0000E94CAE40E94CE65882359F088890E943C
:1008F0003E6980E090E0A0ECBFE78B879C87AD87E6
:10090000BE876B857C858D859E859B01AC010F9490
:10091000D52F811159C08F85811126C082E0F82E14
:1009200002E094E0C92E12E0DC2CD11A21E041E073
:10093000612F802F0E949D2221E04FEF612F8F2D8C
:100940000E949D222FEF41E06D2D802F0E949D225D
:100950002FEF4FEF6D2D8F2D0E949D22115020F70C
:100960000150F3940F3FF9F60E94A5400E94CB1E60
:100970008F85811124C084E29CE00E94B51D4B014B
:100980005C018CE19CE00E945B1F9B01AC01C501F6
:10099000B4010F9479269B01AC016091240C7091F5
:1009A000250C8091260C9091270C0F94E22C6093DB
:1009B000240C7093250C8093260C9093270C8F8524
:1009C0008111E888E0922D0C0E94EC1C80912D0C86
:1009D00081110E94282B0E94B8670E94C2306B854B
:1009E0007C858D859E8511E09B01AC010F94D52FF0
:1009F00081115FCC3DCB8F929F92AF92BF92CF92ED
:100A0000DF92EF92FF920F931F93CF93DF9300D06B
:100A10001F92CDB7DEB75C016B017A01122F002364
:100A2000E1F10E94334E88E999E00E94603861E06C
:100A3000812F0E94543A90900C0583E080930C051E
:100A400081E080931B0C0E944B4082E080938611D2
:100A500040E368E879E084E799E00E94504040E094
:100A600069E171E18DE699E00E94504061E088E61D
:100A700099E00E9432408AE799E00E9459228091D1
:100A80001B0C882341F060E0812F0E94543A81E0E2
:100A90000E943B5AF4CF90920C0520E030E0A9016F
:100AA000F50160817181828193810F9413268823DF
:100AB00071F080E090E0A0ECB0E489839A83AB838E
:100AC000BC83BE016F5F7F4FC5010E947E6820E03E
:100AD00030E0A901F60160817181828193810F94D8
:100AE0001326882351F18090660C9090670CA0909B
:100AF000680CB090690C80E090E0A0E7B1E48093CE
:100B0000660C9093670CA093680CB093690C80E01E
:100B100090E0A0EAB1E489839A83AB83BC83BE01F1
:100B20006F5F7F4FC6010E947E688092660C909234
:100B3000670CA092680CB092690C20E030E0A9012B
:100B4000F70160817181828193810F94432F181680
:100B500074F480E090E0A0E4B0E489839A83AB83EE
:100B6000BC83BE016F5F7F4FC7010E947E6880918A
:100B7000E10429E131E1882311F029E439E047E576
:100B800059E061E679E081E00E9473400E944B40A9
:100B900081E00F900F900F900F90DF91CF911F91F8
:100BA0000F91FF90EF90DF90CF90BF90AF909F900C
:100BB0008F900895CF93C82F8091DA0B83FD14C0D6
:100BC0008091F708811110C080915F0290916002BE
:100BD0009C01215031094091E2115091E3114217DB
:100BE000530714F40E94461FCC2329F061E080E0F3
:100BF000CF910C94FDBC8091F70891E089278093F8
:100C00003C0280913C02882389F08091E011909110
:100C1000E1112091E2113091E311821B930B97FFB8
:100C200003C0919581959109029744F410923C027A
:100C30008091DA0B83FF06C0C1E01AC080E00E94F9
:100C40003B5ADFCFC091F708C11112C080915F02FB
:100C50009091600201972091E2113091E3112817E1
:100C6000390754F70E94334E8BE299E00E946038B6
:100C70008C2FCF910895AF92BF92CF92DF92EF92D7
:100C8000FF920F931F93CF93DF93CDB7DEB7649797
:100C90000FB6F894DEBF0FBECDBF0E94324F87FD66
:100CA000AFC08AE50E94BE1E882309F4BAC040E0A6
:100CB00050E0BA018AE50E94EE247B018C0120916C
:100CC000240C3091250C4091260C5091270C60E0AB
:100CD00070E08BEE93E40F94E22C5B016C019701C2
:100CE000A8010F94432F181614F07501860120E017
:100CF00030E0A901B701C8010F94432F181624F45E
:100D0000E12CF12C00E010E0B701C8010F944F2E48
:100D1000072E000C880B990B0F941A26698B7A8B7F
:100D20008B8B9C8B20E030E0A9010F941326882345
:100D300021F0CE0141960E94FC7280E090E0A0EA92
:100D4000B1E48D879E87AF87B88B19861A861B867C
:100D50001C868CE40E94701E882309F467C00E94E0
:100D6000C4246B017C0120E030E0A901C701B60179
:100D70000F94432F87FF04C0F7FAF094F7F8F0942C
:100D8000CD82DE82EF82F8862091E2113091E3116C
:100D90002430310574F08091E0119091E111821BB3
:100DA000930B97FF03C091958195910901E00497FA
:100DB0000CF400E080E00E94DA85882359F022E0FC
:100DC000AE01435F5F4FBE016B5F7F4FCE0109965F
:100DD0000E94FB8469897A898B899C898B019C019B
:100DE000305809831A832B833C8320E030E0A9012B
:100DF0000F941326882321F0CE0101960E94FC72E5
:100E000064960FB6F894DEBF0FBECDBFDF91CF91D1
:100E10001F910F91FF90EF90DF90CF90BF90AF9018
:100E20000895E12CF12C00E211E449CFC090BD05FA
:100E3000D090BE05E090BF05F090C00594CF7F92A2
:100E40008F929F92AF92BF92CF92DF92EF92FF92DA
:100E50000F931F93CF93DF9300D000D01F921F9268
:100E6000CDB7DEB76C015B014A01722E78010091AB
:100E70000A060E94521F8091E2119091E3118E1593
:100E80009F051CF4C7010E94461F80E00E94DA857E
:100E9000882331F0272DA401B501C6010E94FB84EF
:100EA0001E141F043CF4C7010E94461F60E080E04E
:100EB0000E94FDBC81E00E94DA8580E090E0A0E71E
:100EC000B2E489839A83AB83BC8380E090E0A0E89E
:100ED000B0EC8D839E83AF83B887BE016F5F7F4F79
:100EE000CE0105960E947E6887E00E943F2A81110C
:100EF00058C08091240C9091250CA091260CB091A3
:100F0000270C4091E6045091E7046091E804709149
:100F1000E904C090E204D090E304E090E404F0908F
:100F2000E504C0926807D0926907E0926A07F092E0
:100F30006B0740936C0750936D0760936E07709337
:100F40006F078093700790937107A0937207B09317
:100F5000730780E090E0A8E4B2E489839A83AB83CE
:100F6000BC83CE0101960E9495728091EA04909113
:100F7000EB04A091EC04B091ED0480937007909382
:100F80007107A0937207B093730780E090E0A0EA26
:100F9000B0E489839A83AB83BC83CE0101960E941F
:100FA0009572C12CD12C80E7E82E82E4F82EC982FC
:100FB000DA82EB82FC8280E090E0A0E8B0E48D83EE
:100FC0009E83AF83B887BE016F5F7F4FCE010596CA
:100FD0000E947E6820E030E0A9016091EE047091EB
:100FE000EF048091F0049091F1040F94132687FF91
:100FF0000BC0C982DA82EB82FC82BE016F5F7F4F39
:101000008EEE94E00E947E688091EE049091EF0451
:10101000A091F004B091F1048093280C9093290CD6
:10102000A0932A0CB0932B0C8093740790937507B0
:10103000A0937607B093770784E797E00E94B661A4
:101040008091C10581110E947AF761E087EB99E0F8
:101050000E949B3F8091181181508093181146E6A1
:1010600058E16FEB79E085E00E944FE38091181121
:10107000882339F00E9436AB8091181181508093FB
:10108000181180E00E9441F90E94BC318091191131
:10109000823011F40E946E380E94CAE428960FB67E
:1010A000F894DEBF0FBECDBFDF91CF911F910F919E
:1010B000FF90EF90DF90CF90BF90AF909F908F9078
:1010C0007F900895CF92DF92EF92FF920F931F933C
:1010D000CF93DF9300D01F92CDB7DEB77C016B01B9
:1010E0008A0161E08CE399E00E949B3F46E658E16B
:1010F00063E479E085E00E944FE39091181181E06C
:10110000890F809318118091261482FF06C08B7F6F
:10111000809326149E5F909318110E94603980E19D
:10112000ECE1FCE0A2EEB4E001900D928A95E1F7CB
:101130000E94A56181E00E9441F920E030E0A90110
:10114000F70160817181828193810F941326882336
:10115000F1F08091F70881110CC080915F029091AD
:10116000600201972091E0113091E11128173907B1
:1011700074F080E090E0A0E7B2E489839A83AB83C7
:10118000BC83BE016F5F7F4FC7010E947E6887E00E
:101190000E943F2A811103C0B6010E94D26720E05D
:1011A00030E0A901F80160817181828193810F94FF
:1011B0001326882341F080E00E94DA85882319F005
:1011C000C8010E94AE68129A64E670E080E090E088
:1011D0000E94322681E00F900F900F900F90DF91C8
:1011E000CF911F910F91FF90EF90DF90CF900895D6
:1011F000CF92DF92EF92FF92CF93DF936B017C014E
:10120000D42FC0910C0583E080930C0581E080937E
:101210001B0CC114D104E104F10431F00E9472FDF1
:10122000C60ED71EE81EF91E80911B0C882389F07C
:10123000C114D104E104F10421F48D2F0E943B5A22
:10124000F3CF0E9472FD6C197D098E099F0997FDED
:10125000F4CF10921B0CC0930C05DF91CF91FF903F
:10126000EF90DF90CF9008950F931F93CF93DF936C
:10127000C82F162F0E94334EC11194C0CFE8D8E07A
:10128000CE010E94603861E0812F0E94543A0E9492
:1012900072FD685370458F4F9F4F609306067093A1
:1012A0000706809308069093090610920A0600919B
:1012B0000C0583E080930C0530E020E049E151E12A
:1012C0006DE179E082E00E9473408DE199E00E9437
:1012D000592281E080931B0C80911B0C882309F418
:1012E00064C060E0812F0E94543A80910A068823EE
:1012F00009F454C00E94334E83E099E00E946038A4
:1013000030E020E04DEE58E064EF78E082E00E94AB
:10131000734084EF98E00E94592241E060E070E061
:10132000CB010E94F88830E020E050E040E060EE21
:1013300078E085E00E94734080EE98E00E94C3351B
:101340000E94521F80E00E94DA850E94334ECE0137
:101350000E9460380E9472FD685370458F4F9F4F06
:10136000609306067093070680930806909309061B
:1013700010920A0630E020E049E151E164ED78E0A6
:1013800082E00E94734083EC98E00E94592281E041
:1013900080931B0C61E0812F0E94543A81E00E94EF
:1013A0003B5A9ACFC4EAD8E06BCF00930C05DF918B
:1013B000CF911F910F910895CF92DF92EF92FF92FC
:1013C0000F931F93CF93DF93CDB7DEB7A0970FB6E0
:1013D000F894DEBF0FBECDBF0E94324F87FDCCC058
:1013E00085E40E94701E882309F4D5C00E94C4249D
:1013F0006B017C0120E030E0A9010F94432F87FFAF
:1014000004C0F7FAF094F7F8F094F7FAF094F7F8CC
:10141000F094CD8EDE8EEF8EF8A28CE0E4ECF2E05C
:10142000DE01119601900D928A95E1F78AE50E94FE
:10143000BE1E882351F040E050E0BA018AE50E94C8
:10144000EE2469877A878B879C8788E50E94BE1E79
:10145000882351F040E050E0BA0188E50E94EE2474
:1014600069837A838B839C8389E50E94BE1E8823CF
:1014700051F040E050E0BA0189E50E94EE246D830E
:101480007E838F83988785E50E94701E882309F4E8
:1014900089C00E94C4246B017C0120E030E0A901D6
:1014A000C701B6010F94432F87FF04C0F7FAF094E9
:1014B000F7F8F094F7FAF094F7F8F094C98EDA8E12
:1014C000EB8EFC8E1D8A1E8A1F8A188E8CE40E9469
:1014D000701E882309F46FC00E94C4246B017C0134
:1014E00020E030E0A901C701B6010F94432F87FF28
:1014F00004C0F7FAF094F7F8F094C98ADA8AEB8A14
:10150000FC8A62E070E082E40E94B524F82E8091AB
:101510001811811131C021E0AE01475E5F4FBE015D
:101520006F5F7F4FCE014D960E946288882321F124
:101530006F2D81E00E94348982E50E94BE1E8823BF
:1015400009F442C00E94B12440E050E060EA71E436
:101550004D875E876F87788B20911811222361F069
:101560008C012F2DAE01435F5F4FBE016F5E7F4F39
:10157000CE0145960E941F87A0960FB6F894DEBF55
:101580000FBECDBFDF91CF911F910F91FF90EF90D4
:10159000DF90CF900895C12CD12C80E8E82E80E414
:1015A000F82E33CFC090B905D090BA05E090BB05B6
:1015B000F090BC0572CFC090BD05D090BE05E09004
:1015C000BF05F090C0058CCF90E080E0BDCFCF92FA
:1015D000DF92EF92FF920F931F93CF93DF93CDB7DC
:1015E000DEB76C970FB6F894DEBF0FBECDBF8CE4AC
:1015F0000E94701E882309F4B0C00E94C4246B01AD
:101600007C0120E030E0A9010F94432F87FF04C044
:10161000F7FAF094F7F8F094F7FAF094F7F8F094FA
:10162000C98EDA8EEB8EFC8E8CE0E4ECF2E0DE010B
:10163000119601900D928A95E1F788E50E94BE1EF1
:101640008823A1F040E050E0BA0188E50E94EE2432
:101650002091C4083091C5084091C6085091C70830
:101660000F94E22C69837A838B839C8389E50E94A3
:10167000BE1E8823A1F040E050E0BA0189E50E9437
:10168000EE242091C4083091C5084091C6085091BD
:10169000C7080F94E22C6D837E838F8398878AE539
:1016A0000E94BE1E882351F040E050E0BA018AE556
:1016B0000E94EE2469877A878B879C871D861E8609
:1016C0001F86188A80911811811138C020E0AE0160
:1016D000435F5F4FBE016F5F7F4FCE0149960E940F
:1016E0006288882359F18091C10581110E947AF79F
:1016F00060E080E00E943489898D9A8DAB8DBC8D2D
:10170000B0588D8B9E8BAF8BB88F198A1A8A1B8A23
:101710001C8A1D861E861F86188A809118118823B0
:1017200069F010E000E020E0AE014B5E5F4FBE01CB
:101730006F5E7F4FCE010D960E941F876C960FB68D
:10174000F894DEBF0FBECDBFDF91CF911F910F91F7
:10175000FF90EF90DF90CF900895C12CD12C80E8BE
:10176000E82E80E4F82E58CF2F923F924F925F924E
:101770006F927F928F929F92AF92BF92CF92DF92A1
:10178000EF92FF920F931F93CF93DF93CDB7DEB706
:10179000E5970FB6F894DEBF0FBECDBF8DAB20919D
:1017A0000C052CAB21E020930C0580912A058D348B
:1017B00009F405C6843511F40C9407A1873409F0A7
:1017C00091C180912805909129058B31910509F4EB
:1017D000DDC108F079C18430910508F030C1209155
:1017E000DD068230910508F48EC1213009F091C1E7
:1017F00011E0029709F010E00E94052519821A8273
:101800001B821C821D821E821F82188682E50E9416
:10181000BE1E882309F490C10E94C4246B017C0180
:1018200020E030E0A9010F941326882309F4EAC0D0
:1018300040901C0C50901D0C60901E0C70901F0C62
:101840008091200C9091210CA091220CB091230C3E
:101850008CA79DA7AEA7BFA7809068079090690747
:10186000A0906A07B0906B0780916C0790916D070C
:10187000A0916E07B0916F0788AB99ABAAABBBABD9
:10188000A5019401C301B2010F94132681110DC06B
:1018900028A939A94AA95BA96CA57DA58EA59FA5F4
:1018A0000F941326882309F4ADC0A3019201C5014A
:1018B000B4010F94E22C20E030E040E05FE30F94AD
:1018C000792668A779A78AA79BA72CA53DA54EA531
:1018D0005FA568A979A98AA99BA90F94E22C20E0A9
:1018E00030E040E05FE30F9479262B013C0120E0DB
:1018F00030E0A901C701B6010F941326881F88277D
:10190000881F181709F40FC180E090E0A0E8BFEB32
:101910008CA79DA7AEA7BFA728A539A54AA55BA5FB
:10192000CA01B9010F9479264B015C01A301920110
:10193000C301B2010F9479269B01AC01C501B4012A
:101940000F94E32C0F94912F4B015C01AC019B0190
:10195000C701B6010F94E22C68AB79AB8AAB9BABA5
:10196000A5019401C701B6010F94E32C9B01AC01C2
:1019700068A979A98AA99BA90F9479266B017C0192
:1019800020E030E0A9010F94432F87FDD1C0C701AB
:10199000B6010F94912F6B017C01C301B2019058E5
:1019A000A50194010F94DD2D2CA53DA54EA55FA5A5
:1019B0000F947926A70196010F94792628A539A5B9
:1019C0004AA55BA50F94E32C69837A838B839C8360
:1019D000A501940168A579A58AA59BA50F94DD2D85
:1019E0002CA53DA54EA55FA50F947926A7019601CC
:1019F0000F947926A30192010F94E32C6D837E83CB
:101A00008F83988720E030E0A90169817A818B81FA
:101A10009C810F9413268111A3C020E030E0A9011E
:101A20006D817E818F8198850F941326811198C0D6
:101A30000E942F4E8BEB9FE00E9460386AC0853178
:101A4000910509F466C08A31910509F49CC0049798
:101A500009F048C080E50E94BE1EC12CD12C760141
:101A6000882321F00E943E246B017C0183E50E94C3
:101A7000BE1E882361F00E94C42420E030E04AE7C3
:101A800054E40F9479260F94562E6B017C010E942A
:101A9000A56180911A11811105C060E081ED9FE080
:101AA0000E94CE3F0E9472FDC60ED71EE81EF91E90
:101AB0000E9472FD6C197D098E099F0997FF29C04C
:101AC00080E00E943B5AF4CF8A32910509F4ECC2BF
:101AD00060F48D31910509F415C208F470C04E9779
:101AE00009F468C20E9493F914C08B35910509F47A
:101AF000BEC38C35910509F4BEC38A35910591F7B3
:101B00001092E80706C0213021F40E9405250E94AA
:101B1000E26F3DA9311102C00F94F8148CA9809393
:101B20000C050C94689980E090E0A0E8BFE3F0CE4B
:101B3000C12CD12C760131CF89E40E94BE1E8823AE
:101B400031F00E94C42469837A838B839C838AE466
:101B50000E94BE1E882309F455CF0E94C4244ECF94
:101B6000412FBE016F5F7F4F88E697E00F944B15C2
:101B70000E9472FD60936B1170936C1180936D11D4
:101B800090936E11C6CF0E94D177C3CF87E00E9499
:101B9000434E8111BECF8CE0E0EDF2E0DE01119604
:101BA00001900D928A95E1F770E060E080E50E9477
:101BB0005E24BE016F5F7F4F0E94D267AACF87E08D
:101BC0000E943F2A811106C060E08FE40E949C249D
:101BD00081119FCF0E94A5611092460260912D0C49
:101BE0008CE40E949C24E82E80E00E943E690E94C2
:101BF00072FD60936B1170936C1180936D119093D3
:101C00006E110E94051D81E0809399060E94972B1A
